:020000040801F1
:10000000285500200502010825650108195B010833
:1000100021650108F319010825A10108000000006D
:10002000000000000000000000000000C193010873
:100030008330010800000000C166010839990108F9
:10004000E5A10108B1660108319B01084D80010856
:10005000AD5301084D7E0108D9510108DD51010859
:10006000295201087552010879520108ED2E010844
:10007000EF2E0108F12E0108F32E0108F52E0108DC
:10008000F72E0108F92E01084B14010837A00108CA
:1000900039A00108FD190108FF190108C55201081E
:1000A000339B0108399B0108379B0108359B0108E8
:1000B0003B9B01083D9B01083F9B01081F5B01081A
:1000C0001D5B0108235B0108215B0108BB9301084C
:1000D000BD930108C59D0108C99D01086D9E0108D9
:1000E000DB5101081D7F010835A00108479B01086D
:1000F0004D9B01084B9B0108499B01084D140108C9
:10010000E1530108B9930108419B0108BF9301081D
:10011000C19D0108C39D0108439B0108459B01083F
:10012000FB2E0108FD2E0108FF2E0108012F0108FA
:1001300000F002F800F057F80AA090E8000C8244A2
:100140008344AAF10107DA4501D100F04CF8AFF27F
:10015000090EBAE80F0013F0010F18BFFB1A43F0A5
:1001600001031847FC5D02001C5E02000A4410F8FF
:10017000014B14F00F0508BF10F8015B240908BFFC
:1001800010F8014B6D1E05D010F8013B6D1E01F8F3
:10019000013BF9D1641E03D0641E01F8015BFBD161
:1001A0009142E4D37047000000230024002500267C
:1001B000103A28BF78C1FBD8520728BF30C148BFCA
:1001C0000B607047692900F06180002070471FB5FF
:1001D0009DE8030000F0F8FC00F082FE1FBD10B5A2
:1001E00000F0E7FE10BD00F01BFF1146FFF7EFFF28
:1001F0000CF074FB01F082F803B4FFF7F0FF03BCCE
:100200000AF02AFC0348004703480449044A054B06
:100210007047000031010108284B002028550020BC
:10022000285000202850002070470FB4014610B518
:1002300004AA039800F0A2FB10BC5DF814FB70B593
:10024000044685690068C10601D5302600E02026F5
:10025000C00707D070BDD4E9012130469047206A1D
:10026000401C20626D1EF6D570BD70B504468569D0
:100270000078C00707D170BDD4E901212020904744
:10028000206A401C20626D1EF6D570BD2DE9F0413C
:100290000646002410687529314616A510D0AFF324
:1002A0000080002802DA404213A507E031688A077F
:1002B00001D512A502E0490704D511A5012401E0EA
:1002C000AFF3008000210A2206F1240709E0B0FB09
:1002D000F2FCB0FBF2F302FB1C00303078541846FD
:1002E000491C0028F3D123462A463046BDE8F04198
:1002F00000F0EBBA000000002D0000002B00000011
:10030000200000002DE9F05F894604464FF0000A06
:10031000DFF824B1FB44C0F820A02046E1688847FC
:1003200000287DD0252806D0D4E901219047206AF5
:10033000401C2062F1E700255F462046E1688847BF
:100340002028064607DB312E05D2B81910F8200CFC
:1003500008B10543F1E7A80701D525F00405C4F865
:100360001CA00027C4F818A02A2E09D030460AF095
:1003700061FB38B304EB8708303EC8F8186019E019
:1003800059F8041B204604EB87029161E168884715
:10039000012F064618D1E069002820DA25F0200553
:1003A0001DE0D8F8180000EB800006EB4000303864
:1003B000C8F818002046E168884706460AF03AFB6C
:1003C0000028EED1012F0AD02E2E08D12046E16858
:1003D00088477F1C0646022F45F02005C4DBA06934
:1003E000002803DA404245F00105A061E80701D08A
:1003F00025F01005A6B1A6F14100192802D8203633
:1004000045F400654A463146204625604D46FFF7D3
:10041000D9FE60B1012807D0ED1D25F0070000E0EE
:1004200007E000F1080978E705F1040975E73046AF
:100430007AE7206ABDE8F09F3F3E02002DE9F041D7
:1004400017460D4604460646012913DD38460BF0D3
:10045000B9FC411C0CD0C0B20A2804F8010B02D030
:100460006D1E012DF2DC002020703046BDE8F081C9
:10047000B44201D10020F9E7384600F091FA002893
:10048000F1D00026EFE700002DE9F0410C460746C9
:100490001646104600F06EF82078611C61280AD0DC
:1004A000722802D077283CD102E00125002405E023
:1004B0000225042402E0082448F2020511F8010B89
:1004C0002B2806D0622809D011F8010C74280AD014
:1004D0000BE045F0030544F00204EFE745F00405A6
:1004E00044F00104EAE744F01004384621460AF0DB
:1004F000C9FA411C15D00021316171604FF40071BF
:10050000F560F1617061200704D5304602220021B8
:1005100000F04AFA306D40F0010030653046BDE829
:10052000F0810020FBE72DE9F0410D460646104C16
:10053000206DC10704D0410804D020F00104F7E782
:1005400022460EE0542000F06AF907000ED0206D1C
:1005500047F00101084354212065384600F0F4F8C3
:100560003A4629463046BDE8F0418DE70020D6E7FF
:10057000C84900202DE9F04704464FF000094FF02C
:10058000FF37C568D4E90486A80707D0204600F0E5
:10059000BBFA30460AF055FA002802DA3846BDE8C0
:1005A000F087280502D5404600F068F94C21204626
:1005B00000F0CAF8206D20F0010020654846EEE703
:1005C00010B5431C02E010F8011B71B18107FAD18C
:1005D0004FF0013202C88C1A8C4314EAC211F9D0D0
:1005E000C01A0A0603D0C01E10BDC01A10BD0A04EE
:1005F00001D0801E10BD0902FCD0401E10BD421E5D
:1006000012F8013F002BFBD111F8013B002B02F83F
:10061000013BF9D17047032A40F2308010F0030CFF
:1006200000F0158011F8013BBCF1020F624498BF45
:1006300011F801CB00F8013B38BF11F8013BA2F1E2
:10064000040298BF00F801CB38BF00F8013B11F05D
:10065000030300F02580083AC0F0088051F8043BFD
:10066000083A51F804CBA0E80810F5E7121D5CBF6A
:1006700051F8043B40F8043BAFF30080D20724BF9D
:1006800011F8013B11F801CB48BF11F8012B24BF31
:1006900000F8013B00F801CB48BF00F8012B704780
:1006A00010B5203AC0F00B80B1E81850203AA0E80D
:1006B0001850B1E81850A0E81850BFF4F5AF5FEA41
:1006C000027C24BFB1E81850A0E8185044BF18C9F4
:1006D00018C0BDE810405FEA827C24BF51F8043B9B
:1006E00040F8043B08BF7047D20728BF31F8023BEF
:1006F00048BF11F8012B28BF20F8023B48BF00F883
:10070000012B70474FF000020429C0F0128010F056
:10071000030C00F01B80CCF1040CBCF1020F18BFDD
:1007200000F8012BA8BF20F8022BA1EB0C0100F070
:100730000DB85FEAC17C24BF00F8012B00F8012B43
:1007400048BF00F8012B70474FF0000200B5134678
:1007500094469646203922BFA0E80C50A0E80C50E1
:10076000B1F12001BFF4F7AF090728BFA0E80C5092
:1007700048BF0CC05DF804EB890028BF40F8042B8B
:1007800008BF704748BF20F8022B11F0804F18BFF8
:1007900000F8012B704700004FF0013C50F8042B8B
:1007A00051F8043B9A4221D1A2EB0C03934313EA84
:1007B000CC1317D150F8042B51F8043B9A4215D1B1
:1007C000A2EB0C03934313EACC130BD150F8042B88
:1007D00051F8043B9A4209D1A2EB0C03934313EA6C
:1007E000CC13DBD04FF00000704700BFD01A01BA25
:1007F000B1FA81F101F0180122FA01F0CB40C1F108
:100800002001DBB2C0B2C01A2CFA01F3D11A914315
:1008100011EAC311E6D1704770477047704770B551
:10082000064600F0B5F9056806F10B0020F0070454
:10083000B4429CBF002070BD2B466A68BAB11068F4
:10084000A04210D304F1080188423CBF50685860B0
:1008500007D35168101941601168091B0160586085
:100860001460101D70BD13465268002AE7D121465E
:10087000284600F095F90028DED170BD70B5044619
:10088000051F00F085F90068002C14BF446870BD96
:10089000002C18BFAC423CBF20466468F8D3016806
:1008A0000A18AA4218BF456003D12A6805461144B8
:1008B000016028684119A1421CBF6C6070BD61686D
:1008C000696021680844286070BD2DE9F0470D4635
:1008D00099469246044600F124080168880604D52A
:1008E000E06921F01001216000E00120A84201DD53
:1008F000471B00E00027A1697A1902EB0900081ADA
:10090000A0612078C00602D42046FFF798FC00269C
:1009100008E0D4E901211AF806009047206A401C3B
:10092000761C20624E45F4DB2078C0060AD52046AE
:10093000FFF785FC06E0D4E9012130209047206ACA
:10094000401C2062381EA7F10107F4DC07E0D4E95F
:10095000012118F805009047206A401C2062281EDB
:10096000A5F10105F3DC2046FFF77FFC20780006A7
:1009700002D50220BDE8F0870120FBE7074B70B5E8
:100980000D467B4400F05BF90446284600F008F869
:1009900010B14FF0FF3070BD204670BDDBB40000D9
:1009A000007B00F0800070472DE9F04104461646B8
:1009B0000D464769007B80072ED038460AF059F86B
:1009C00050BB3EB3012E02D0022E25D104E02046BA
:1009D00000F065FA05441DE038460AF03FF8E1688A
:1009E000002841F01001E16005DA204600F058F8D7
:1009F0000120BDE8F081C9030BD56268E16A91422C
:100A000000D81146A26911442269891A814200DD89
:100A100008460544002D01DA0220EAE7E16A606831
:100A2000E268814206D29103E06203D522F40031EC
:100A300041F01002A6690027AE4213DCE16A814250
:100A400001D90B4600E0034603EB060C2369ACEB2F
:100A5000030CAC4506DD814201D98C4600E084469A
:100A60009C4505D1A760276042F02000A5620DE0FB
:100A7000AD1BE669AE1B8142A66000D90846C01ACC
:100A8000281A20605819606022F0200003490840AD
:100A9000E060002084F84870ABE70000BFCFD7FFCC
:100AA000C16821F4001141F08001C1600021816022
:100AB000016070472DE9F047814614460E464FF01D
:100AC000FF383248D5685769054209D03846A169D0
:100AD0000AF017F8002811DB2C48C0430540E560F8
:100AE0002B463246494638460AF019F8A16920F0EB
:100AF0000042B21A11440028A16103D02046FFF73A
:100B0000CFFF4046BDE8F08770B504460569C06A6E
:100B10006168884200D80846E16821F42011E1604C
:100B2000C90312D5A84208D02246411B2846FFF728
:100B3000C1FF10B14FF0FF3070BD0020E562C4E985
:100B40000150E06820F48030E060002070BD10B5F6
:100B50000446C06820F02000E060A16AA0698842D5
:100B60000DD02046FFF7D0FFE06820F4405040F061
:100B70001000E060A06AA0612069E062606044F259
:100B80004001E0688843E06010BD000010000200F2
:100B900000487047CC4A0020704770477047704744
:100BA00038B504460A4600206946AFF300800028A5
:100BB00008BF38BD02460099204600F05BFA0120CC
:100BC00038BD012000F0A7BBF8B5AFF300800546A3
:100BD00000200C46102000BF0646A819A0420DD9DF
:100BE000324669460020AFF30080070008BF00F0DE
:100BF00092FB0098A04218BF0546C419FFF7C8FF32
:100C000005600746F01D20F007004619284600F051
:100C10000AF8B44208BFF8BDA21B31463868BDE8E7
:100C2000F84000F027BA00210160C0E901107047C8
:100C30001020704701694A1C02610878704700B5AE
:100C40008FB0CDE901310021059105497944CDE905
:100C5000031011466846FFF755FB0FB000BD0000BA
:100C6000E5FFFFFF70B50D4601461446D368506995
:100C70002A4609F033FF002807DA411C07D0E16853
:100C800020F0004041F48041E160281A70BD204608
:100C9000FFF706FF4FF0FF3070BDC1680022026011
:100CA00021F4805141F0400111F4C06FC16001D0C6
:100CB0008260704702694168891AC269891A816035
:100CC00070472DE9F0470446C06840F48000E060BA
:100CD000010312D520F40020E060810606D4E26A08
:100CE00061688A4200D80A46511A216040F4001017
:100CF000E06094F82500BDE8F08720F40010E06083
:100D0000800602D52046FFF722FFE06842F281010B
:100D10004FF0FF390140012903D02046FFF7C0FE04
:100D2000B6E02168002600290ADAC94340F4805061
:100D30002160C4E902606068411C61600078DAE704
:100D400044F2400108420CD020F4A04040F04000A2
:100D50002660E06021696068401AE169401AA0607D
:100D600096E0216991B9C00310D4E069FFF757FDFF
:100D70002061B0B1E06840F4006010F4407FE060B2
:100D800002D140F48070E06020696060E068D4F8CF
:100D900014A0C1061AD5C0030ED52046FFF7B4FE35
:100DA00014E004F1240020610120E061E06820F4F7
:100DB000407040F48060E6E721696068401AA169EC
:100DC0000144504609F09DFE0028A6DBE068C00300
:100DD0002AD56168E06A884200D808462169451A28
:100DE000E069471B1BD02046D4F81880FFF78CFE23
:100DF00008EB05015046C4F8188009F082FE00286F
:100E00008BDBE06840F40030E060000202D5A069AE
:100E10002844A061E1692069C91B45180DE02046FE
:100E2000FFF772FEE769F5E725696168D4E906070F
:100E3000491BE56208446560A061E06820F010008D
:100E400010F4C06FE06002D0204600F03BFAE0688A
:100E500040F48050C4E90260000205D52069E062D8
:100E600060606FF0010046E7224639462846FFF7EA
:100E7000F9FE411C0CD02918E16258B1401E2060D7
:100E8000681C6060E06840F40030E060287832E779
:100E9000484630E765602046FFF7FFFEF8E710B5EB
:100EA0000146C268900703D0900607D5886A0AE019
:100EB00000F0DCF801210160881E10BD8B694868D4
:100EC00018440B69C01A91F848301BB191F84910C9
:100ED000401A10BD1103FCD50028FADD401E10BDDC
:100EE00010B542485421FFF72FFC41485421FFF729
:100EF0002BFC40485421FFF727FC3F493B483C4A24
:100F00003F4B08603D490A603A491960531C03652C
:100F1000481C1065012008653B48344A39A17844D3
:100F2000FFF7B2FA20B9384878440A3800F0ECF9F3
:100F300037482F4A35A17844FFF7A6FA20B934483C
:100F400078440A3800F0E0F932482A4A2FA1784460
:100F5000FFF79AFA20B92F4878440A3800F0D4F9FC
:100F600040232248DC000021224600F088F920B10D
:100F700025487844543800F0C7F91D4822464023DC
:100F8000002100F07CF920B121487844543800F069
:100F9000BBF9184822461023002100F070F9002800
:100FA00006D01C487844BDE81040563800F0ACB973
:100FB00010BD104870B5006D20F001040B48FFF71C
:100FC000D9FA0B48FFF7D6FA0A48FFF7D3FA09E037
:100FD000206D20F001052046FFF7CCFA2046FFF7F0
:100FE0004DFC2C46002CF3D170BD0000C8490020F8
:100FF0001C4A0020704A00208C0200209002002031
:101000009402002072000000A22A01007700000074
:10101000902A01007F2A010000487047C44A00203E
:101020007546FFF7F9FFAE4605006946534620F0C6
:101030000700854618B020B5FFF7E6F8BDE8204068
:101040004FF000064FF000074FF000084FF0000B84
:1010500021F00701AC46ACE8C009ACE8C009ACE837
:10106000C009ACE8C0098D467047000000487047D1
:10107000C44A0020034640688C46002818BF8842B6
:101080003CBF03464068F8D318681844884207D02C
:101090000CF1030020F00700001D411A521A01460E
:1010A000081D0A60FFF7EABB2DE9F04705460C462C
:1010B000C86820F4201040F48000C860800602D583
:1010C0000846FFF744FDE06841F282014FF0FF3926
:1010D0000140022903D02046FFF7E2FCB5E000F40E
:1010E0002041B1F5004F0FD1C00306D56168E06A19
:1010F000884200D80846606006E02069E0626060CF
:10110000606909F0ABFCA061A0680022EEB2002883
:101110000DDAE1688B050AD4C043A06041F4903039
:101120002260E0606068411C61600670A5E0E068D4
:101130009046226040F40050E060206968BB60691E
:1011400009F097FC012704F12405A0B1A08910F44F
:10115000407F08D0E069FFF762FB206118B1E068CA
:1011600040F4006016E0E7612561E06820F440701B
:1011700040F480600EE0E069FFF751FB0028206139
:10118000F1D0E06840F4006010F4407FE06002D1EC
:1011900040F48070E06020696060E06825696FF06D
:1011A000010AC1051FD56168E06A884200D8084677
:1011B000411B04D022462846FFF77CFCF0BBE068C8
:1011C000010203D5E562C4E9015854E0691CE162FB
:1011D0006160E16940F48030491EC4E90210304684
:1011E0002E70BDE8F087010202D500F480320AE0DB
:1011F0006068411C61600670E0680A2E40F480302F
:10120000E06006D00022E16A6068814203D90B46A3
:1012100002E00122F7E70346A7895B1B7F0503D4A1
:10122000E7699F4200DDE2B1814200D80146E562F4
:101230000F1AC4E90158002B09DD00E005E0224641
:1012400019462846FFF736FC08B14846C9E747B1BA
:10125000A069E5626560C01BA061E06840F0100015
:10126000E060E068000208D56168A069E562491B9A
:1012700008446560A0615046B3E73046B1E770B5F9
:10128000C468A50713D0650211D4B2F5807F09D0D8
:10129000B2F5007F06D0B2F5806F08D1012300F1CE
:1012A000240106E05D1E6FF07F46B54201D30120A8
:1012B00070BD0161C361416024F470611143C1607C
:1012C000002070BD70B5054640F202260A4C0FE0C2
:1012D00094F85000C00708D0AC4206D0E06836EA67
:1012E000000002D1204600F01DF8206D20F001041E
:1012F000002CEDD170BD0000C84900200446AFF3BA
:1013000000802046FEF778FF10B500F043F8BDE8F6
:10131000104000F039B810B500F056F8BDE81040A4
:1013200000F032B870B50446C068810713D080065B
:1013300001D5A56A04E0A169606808442169451ADD
:101340002046FFF7E1FB0022064629462046FFF72C
:101350002BFB304670BD002070BD70B510B1BDE8EC
:101360007040DFE70025074C6E1E07E02046FFF7C0
:10137000D9FF00B13546206D20F00104002CF5D1D5
:10138000284670BDC8490020002801D009F064BB80
:101390007047000010B5014602A000F03DF80120A2
:1013A00010BD000053494752545245443A205265FB
:1013B0006469726563743A2063616E2774206F708C
:1013C000656E3A200000000010B5012805D000210C
:1013D00003A000F021F8012010BD09A1F8E70000EA
:1013E00053494752544D454D3A204F7574206F660E
:1013F0002068656170206D656D6F72790000000076
:101400003A2048656170206D656D6F727920636F59
:10141000727275707465640070B505460C460A20DA
:1014200000E06D1C09F08EFB35B128780028F8D15A
:1014300002E0641C09F086FB14B120780028F8D182
:10144000BDE870400A2009F07DBB70477047002955
:10145000816802D041F0010101E021F001018160C9
:101460007047000010B50020214908600120087174
:1014700048714FF4602088600020C8600320087421
:101480001C4800F059F8072301220F21194800F0E9
:1014900077F8072302220821164800F071F8072385
:1014A00003220921134800F06BF80121114800F0D4
:1014B0002DF801210F4800F01FF801210D48FFF71A
:1014C000C6FF0C4800F096F800BF0A4800F02DF85F
:1014D0000028FAD1074800F09CF800BF054800F04A
:1014E0001DF80028FAD10121024800F088F810BD4B
:1014F0006C0C0020002401400029816802D041F4D6
:10150000807101E021F48071816070474268491E5A
:1015100022F4604242EA41314160704701460020B6
:101520008968490700D50120704701460020896875
:10153000090700D50120704710B542680E4B0C79A1
:101540001A400B6842EA04221343436082680B4B43
:101550001A40D1E9024323434C7942EA440213433F
:101560008360C26A097C22F47002491EC9B242EA51
:101570000151C16210BD0000FFFEF0FFFDF7F1FF59
:1015800070B5072509290AD9C468A1F10A0606EB36
:101590004606B540AC43B3401C43C46007E0046951
:1015A00001EB4106B540AC43B3401C4304611F232B
:1015B000072A09D2446B521E02EB820293409C43DD
:1015C00091400C43446370BD0D2A09D2046BD21FB5
:1015D00002EB820293409C4391400C43046370BD34
:1015E000C46A0D3A02EB820293409C4391400C4343
:1015F000C46270BD816841F00801816070470029B4
:10160000816802D041F4A00101E021F4A0018160D1
:101610007047816841F004018160704710B5184837
:10162000007858B30121174804F06FF930BB6521E9
:101630001548006808F026FF00241CE0002240F254
:101640002551124808F08FFC66220F4801680020DF
:1016500001F018FC0C48006807F0CEFD01F032FCE8
:10166000012240F22551094808F07DFC0020044980
:101670000870601CC4B2032CE0DB00BF10BD00008A
:10168000D000002000080140CC00002000440040B1
:1016900011480068114909680844401C00EB4000EB
:1016A0000F4901EB80008068A8B10C48006804284D
:1016B00005DA0A480068401C0849086008E0064846
:1016C0000068182804DA04480068401C02490860D1
:1016D0000120044908707047D00100202801002033
:1016E000D80A0020370100200C480068002808DDD7
:1016F0000A480068401E094908600120084908702E
:101700000BE008480068002807DD06480068401E16
:101710000449086001200249087070472801002030
:1017200037010020D001002000B502460B461846C4
:1017300000F010F802EB820100EB410000BD014611
:10174000092903DD01F13700C0B2704701F1300013
:10175000C0B2FAE70146302901DB392901DD00205A
:1017600001E001F00F0070470149405A7047000046
:10177000006C0040014A815270470000006C00403C
:101780002DE9F84300244EA14E48FEF7CCFE4E4909
:1017900008600846006800287ED04FF480614B48FE
:1017A00004F0C1F801204A4908704AA1464800687F
:1017B000FEF73BFD642006F0FDFC642190FBF1F296
:1017C00001FB1205084606F0F5FC642190FBF1F0E0
:1017D00090FBF1F201FB1206084606F0EBFC42F228
:1017E000107190FBF1F733463A4641A13648009517
:1017F0000068FEF71AFD474800683C2190FBF1F2B3
:1018000001FB12054348006890FBF1F62B46324677
:1018100041A12D480068FEF708FD692006F0CAFCCA
:101820000546682006F0C6FC642190FBF1F66820AE
:1018300006F0C0FC642190FBF1F201FB1207334675
:101840003A463AA1204800950068FEF7EEFC00BF3A
:10185000204603F0FDFD8046204604F0EFFC50B129
:10186000404604F0BDF805462B46424636A11648D0
:101870000068FEF7DAFC04F065F900F055FD611C24
:101880000C46084604F0F4FC0028E1D030A10E48D4
:101890000068FEF7CAFC00E010E04FF4FA502E4951
:1018A000086001E004F04EF92B4800680028F9D1E7
:1018B0000749087004480068FEF75CFEBDE8F8833D
:1018C000770000007040030874020020000C014003
:1018D000D00000202A2A204D69737454696D652058
:1018E0006261636B75702066696C652E0A0000008A
:1018F0002A2A2050726F6772616D20566572736973
:101900006F6E3A2025692E253032692E25303269D6
:101910000A000000300000202A2A2054696D653A30
:1019200020253032693A253032690A002A2A2044BB
:101930006174653A20253032692D253032692D25B4
:101940003034690A0000000025693D25690A00005D
:101950002A2A20456E640A0018000020F0B50646C9
:101960000C461746BC420BD1C4EBC400104951F8D9
:101970002000B04201D12046F0BD4FF0FF30FBE720
:10198000E01900EBD0714D10C5EBC500084951F8C6
:101990002000B04205DA3A46691C3046FFF7DEFF08
:1019A000EAE72A4621463046FFF7D8FFE4E7000081
:1019B0003CDC010810B500240FE004F29310002174
:1019C00008F094FC04F2C510002108F08FFC04F22A
:1019D000F710002108F08AFC641C322CEDD30021A2
:1019E0004FF4C97008F082FC0021662008F07EFCEC
:1019F00010BD00BFFEE701460120704770477047E9
:101A00000120704710B50121224803F07EFF002815
:101A10003FD10AF0E7F900283BD11F49A1F80401A2
:101A20001E480AF0F3F810B906F032FF31E007F073
:101A300017FE00220421084607F02EFE012206218F
:101A4000042007F029FEFFF79BFE00201249A1F8B1
:101A5000040113A00AF0DAF890B901210A2008F075
:101A600045FC01210B2008F041FC01210C2008F06D
:101A70003DFC02220721042007F00EFE00BFFEE716
:101A800000210A2008F032FC04F0B6FC01200649CF
:101A9000087010BD000801409848002070400308FD
:101AA0004D545F562A000000370100202DE9FC5FED
:101AB0004FF0000B3B480068C0EBC0003A4951F8BA
:101AC0002090484603F0EAFC0090484603F088FF67
:101AD0000546009803F0B2FC0746009803F0A4FC0A
:101AE0008046009803F096FC0190009804F0B4FB47
:101AF0008246BAF5204F3DD1642095FBF0F695FB68
:101B0000F0F100FB115465B30D2E26D2DFE806F08C
:101B1000250714081B091C0A0B1D0C1E0D0000BF15
:101B200000BF00BF00BF00BF00BF012C01DB1F2CA6
:101B300001DD4FF0010B13E0012C01DB1D2C01DD59
:101B40004FF0010B0CE000BF00BF00BF012C01DB18
:101B50001E2C01DD4FF0010B02E04FF0010B00BF26
:101B600000BFBBF1010F0ED101224846019908F0D8
:101B7000D1FB08E0BD4201DB454504DD01224846BA
:101B8000019908F0C7FB07480068401C0549086038
:101B90000846006804F06CFB10B1002001490860A1
:101BA000BDE8FC9F200000203CDC010810B50121AD
:101BB000294803F0AAFE90BB682006F0FBFA044611
:101BC00040F2E63225480168204608F0D7FB00BF06
:101BD00006F03EFE03F0B6FF214800680F2190FB9F
:101BE000F1F201FB120080B94FF480611D4803F04F
:101BF00093FE28B14FF480611A4803F094FE04E08C
:101C00004FF48061174803F090FE154800680028E3
:101C1000DED142F2D871642008F068FB1AE0FFE7D9
:101C200000BFFFF743FF03F08DFF4FF480610D48C5
:101C300003F072FE28B14FF480610A4803F073FE8E
:101C400004E04FF48061074803F06FFE0448006829
:101C50000028E6D110BD000000080140300000203F
:101C600020000020000C01407047000010B5034820
:101C70000078012801D106F0A9FD10BD3601002031
:101C80002DE9F041064640F2831006F093FA4FEA40
:101C90008008002422E0301906F08CFA074631193A
:101CA000481C06F087FA0546AF420ADA0D4800687C
:101CB000B84206DB0B480068A84202DA3019BDE8DA
:101CC000F081AF4209DD07480068A84203DB054800
:101CD0000068B84201DB3019F1E7241D4445DADB26
:101CE0000020ECE73000002010B50B2006F062FA6F
:101CF000012817D107F0B4FC03220421084607F09D
:101D0000CBFC04220621104607F0C6FC002018492F
:101D1000086000BF06F09CFD03F014FF1448006843
:101D20000028F7D100210B2008F0E0FA0C2006F083
:101D300041FA012812D100200AF054F870B90020AD
:101D40000C49A1F804010C4809F060FF30B90522E4
:101D50000621042007F0A0FC06F09AFD00210C20CB
:101D600008F0C4FA04F048FB01200449087010BDD3
:101D70002000002098480020704003083701002010
:101D80002DE9F05F6B2006F015FA8246002499E0F9
:101D900004EBC40000EB400505F16C0006F00AFA04
:101DA000012806D0022813D0032825D004280ED1FC
:101DB00052E0494850F8240048B9601C05F00CFF77
:101DC00005F1700006F0F6F9434941F8240077E088
:101DD00005F16E00FFF754FF074667B13E4850F823
:101DE000240040B9601C05F0F7FEB81C06F0E2F9CB
:101DF000394941F8240063E005F16D0006F0DAF995
:101E0000064636480068B04225DB334850F82400C7
:101E100008BB05F1710006F0CDF9804605F17000B0
:101E200006F0C8F9814606EB0A002C490968884289
:101E300001DCC34609E029480068801BA8EB0901C2
:101E4000484390FBFAF000EB090B601C05F0C4FE60
:101E5000214840F824B033E005F16E00FFF710FF91
:101E6000074667B305F16D0006F0A4F906461B4866
:101E70000068B04223DB184850F82400F8B9F81C79
:101E800006F098F98046B81C06F094F9814606EBF6
:101E90000A0012490968884201DCC34609E00F487C
:101EA0000068801BA8EB0901484390FBFAF000EBA7
:101EB000090B601C05F090FE074840F824B000BFF5
:101EC00000BF641C4FF4BD7006F074F9A0423FF7E8
:101ED0005FAFBDE8F09F0000B00A00203400002092
:101EE00010B54FF4BF7006F065F9234909688842C0
:101EF0000BDD214801684FF4BF7008F0F7F91F4867
:101F0000016840F27F1008F0F1F94FF4C07006F05C
:101F100051F91949096888420BDA174801684FF4EA
:101F2000C07008F0E3F91548016840F2811008F02C
:101F3000DDF94FF4C27006F03DF90446DCB10F48FC
:101F40000068844217D10C4801684FF4BF7008F054
:101F5000CDF90A48016840F27F1008F0C7F9064839
:101F600001684FF4C07008F0C1F90448016840F2FC
:101F7000811008F0BBF910BD3400002030000020B3
:101F800010B56148046861480068844204D05F4825
:101F9000046001205E4908605B4844685D48006851
:101FA000844204D05B4804600120594908605648C7
:101FB000846859480068844204D05748046001206E
:101FC00053490860012003F02FFD04465348006880
:101FD000844204D05148046001204D490860022029
:101FE00003F022FD04464E480068844204D04C4869
:101FF0000460022046490860032003F015FD0446F2
:1020000048480068844204D04648046001204049A2
:102010000860042003F008FD044643480068844239
:1020200004D0414804600120394908603F480068F5
:102030000B2836D2DFE800F0060A0E12161A1E220E
:10204000262B300000203A4908602EE00220384953
:1020500008602AE004203649086026E00820344958
:10206000086022E01020324908601EE0202030493C
:1020700008601AE040202E49086016E080202C49B4
:10208000086012E04FF48070294908600DE04FF4B9
:1020900000702749086008E04FF480602449086018
:1020A00003E000202249086000BF00BF214800680B
:1020B000012805D11E48006880F001001C49086015
:1020C0001D480068012806D11948006840F40060E6
:1020D0001749086005E01648006820F400601449BC
:1020E000086016480068012806D11148006840F4CD
:1020F00080500F49086005E00D48006820F48050CA
:102100000B49086010BD0000780A0020580000202C
:10211000B00100205C00002078000020600000205A
:1021200064000020680000206C0000207000002087
:1021300048000020740000207C0000208000002067
:1021400010B53248006820B1012823D0022856D1AA
:102150003EE02F4800682F490968884216D02E4873
:10216000006860B901202C49086040F27D1006F03B
:1021700021F82A49086001202449086009E000206C
:102180002649086001202149086002E00020224918
:10219000086038E021480068C8B921481C4909682E
:1021A00050F821001F49086001201F4908601D499F
:1021B0000968491E01EBC10101EB410101F18600F3
:1021C00005F0F8FF154908600220104908601AE080
:1021D0001248006890B90020124908600120124995
:1021E00008600B480068401C142190FBF1F201FBD1
:1021F00012000749086000200449086003E000203D
:102200000249086000BF00BF10BD0000C8000020E8
:10221000C0000020C40000208800002084000020AE
:10222000AC0C002038000020B001002070B5002563
:10223000002414E004EB4400114901EB80008068A5
:1022400001280BD104EB44010D4A52F8211001F290
:10225000851005F0AFFF012800D10125641C192C61
:10226000E8DB35B90748006840F00100054908601F
:1022700005E00448006820F001000249086070BDD4
:10228000D80A00204800002010B50221234803F09E
:102290003CFB30B12248006840F001002049086052
:1022A00005E01F48006820F001001D490860042176
:1022B0001A4803F02AFB30B11948006840F00200C8
:1022C0001749086005E01648006820F0020014492C
:1022D00008608021114803F018FB30B110480068F5
:1022E00040F004000E49086005E00D48006820F049
:1022F00004000B49086010210A4803F006FB30B1C6
:102300000748006840F008000549086005E00448F7
:10231000006820F008000249086010BD0008014074
:1023200054000020001001402DE9F05F684800785B
:10233000002867D00020664908706648006820B110
:1023400064480068401E634908606348006820B123
:1023500061480068401E604908606048006820B11C
:102360005E480068401E5D4908605D48006820B115
:102370005B480068401E5A4908605A48006820B10E
:1023800058480068401E574908605748006820B107
:1023900055480068401E54490860544800680028A9
:1023A00005DD52480068401E5049086005E00A20DB
:1023B0004E49086001204E4908604E48D0F800B0F0
:1023C00005F02AFE3C21B0FBF1F9B9F5B46F01DB51
:1023D00040F29F59CB4512D04648C0F800900027E4
:1023E0000BE0454850F8270030B1434850F827002B
:1023F000401E414941F827007F1C0A2FF1DB0120D4
:102400003E4908703E48007800285ED0692005F0FB
:10241000D1FE0546E91705EB91718910A5EB810105
:1024200041B9642195FBF1F201FB125111B14FF05A
:102430001D0A01E04FF01C0A682005F0BBFE0646AD
:10244000642196FBF1F496FBF1F201FB126000F1BE
:1024500001080D2C1BD2DFE804F01A0714081A0932
:102460001A0A0B1A0C1A0D0000BF00BF00BF00BFF4
:1024700000BF00BFB8F11F0F02DD641C4FF0010860
:102480000CE0D04502DD641C4FF0010806E0B8F115
:102490001E0F02DD641C4FF0010800BF00BF0C2CB2
:1024A00004DD0124691C692007F020FF04EBC4004F
:1024B00000EB041008EB80063146682007F016FF99
:1024C0000F480078401E0E490870BDE8F09F0000DC
:1024D00000000020F0010020A4010020AC0000203A
:1024E000A0000020F000002084000020B4000020A4
:1024F000B001002030000020B00A0020A800002019
:102500000100002010B53448046804F0010008B14F
:1025100005F0EEFF04F0020010B106F021F801E032
:1025200006F016F804F0040010B106F02BF801E0F4
:1025300006F01EF804F0080010B106F037F801E0CC
:1025400006F02AF804F0100010B106F043F801E09C
:1025500006F036F804F0200010B106F04FF801E064
:1025600006F042F804F0400010B106F05BF801E01C
:1025700006F04EF804F0800010B106F067F801E0B4
:1025800006F05AF804F4807010B106F073F801E018
:1025900006F066F804F4007010B106F07FF801E070
:1025A00006F072F804F4806010B105F099FF01E0C4
:1025B00005F08EFF04F4006010B105F0BFFF01E0EC
:1025C00005F0B2FF04F4805010B105F0A5FF01E062
:1025D00005F09AFF10BD0000480000204A4800683E
:1025E0000B287ED2DFE800F0060F1A25303B46515B
:1025F0005C6772004548006820F4FF7020F4C060FA
:10260000424908606DE04148006820F4FF7020F402
:10261000C06040F002003D49086062E03B4800684D
:1026200020F4FF7020F4C06040F0040037490860D7
:1026300057E03648006820F4FF7020F4C06040F096
:102640000800324908604CE03048006820F4FF7010
:1026500020F4C06040F010002C49086041E02B4895
:10266000006820F4FF7020F4C06040F0200027498B
:10267000086036E02548006820F4FF7020F4C06050
:1026800040F04000214908602BE02048006820F419
:10269000FF7020F4C06040F080001C49086020E01A
:1026A0001A48006820F4FF7020F4C06040F4807085
:1026B0001649086015E01548006820F4FF7020F402
:1026C000C06040F40070114908600AE00F480068DB
:1026D00020F4FF7020F4C06040F480600B49086073
:1026E00000BF00BF0A48006830B10848006840F4E5
:1026F00000600649086005E00448006820F40060B6
:10270000024908607047000038000020480000209F
:10271000880000200146A1F13000C1B2092901DD85
:10272000C81FC1B201F00F00704700000021002057
:1027300009E0084A525C00EB800302EB4302A2F17D
:1027400030004A1CD1B2034A525C0AB10829F0DBBE
:1027500070470000390100202DE9F05F4FF00009BB
:1027600000240027A04600250026F748007800280E
:1027700077D008F0E9F9F54901EB0010D0F800A096
:10278000504602F08BFEF249086008F0DDF9EF498F
:1027900001EB0010D0F800B0584602F07FFE8246F0
:1027A00003F05AFDB0F5A04F70D014DCB0F5605FB7
:1027B0006DD009DCB0F5005F1FD0B0F5205F38D0D8
:1027C000B0F5405F34D168E0B0F5804F73D0B0F51C
:1027D000904FF7D101E1B0F5304F6DD006DCB0F588
:1027E000084F6AD0B0F5204FECD130E2B0F5484F39
:1027F0007ED0B0F5943FE5D17EE114E0D248005D93
:102800002C2803D0D048005D2D2802D14FF00109BB
:1028100007E0CD48005D05EB850100EB4100A0F12C
:102820003005601CC4B2C848005D08B1082CE5DB67
:1028300085E221E0C448005D2D2802D14FF0010956
:1028400018E0C148005D2C2801D1012712E04FB1EA
:10285000BD48005D06EB860100EB4100A0F13006AB
:1028600008E090E2B848005D05EB850100EB41000F
:10287000A0F13005601CC4B2B348005D08B1082C5B
:10288000D8DB092E04DD4FF0010905E0E4E03CE06F
:1028900005EB850006EB400551E223E0AA48005D08
:1028A0002D2802D14FF001091AE0A748005D2C281D
:1028B00004D1012714E05CE08CE14BE147B1A24870
:1028C000005D06EB860100EB4100A0F1300607E059
:1028D0009D48005D05EB850100EB4100A0F130054E
:1028E000601CC4B29848005D08B1082CD6DB00E03B
:1028F000FCE1632E02DD4FF0010905E005EBC500A8
:1029000000EB051006EB800519E220E08E48005D23
:102910002D2802D14FF0010917E08B48005D2C28CB
:1029200001D1012711E047B18748005D06EB860120
:1029300000EB4100A0F1300607E08348005D05EBA5
:10294000850100EB4100A0F13005601CC4B27E4857
:10295000005D08B1082CD9DBB6F57A7F02DB4FF0B9
:10296000010905E005EB4500C0EBC51006EBC0050D
:10297000E5E120E07448005D2D2802D14FF0010907
:1029800017E07148005D2C2801D1012711E047B103
:102990006D48005D06EB860100EB4100A0F13006BA
:1029A00007E06948005D05EB850100EB4100A0F1FF
:1029B0003005601CC4B26448005D08B1082CD9DB46
:1029C00042F20F70864202DD4FF0010904E040F24E
:1029D0007120684306EB0015B1E15B48007870B3E5
:1029E000594800782D282BD057480078A0F13005A1
:1029F0005548407800B35448407805EB850100EB1A
:102A00004100A0F130055048807890B14E48807860
:102A1000A0F130064C48C07840B14B48C07806EB76
:102A2000860100EB4100A0F130060BE04FF00109F8
:102A300008E04FF0010905E04FF0010902E0FFE76F
:102A40004FF001093B2E02DD4FF0010903E0C5EB19
:102A5000051006EB800572E13B4800782D2802D175
:102A60004FF00108012419E03748005D2C2801D1FE
:102A7000012711E047B13448005D06EB860100EB09
:102A80004100A0F1300607E02F48005D05EB85010D
:102A900000EB4100A0F13005601CC4B22A48005D83
:102AA00008B1082CE0DB092E02DD4FF0010922E01D
:102AB000B8F1010F06D105EB850006EB4000C0F52B
:102AC0002F7505E005EB850006EB400000F52F753E
:102AD00040F27B1005F06EFB68B1A5F57F7000EB4E
:102AE000C00101EB00102D2101EB40005A2190FBA9
:102AF000F1F000F52F7522E1134800782D2802D15E
:102B00004FF00108012410E00F48005D2C2802D18D
:102B10004FF0010909E00C48005D05EB850100EB71
:102B20004100A0F13005601CC4B20748005D08B147
:102B3000082CE9DBB8F1010F02D1C5F52F7501E0D2
:102B400005F52F75FBE0000039010020302A002038
:102B5000C8010020994800782D2802D14FF00109C2
:102B60001FE019E09548005D2C2801D1012711E0F4
:102B700047B19248005D06EB860100EB4100A0F1F1
:102B8000300607E08D48005D05EB850100EB410054
:102B9000A0F13005601CC4B28848005D08B1082C63
:102BA000E0DB092E02DD4FF0010912E005EB8500A4
:102BB00006EB400540F27B1005F0FCFA48B105EB4E
:102BC000C50000EB05102D2101EB40005A2190FBC0
:102BD000F1F5B4E0794800782D2802D14FF00108D2
:102BE000012419E07548005D2C2801D1012711E06E
:102BF00047B17248005D06EB860100EB4100A0F191
:102C0000300607E06D48005D05EB850100EB4100F3
:102C1000A0F13005601CC4B26848005D08B1082C02
:102C2000E0DB092E02DD4FF001090FE0B8F1010FE2
:102C300006D105EB850006EB4000C0F52F7505E0D9
:102C400005EB850006EB400000F52F7577E05B484B
:102C500000782D2802D14FF0010946E0574841780D
:102C60000078303800EB800001EB4000A0F1300527
:102C70005248C1788078303800EB800001EB40008A
:102C8000A0F130060D2E26D2DFE806F02507140845
:102C90001B091C0A0B1D0C1E0D0000BF00BF00BF4E
:102CA00000BF00BF00BF012D01DB1F2D01DD4FF074
:102CB000010913E0012D01DB1C2D01DD4FF001099D
:102CC0000CE000BF00BF00BF012D01DB1E2D01DDA8
:102CD0004FF0010902E04FF0010900BF00BF06EB11
:102CE000C60000EB061005EB800528E033480078AD
:102CF0002D2802D14FF0010920E03048007830380B
:102D0000642148432D494978303901EB810100EBBA
:102D100041002A4989780844A0F130052748017903
:102D2000C078303800EB800001EB4000A0F13006A5
:102D300005EB4500C0EBC51006EBC00500BF00BFAA
:102D4000B9F1000F36D107F0FFFE1D4901EB00106D
:102D5000D0F800B0584602F0A1FB824602F06EFBAC
:102D6000A8420EDC07F0F0FE154901EB0010D0F888
:102D700000B0584602F092FB824602F055FBA84292
:102D800002DA4FF0010915E007F0DEFE0C4901EB15
:102D9000001001222946D0F800A0504607F0BAFAE8
:102DA00007F0D2FE064901EB0010006810B9284672
:102DB00006F0C8FB4846BDE8F09F0000390100203E
:102DC000302A002030B50024002351E0184603F0DB
:102DD00007FA01284AD128480068CD2148432749ED
:102DE00001EB8000143000EB03100568244800EB71
:102DF0000410056020480068CD2148431F4901EBBD
:102E00008000143000EB031040681D4901EB0411F1
:102E1000486019480068CD214843184901EB8000FB
:102E2000143000EB03108068154901EB0411886031
:102E300011480068CD214843104901EB800014304F
:102E400000EB0310C0680E4901EB0411C8600C4888
:102E500000EB04100068401C30B932230121601ED1
:102E6000074A02EB00108160601CC4B2581CC3B258
:102E7000322BABDB30BD000080010020004D02088A
:102E8000302A002070B506460C46154600200C4935
:102E90000860012006F058F9304606F0ADF92C2004
:102EA00006F052F9204606F0A7F92C2006F04CF95E
:102EB000284606F0A1F9022006F046F970BD000090
:102EC000F800002010B5032006F03EF90548006820
:102ED00006F01EFA042006F037F9002002490870B7
:102EE00010BD0000F800002004010020704770476A
:102EF000704770477047704770477047704770471A
:102F000070470029016802D041F0010101E021F081
:102F1000010101607047000010B5114800F028F869
:102F2000104811490860114848600020886003205B
:102F3000C8600020086180204861400088618000EE
:102F4000C8612020086200024862002088620448AC
:102F500000F07AF801210248FFF7D3FF10BD00000E
:102F6000080002404C240140800C0020040C00208A
:102F7000016821F001010160002101604160816070
:102F8000C1602D4B2C49C21A8039984243D018DCBD
:102F90002A4BA0EB0302984235D00ADC284A80185D
:102FA00029D014282BD0282824D1486840F47060F8
:102FB00034E0142A2BD0282A1CD1486840F4700031
:102FC0002CE02048B2F56C7F2ED009DCB2F5627F90
:102FD00026D0B2F5677F0DD1016841F0F00108E01D
:102FE000B2F5717F24D0B2F5767F03D1016841F448
:102FF000702101607047486840F00F000EE048689B
:1030000040F0F0000AE0486840F4704006E048688C
:1030100040F4702002E0486840F0706048607047FB
:10302000016841F00F01E4E7016841F47061E0E7F5
:10303000016841F47041DCE7800002404400024036
:10304000F8FFFDBF0404024030B5036847F6F07294
:1030500093430C6A8A682243D1E904452C432243F6
:103060008C692243CC6922434C6A22438C6A2243F6
:103070001A430260CA6842600A6882604968C16097
:1030800030BD7047002000E0401C41F2883188428A
:10309000FADB7047002000E0401CB0F57A7FFBDBD4
:1030A00070470000F8B500244748007850B103F09D
:1030B00057FD0021084602F025FD0122A421002031
:1030C00003F0F0FC00204149086065E040480068DA
:1030D0003E490968084400EB40003E4901EB80008E
:1030E000806808B9012457E038480168891C052028
:1030F00002F008FD3448007868B30120334D009099
:103100002D68354E3668B54201D1012500E0002515
:103110002B462F4D2D682D4E3668354405EB450561
:103120002C4E06EB8505AA68294D2D68274E36687A
:10313000354405EB4505274E06EB85056968244DAA
:103140002D68224E3668354405EB4505214E56F86C
:10315000250007F08BF81D4A12681F4B1B689A4226
:1031600001D1012200E000221146194A1268174BD2
:103170001B681A4402EB4202164B03EB8202906872
:1031800003F08AF911480068401C1049086008469D
:103190000068052800DB0124002C97D00A4800783D
:1031A00068B10A48006850B9012C08D104210F20E9
:1031B00002F0A8FC0022A521104607F0A7F9002084
:1031C00001490870F8BD000037010020D40100203B
:1031D000D0010020D80A00202801002038B53E4840
:1031E0000078002877D000203B49087001222B216D
:1031F00003F04CFD0221002002F084FC0020374B3C
:1032000000901B68364C2468234403EB4303354C81
:1032100004EB83039A68314B1B68314C24682344C8
:1032200003EB43032F4C04EB830359682B4B1B68C0
:103230002B4C2468234403EB43032A4C54F823000B
:10324000002307F013F80421084602F05BFC00227B
:10325000C021104607F05AF90521042002F052FC63
:103260000022BF21104607F051F90621022002F08A
:1032700049FC00228D21012004F0A6FB062112202A
:1032800002F040FC00228E21012004F09DFB06216B
:10329000222002F037FC00228F21012004F094FB51
:1032A0000621482002F02EFC00228A21012004F091
:1032B0008BFB0621582002F025FC00228B210120E7
:1032C00004F082FB0621682002F01CFC00228C2105
:1032D000012004F079FB38BD37010020D001002027
:1032E00028010020D80A00202DE9F041FD4805689A
:1032F0004FF4C17004F05EFFFB49086040F2831098
:1033000004F058FF0446022C03DB0120F749086053
:1033100002E00020F5490860032C03DB0120F4499A
:10332000086002E00020F2490860042C03DB012061
:10333000F049086002E00020EE490860052C03DB3C
:103340000120ED49086002E00020EB490860062CEE
:1033500003DB0120E949086002E00020E74908603A
:103360004FF4BD7004F026FF0446022C03DB01205D
:10337000E349086002E00020E1490860032C03DB18
:103380000120E049086002E00020DE490860042CCA
:1033900003DB0120DC49086002E00020DA49086014
:1033A000052C03DB0120D949086002E00020D74941
:1033B0000860062C03DB0120D549086002E00020EC
:1033C000D3490860072C03DB0120D249086002E0E2
:1033D0000020D0490860082C03DB0120CE4908609A
:1033E00002E00020CC490860092C03DB0120CB4916
:1033F000086002E00020C94908600A2C03DB0120B4
:10340000C749086002E00020C5490860B548006867
:103410001D2872D2DFE810F01D0038024202710050
:10342000B60221034F03C603F1031C0471007100AF
:1034300071007100710071007100EC011E02EC005E
:1034400071007100710071006F0281008B00240314
:103450007A034FF41670B34908600020B24908702F
:10346000B249087003F010F9472847D006DC1B2842
:1034700038D01E2848D02E284DD11AE04D2807D02C
:10348000872825D08D2846D101209649086042E042
:10349000672004F08FFE0446601C0446022800DD0D
:1034A00000242146672006F021FF0120A049086082
:1034B00031E040F27B1004F07DFEC0F101063146A0
:1034C00040F27B1006F012FF01209949086022E0CB
:1034D000002098490860132082490860012094491F
:1034E000086018E0002094490860944908609449F5
:1034F000086011207B4908600DE042E200209149FC
:1035000008604FF47A7506E013208D490860192091
:103510007449086000BF00BFC5E301230022AB214E
:10352000AA2000F0F5FB1A206E490860BBE304F006
:103530008DFE0746172F08D0472F02D0872F50D176
:1035400000BF00206749086050E0FFF7EFF806462B
:10355000012E42DB4FF4BD7004F02CFEB0423CDB88
:103560000B2E2FD2DFE806F02E060A0E12161A1EB8
:1035700022262A0005206F49086023E00C206D49AF
:1035800008601FE013206B4908601BE01A2069499E
:10359000086017E021206749086013E0282065498A
:1035A00008600FE02F20634908600BE03620614976
:1035B000086007E03D205F49086003E044205D4962
:1035C000086000BF00BF00205D4908600420454935
:1035D000086001205649086002E01920414908604E
:1035E00004E00021384602F075FC00BF00BF5AE33A
:1035F000002000F0CDFD04F029FE0746472F0AD039
:1036000004DC172F11D02D2F09D10AE0872F03D00A
:103610008D2FF9D104E000BF002032490860E5E0B9
:1036200000BF384606F00CFDE0E04748007843490B
:1036300009780844C6B20C2E12D2DFE806F0061252
:103640001F2C39458794A1AEBBC800203A490860B9
:103650003A49086013203A4908601120214908605E
:10366000C2E0032033490860132035490860042074
:103670001C49086001202E490860B5E005202D494D
:10368000086013202E4908600420164908600120B4
:1036900027490860A8E00C20264908601320284923
:1036A000086004200F4908600120214908609BE060
:1036B0001320204908602249086004200949086055
:1036C00001201B4908608FE01A201A490860132066
:1036D0001B49086004200349086001201449086060
:1036E00082E00000980100204401002048010020F1
:1036F0004C010020500100205401002058010020FE
:103700005C010020600100206401002068010020AD
:103710006C0100207001002074010020780100205D
:103720007C010020F001002036010020340100203F
:10373000B001002080010020D001002028010020DD
:10374000A001002088010020840100202120FE49E2
:1037500008601320FD4908600420FD49086001202D
:10376000FC49086040E02820F74908601320F74929
:1037700008600420F64908600120F649086033E03B
:103780002F20F14908601320F04908600420F04917
:1037900008600120EF49086026E03620EA49086009
:1037A0001320EA4908600420E94908600120E9493A
:1037B000086019E03D20E44908601320E3490860EF
:1037C0000420E34908600120E24908600CE044203D
:1037D000DD4908601320DD4908600420DC490860E9
:1037E0000120DC49086000BF00BF00BF00BF5AE2F3
:1037F000FFF758FC04F02AFD472810D004DC1728F6
:1038000016D02D2824D104E087280DD08D281FD173
:1038100002E0FDF73DFF1BE0FDF766FF18E0CB4837
:103820000068CB49086013E00020C94908600FE038
:10383000C9480068C9490968084400EB4000C84904
:1038400001EB8000806810B11220C149086000BF00
:1038500000BF28E2FFF7C2FC04F0F8FC172807D0ED
:1038600047280BD087280DD10020B949086009E00E
:1038700006F094FC1120B649086003E01120B44919
:10388000086000BF00BF0EE2012300221B211C20A4
:1038900000F03EFA0220AE49086004E204F0D6FCD3
:1038A0000746172F08D0472F02D0872F1CD100BF03
:1038B0000020A74908601CE0FEF738FF064640F6E6
:1038C0000A30864202D0A748864209D101209E498B
:1038D000086018209E4908600120A349087002E092
:1038E00000209B49086004E00121384602F0F2FA0A
:1038F00000BF00BFD7E1012000F04AFC04F0A6FCA5
:103900000746002099490870472F0AD004DC172F7A
:1039100013D02D2F34D10CE0872F03D08D2F2FD132
:1039200006E000BF0020914908708949086027E03F
:1039300000BF384606F084FB22E08D4800788749B6
:1039400009780844C6B216B1012E17D109E0022049
:103950007D49086018207D49086004207C49086082
:103960000CE04B2078490860182078490860042052
:103970007749086001207D49087000BF00BF00BF83
:1039800000BF90E17048006800F022FB04F05EFC8C
:1039900006464B2E4CD006DC172E18D02D2E09D003
:1039A000472E58D10AE04E2E2ED0872E0BD08D2ECA
:1039B00051D100BF304606F043FB4CE0634800683D
:1039C0006349086047E000206149086043E007F070
:1039D000BBF8684901EB0010D0F80080404601F0C8
:1039E0005DFD074602F02AFC68B1042062490860C8
:1039F00005205749086059480068604908605C48DC
:103A000000685F49086026E000BF4F480068CD218C
:103A100048435C4901EB800040684B490860084618
:103A2000006802F035FC0028EFD04FF47A7512E000
:103A300000BF45480068CD214843524951F8200055
:103A4000414908600846006802F022FC0028F0D0D6
:103A50004FF47A7500BF00BF25E102F09FF822E124
:103A600001F050F9172804D0472803D0872820D127
:103A70001BE000BF40480068354908603E480568C3
:103A80003E480068354908603D480068384908608C
:103A90002D480068CD2250433A4A02EB80000122B3
:103AA0008168002003F0F2F803E000202849086054
:103AB00000BF00BFF7E001F045F8172804D0472801
:103AC00003D0872820D11BE000BF2B480068204985
:103AD0000860294805682948006820490860284886
:103AE00000682349086018480068CD225043254AE1
:103AF00002EB800001228168002003F0C7F803E098
:103B000000201349086000BF00BFCCE000F042F97C
:103B1000172804D0472803D0872841D13CE000BFB4
:103B2000154800680A49086013480568134800688A
:103B30000A490860124800680D4908600248006898
:103B4000CD2250430F4A1FE080010020A001002039
:103B500098010020B0010020D001002028010020A1
:103B6000D80A0020C6D53C003601002034010020D0
:103B700084010020302A00209C010020F801002050
:103B8000FC010020004D020802EB80000122816848
:103B9000002003F07BF803E000205149086000BFDB
:103BA00000BF80E000F0DAFD172804D0472803D0DA
:103BB000872820D11BE000BF4A48006848490860B8
:103BC000484805684848006848490860484800680F
:103BD0004849086048480068CD225043474A02EBF4
:103BE000800001228168002003F050F803E00020EB
:103BF0003B49086000BF00BF55E000F0AFFB17284D
:103C000004D0472803D0872820D11BE000BF3548C7
:103C10000068334908603348056833480068334911
:103C20000860334800683349086033480068CD2293
:103C30005043324A02EB800001228168002003F0E9
:103C400025F803E000202649086000BF00BF2AE0F5
:103C500001F050F9172804D0472803D0872820D135
:103C60001BE000BF1F4800681D4908601D4805682B
:103C70001D4800681D4908601D4800681D4908600E
:103C80001D480068CD2250431C4A02EB80000122EF
:103C90008168002002F0FAFF03E00020104908606C
:103CA00000BF00BF00BF00BF1548006858B9002022
:103CB0000B490860134908600120134908704FF44C
:103CC00016700F49086006480068854205D000203C
:103CD0000E49086001200C490870BDE8F081000021
:103CE000980100209C010020F801002028010020FC
:103CF000FC0100208401002080010020004D02080A
:103D0000F00100208801002037010020A4010020DC
:103D1000F8B504460F4615461E4607F0D7F80122AF
:103D20002146002002F0B2FF0321042001F0EAFE48
:103D300000223946104606F0E9FB3EB90620002372
:103D40001A4629460090184603F0C2FD0421084691
:103D500001F0D8FE00220821022003F035FE0022E7
:103D60000921022003F030FE00220921022003F085
:103D70002BFE00220921022003F026FE00220B2147
:103D8000022003F021FE04F039FD0521082001F096
:103D9000B9FEF8BD70B57F480078C1004FF07F4094
:103DA000C8407D4908607B480078C1004FF08070B2
:103DB00008417A49086077480078C1004FF0005008
:103DC00008417749086073480078C1004FF0FE4011
:103DD00008417449086004F039FA04460020724929
:103DE00008706C480078042874DA70480068000E87
:103DF0006F4908706D480068000C6E4908706B4888
:103E00000088000A6C490870684800786B4908709F
:103E100060480078C0EB001008306949086008204D
:103E20006849087068480068B0F5FA7F07DA084604
:103E3000007863490968884201D1012000E0002030
:103E400002465B480178012003F0BEFD5D48007822
:103E5000001D5C4908705C480068B0F5FA7F07DA1D
:103E60000846007856490968884201D1012000E0DF
:103E7000002002464F480178012003F0A5FD51487B
:103E80000078001D4F4908704F480068B0F5FA7F70
:103E900007DA084600784A490968884201D10120BA
:103EA00000E00020024644480178012003F08CFD28
:103EB00044480078001D4349087043480068B0F545
:103EC000FA7F08DA084600783D490968884202D13D
:103ED000012001E00AE00020024638480178012074
:103EE00003F072FD36480078364908704B2C33D009
:103EF00004DC172C07D02D2C49D137E04E2C21D0D3
:103F00008D2C44D10DE0172406F01EFE2F4901EB45
:103F100000100122056825480168284606F0FAF9D4
:103F200035E0224800681C49096808401D490968B5
:103F3000884206DA1D4800681849096808441B4988
:103F4000086024E013480078002804DD1148007858
:103F5000401E104908701AE00E480078032804DA61
:103F60000C480078401C0B49087010E00F480068AE
:103F70000949096808400A490968884206DD0B4872
:103F8000006806490968401A0849086000BF00BF78
:103F9000204670BD35010020DC010020E00100203A
:103FA000E4010020E801002037010020C0010020CA
:103FB000D8010020D9010020DA010020DB01002017
:103FC000EC0100202D01002014000020302A0020E8
:103FD0002DE9F041074600266448076064480078F0
:103FE00090B1FEF7EFFE61480068CD225043614A70
:103FF00002EB800001228168002002F047FE0020D1
:104000005D4908605D4908600020594908705C48B6
:104010000068002877D000205949086001213A2023
:1040200001F070FD5448006850B10022872110460D
:1040300003F0CAFC00228821104603F0C5FC09E009
:1040400000222021104603F0BFFC00222021104650
:1040500003F0BAFC07213A2001F054FD00E0761C81
:10406000484800EB061080680028F8D042480068F5
:10407000001DB0420CD0052E0ADB0022852110461F
:1040800003F0A2FC00228621104603F09DFC09E00B
:1040900000228921104603F097FC00228921104656
:1040A00003F092FC02203849087033480578002458
:1040B00057E0344800EB05100068401C00284DD044
:1040C0000120324908702D480068844201D1012046
:1040D00000E0002002462021002003F075FC0420AF
:1040E0002A49087025480068844201D1012000E077
:1040F00000200146284602F0C1FC204800688442A6
:1041000002D1012001E02EE00020034601222946D1
:10411000002002F0F7FE72201C4908701748006862
:10412000844201D1012000E000200246202100202D
:1041300003F04AFC11480068844201D1012000E0EC
:10414000002002462946002002F0FAFB681CC5B296
:104150000D480078401C0C49087000E00524601CE4
:10416000C4B2052CA5DBBDE8F08100008001002071
:1041700037010020004D02088401002028010020A2
:10418000B0010020302A00202E0100202D01002047
:1041900070B5064600256848066068480078A0B1FA
:1041A000FEF710FE64480068CD225043644A02EBDB
:1041B000800001228168002002F068FD00205F4934
:1041C000087060490860604908606048006800281D
:1041D00079D000205D49086001213A2001F092FC6D
:1041E0005848006850B100228721104603F0ECFBCC
:1041F00000228821104603F0E7FB09E0002220217D
:10420000104603F0E1FB00222021104603F0DCFB06
:1042100007213A2001F076FC00E06D1C4C4800EBD1
:10422000051080680028F8D046480068001DA842A4
:104230000CD0052D0ADB00228521104603F0C4FBBB
:1042400000228621104603F0BFFB09E000228921ED
:10425000104603F0B9FB00228921104603F0B4FB9D
:1042600002203C490870002463E03648006820447E
:10427000374901EB00100068401C002856D001208F
:104280003549087030480068844201D1012000E0BF
:10429000002002462021002003F096FB2A480068F7
:1042A000844201D1012000E00020024620210020AC
:1042B00003F08AFB032028490870234800688442E1
:1042C00002D1012001E036E0002002461D480068CE
:1042D00020441F4B03EB00104168002006F016F944
:1042E0000BE019480068844201D1012000E0002061
:1042F00002462021002003F067FB17480078782849
:10430000EFDB7720144908700F480068844201D120
:10431000012000E0002002462021002003F054FB91
:104320000C480078401C0B49087000E00524601C14
:10433000C4B2052C99DB70BD80010020370100203C
:10434000004D02088401002028010020B001002057
:10435000302A00202E0100202D01002070B503F02E
:1043600075FF04460020F8490870F84800780528D1
:1043700014DAF7480068B0F5FA7F05DA00225F2109
:10438000012003F021FB04E000222021012003F0A2
:104390001BFBF04800780B38EE4908704B2C7DD0A1
:1043A0000EDC2B2C7BD006DC172C16D01D2C19D044
:1043B000272C16D153E12D2C72D02E2CF9D1F0E000
:1043C0008B2C72D004DC4D2C6CD04E2CF1D18BE0B8
:1043D0008D2C45D08E2CECD123E0FEF7BDF900B139
:1043E0000224ADE1D9480078052819DA3021D748F0
:1043F00002780078401CD54B1870D74881540022B1
:10440000012003F0E1FAD3480078001DD14908707B
:10441000CE480078032803D1084600780F30087092
:104420008EE1CA480078052819DA3121C748027898
:104430000078401CC54B1870C748815400220120E9
:1044400003F0C2FAC3480078001DC2490870BF4893
:104450000078032803D1084600780F3008706FE118
:10446000BA48007805281FDA3221B8480278007867
:10447000401CB64B1870B84881540022012003F04C
:10448000A3FAB4480078001DB2490870AF4800781C
:10449000032809D1084600780F3004E062E0BEE04E
:1044A0009EE002E03FE008704AE1A8480078052855
:1044B00019DA3321A54802780078401CA34B187004
:1044C000A54881540022012003F07EFAA14800781B
:1044D000001DA04908709D480078032803D10846B4
:1044E00000780F3008702BE198480078052819DA19
:1044F0003421964802780078401C944B18709648F6
:1045000081540022012003F05FFA92480078001DD8
:10451000904908708D480078032803D10846007838
:104520000F3008700CE189480078052819DA352128
:10453000864802780078401C844B18708648815465
:104540000022012003F040FA82480078001D8149D2
:1045500008707E480078032803D1084600780F30A1
:104560000870EDE079480078052819DA3621774897
:1045700002780078401C754B1870774881540022EF
:10458000012003F021FA73480078001D714908707A
:104590006E480078032803D1084600780F30087071
:1045A000CEE06A480078052819DA37216748027892
:1045B0000078401C654B1870674881540022012028
:1045C00003F002FA63480078001D624908705F48F2
:1045D0000078032803D1084600780F300870AFE058
:1045E0005A480078052819DA3821584802780078A6
:1045F000401C564B1870584881540022012003F08B
:10460000E3F954480078001D524908704F4800787B
:10461000032803D1084600780F30087090E04B481B
:10462000007805281ADA3922484801780078401CB9
:10463000464B18704848425400223921012003F0AB
:10464000C3F944480078001D424908703F4800788B
:10465000032803D1084600780F30087070E03B480B
:104660000578062D6AD2DFE805F069533D2711036E
:1046700036480078401E3549087000203649334AD4
:104680001278885453203349087057E02F48007837
:10469000401E2E49087000202F492C4A1278885459
:1046A00053202C49087000228921012003F08CF945
:1046B00044202849087041E024480078401E2349DE
:1046C000087000202449214A127888544420214946
:1046D000087000228921012003F076F926201D4967
:1046E00008702BE019480078401E18490870002116
:1046F0001948164A1278815426201649087000225B
:104700008921012003F060F917201249087015E093
:104710000E480078401E0D49087000200E490B4AD3
:104720001278885417200B49087000228921012033
:1047300003F04AF908200749087000BF00BF00BF16
:1047400000BF204670BD0000370100203501002069
:10475000140000202D0100203901002070B503F065
:1047600075FD04460020F2490870F24800780828D8
:1047700014DAF1480068B0F5FA7F05DA00225F210B
:10478000012003F021F904E000222021012003F0A0
:104790001BF9EA4800780B38E84908704B2C7DD0AB
:1047A0000EDC2B2C7BD006DC172C16D01D2C19D040
:1047B000272C16D155E12D2C72D02E2CF9D1F2E0F8
:1047C0008B2C72D004DC4D2C6CD04E2CF1D18CE0B3
:1047D0008D2C45D08E2CECD123E0FDF7BDFF00B130
:1047E0000224A1E1D3480078042819DA3021D14805
:1047F00002780078401CCF4B1870D14881540022B9
:10480000012003F0E1F8CD480078001DCB49087085
:10481000C8480078022803D1084600780F30087095
:1048200082E1C4480078042819DA3121C1480278AD
:104830000078401CBF4B1870C148815400220120F1
:1048400003F0C2F8BD480078001DBC490870B948A3
:104850000078022803D1084600780F30087063E121
:10486000B448007804281FDA3221B2480278007870
:10487000401CB04B1870B24881540022012003F054
:10488000A3F8AE480078001DAC490870A94800782C
:10489000022809D1084600780F3004E064E0C1E046
:1048A000A0E002E040E008703EE1A2480078042861
:1048B0001ADA33229F4801780078401C9D4B18700B
:1048C0009F48425400223321012003F07DF89B4889
:1048D0000078001D9949087096480078022803D195
:1048E000084600780F3008701EE1924800780428CE
:1048F00019DA34218F4802780078401C8D4B1870EB
:104900008F4881540022012003F05EF88B48007824
:10491000001D8A49087087480078022803D108469C
:1049200000780F300870FFE08248007804281ADA17
:104930003522804801780078401C7E4B18708048F2
:10494000425400223521012003F03EF87B480078D4
:10495000001D7A49087077480078022803D108467C
:1049600000780F300870DFE072480078042819DA08
:104970003621704802780078401C6E4B18707048E1
:1049800081540022012003F01FF86C480078001DBC
:104990006A49087067480078022803D10846007801
:1049A0000F300870C0E063480078042819DA372116
:1049B000604802780078401C5E4B18706048815453
:1049C0000022012003F000F85C480078001D5B49DC
:1049D000087058480078022803D1084600780F3044
:1049E0000870A1E05348007804281ADA38225148A8
:1049F00001780078401C4F4B1870514842540022F7
:104A00003821012002F0E0FF4C480078001D4B499E
:104A1000087048480078022803D1084600780F3013
:104A2000087081E043480078042819DA39214148A8
:104A300002780078401C3F4B187041488154002296
:104A4000012002F0C1FF3D480078001D3B4908707D
:104A500038480078022803D1084600780F300870E3
:104A600062E034480578012D46D0022D2ED0032D6A
:104A700016D0042D56D10078401E2E490870002013
:104A80002F492C4A1278885453202C490870002250
:104A90002021012002F098FF44202849087041E0BD
:104AA00024480078401E2349087000202449214AE8
:104AB000127888544420214908700022892101205D
:104AC00002F082FF35201D4908702BE0194800785C
:104AD000401E1849087000201949164A1278885457
:104AE00035201649087000228921012002F06CFF50
:104AF00017201249087015E00E480078401E0D4935
:104B0000087000210E480B4A1278815417200B4977
:104B1000087000228921012002F056FF0820074971
:104B2000087000BF00BF00BF00BF204670BD00007E
:104B30003701002035010020140000202D01002045
:104B4000390100202DE9F0416A48007880B1012048
:104B50006949087000206749087005F0F5FF67494A
:104B600001EB00100668304600F03AFF6449086027
:104B700003F06CFB044605F0E7FF604901EB001011
:104B80000768384600F08AFC064601F065FB0546DA
:104B90000521082000F0B6FF5748007800285CD0B7
:104BA000002055490870B5F5F04F35D00ADCDDB16D
:104BB000B5F5C04F10D0B5F5D04F1DD0B5F5E04FCD
:104BC0004AD121E0B5F5504F2ED0B5F5604F33D026
:104BD000B5F5983F40D137E000231A4648480168B0
:104BE000012001F06EFD37E000231A4644480168B9
:104BF000012002F05BF82FE000231A4640480168CC
:104C0000012002F04DF927E000231A463C480168D4
:104C1000012001F086FD1FE000231A463848016894
:104C2000012002F0DDF817E000231A46344801683D
:104C3000012002F065F90FE000231A4630480168B0
:104C4000012002F02EF907E000231A462C480168E3
:104C5000012001F065FD00BF00BF172C38D02D2CBE
:104C600004D0472C41D08D2C40D118E005F06CFFCA
:104C7000224901EB00100768384600F00FFC064699
:104C800000F0DCFB1E490968884204DA1C48006811
:104C9000401E1B49086001201749087026E005F0F6
:104CA00053FF164901EB00100768384600F0F6FB89
:104CB000064600F0B9FB12490968884204DD104835
:104CC0000068401C0E49086001200B4908700DE087
:104CD00005F03AFF094901EB001001220668084877
:104CE0000168304605F016FB00E000BF00BF20461B
:104CF000BDE8F08137010020C4010020302A0020E7
:104D0000C001002070B57648007880B10120754957
:104D1000087000207249087005F016FF724901EB17
:104D200000100568284600F05BFE7049086003F03B
:104D30008DFA04460521082000F0E4FE6948007859
:104D400010B1002067490870172C73D02D2C04D0A7
:104D5000472C70D08D2C55D155E06548006830B196
:104D600001280AD002281ED003284AD130E00120B1
:104D70005E4908605B49087043E05C4800680428AD
:104D800002D005280DD106E0052058490860012011
:104D90005449087005E001205449086051490870E1
:104DA00000BF00BF2DE051480068022808D003284A
:104DB0000CD102204D49086001204A49087005E0E5
:104DC00001204A4908604749087000BF00BF18E049
:104DD00005F0BAFE444901EB00100668304600F0C9
:104DE0005DFB054600F02AFB40490968884204DA69
:104DF0003E480068401E3D4908600120394908705E
:104E000000BF00BF68E03A48006830B101280AD00E
:104E1000022821D003284FD135E001203349086012
:104E20003049087048E031480068012804D005285E
:104E300010D108E042E04EE005202C490860012036
:104E40002849087006E00420284908600120254907
:104E5000087000BF00BF2FE024480068012802D07E
:104E600002280ED106E002202049086001201D49D9
:104E7000087006E003201D490860012019490870E8
:104E800000BF00BF18E005F05FFE174901EB0010FE
:104E90000668304600F002FB054600F0C5FA1349EB
:104EA0000968884204DD11480068401C0F49086009
:104EB00001200C49087000BF00BF0DE005F044FE62
:104EC000094901EB001001220568084801682846DD
:104ED00005F020FA00E000BF00BF204670BD0000D2
:104EE00037010020C4010020302A0020C00100202A
:104EF000B401002010B50020B1490870B148007815
:104F0000082814DAB0480068B0F5FA7F05DA002204
:104F10005F21012002F058FD04E000222021012041
:104F200002F052FDA94800780B38A849087003F038
:104F30008DF904462E2C6ED010DC1E2C6CD006DCB5
:104F4000172C1AD01B2C68D01D2C1AD11AE0272C34
:104F500076D02B2C75D02D2CF7D1ADE08B2C47D0F3
:104F600006DC4B2C6ED04D2C6ED04E2CEDD155E086
:104F70008D2C2BD08E2CE8D116E0FDF7EDFB00B187
:104F800002241AE18F48007808280CDA30218D4875
:104F900002780078401C8B4B18708D488154002299
:104FA000012002F011FD08E18648007808280CDA9B
:104FB0003121844802780078401C824B1870844864
:104FC00081540022012002F0FFFCF6E07D480078C9
:104FD00008280CDA32217B4802780078401C794B93
:104FE00018707B4881540022012002F0EDFCE4E0BF
:104FF0007448007808280DDA332272480178007866
:10500000401C704B1870724842540022332101201A
:1050100002F0DAFCD1E03CE08AE071E06948007817
:1050200008280CDA3421674802780078401C654B68
:105030001870674881540022012002F0C5FCBCE0D2
:1050400087E04BE013E0FFE75E48007808280DDAC0
:1050500035225C4801780078401C5A4B18705C4837
:10506000425400223521012002F0AEFCA5E0554853
:10507000007808280CDA3621524802780078401C63
:10508000504B1870524881540022012002F09CFCC1
:1050900093E04C48007808280DDA37224948017817
:1050A0000078401C474B1870494842540022372171
:1050B000012002F089FC80E04248007808280CDAE0
:1050C0003821404802780078401C3E4B1870404818
:1050D00081540022012002F077FC6EE0394800780C
:1050E00008280CDA3921374802780078401C354B03
:1050F0001870374881540022012002F065FC5CE002
:1051000030480078082812DA3248007878B92C2222
:105110002C4801780078401C2A4B18702C484254C7
:1051200001202C49087000222E2102F04DFC44E0A1
:105130002448007860B92D21224802780078401C6C
:10514000204B1870224881540022012002F03CFCC0
:1051500033E01C48007800282EDD1A480078401EF5
:10516000184908701A480978405C2C2802D10020A0
:105170001849087000201649124A127888541148BC
:105180000078072809DA00222021012002F01CFC07
:105190000E4800780B380D4908700C4800780B3821
:1051A0000A49087000222021012002F00DFC074866
:1051B00000780B380549087000BF00BF204610BDBD
:1051C0003701002035010020140000202D010020AF
:1051D00039010020380100207047704710B50220C7
:1051E00000F09CF8B8B102210B4800F08EFB60B9CA
:1051F0000A4800680A49884207DA0A48007820B954
:1052000006480068401C054908600A2005490870E6
:10521000022000F07DF810BD000801409802002037
:1052200040420F000200002010B5042000F076F884
:10523000B8B104210B4800F068FB60B90A48406827
:105240000A49884207DA0A48007820B906484068C7
:10525000401C054948600A2005490870042000F0F8
:1052600057F810BD000801409802002040420F008E
:10527000030000207047000010B5102000F04EF829
:10528000B8B110210B4800F040FB60B90A48C06873
:105290000A49884207DA0A48007820B90648C068F7
:1052A000401C0549C8600A2005490870102000F01C
:1052B0002FF810BD001401409802002040420F005A
:1052C0000500002010B5802000F028F8B8B180213A
:1052D0000B4800F01AFB60B90A4880680A49884206
:1052E00007DA0A48007820B906488068401C05495A
:1052F00088600A2005490870802000F009F810BD78
:10530000000801409802002040420F0004000020E5
:10531000014908607047000014040140064A014634
:1053200000201268044B0A4014331B680B4202D061
:10533000002A00D0012070470004014030B5837975
:105340001949026853B30B6893430B600A1D136835
:105350000468A343136002790A4413680468234372
:105360001360114A083213680468A3431360131DC5
:105370001C680568AC431C604479102C05D021449E
:105380000A68006802430A6030BD1168046821435E
:105390001160196800680143196030BD0079084444
:1053A00001689143016030BD000401407047000076
:1053B00004490A6822F010020A600A6802430A607F
:1053C000704700000020024004490A6802F03802D9
:1053D0000A600A6802430A60704700000020024029
:1053E000704710B5044640F27B1002F0E3FE08B9A6
:1053F000204610BDA4F52F70C0EB001000EB40005C
:10540000192101EB4000322190FBF1F000F57F7093
:10541000EFE700000146C1EBC100024A02EB800049
:10542000406970473CDC01080146C1EBC100024AFB
:1054300002EB8000006970473CDC01080146C1EBCB
:10544000C100024A02EB8000C06870473CDC0108E2
:105450000146C1EBC100024A52F82000704700002B
:105460003CDC010810B50446002300E05B1CC3EBE4
:10547000C300094901EB80008068A04207D0C3EB5C
:10548000C30051F820004FF6FF718842EED1184654
:10549000FFF7DEFF10BD00003CDC010870B50446DC
:1054A0004FF0FF3625460648854206DA40F23912AB
:1054B00000212846FCF752FA0646304670BD00002F
:1054C00078D4030008B50121480202F0CFFB012186
:1054D000084602F0B3FB0121084602F0C7FB012198
:1054E000042002F0C3FB0121082002F0BFFB0121D0
:1054F000102002F0BBFB0121202002F0B7FB0121AC
:10550000402002F0B3FB0121480402F0A3FB01217B
:10551000880402F09FFB0121082000F0CFF901214F
:10552000AE4800F0CBF98620ADF8000004208DF8DD
:10553000030003208DF802006946A94800F070F9C5
:105540004FF40070ADF8000003208DF80200182021
:105550008DF803006946A24800F062F94FF48060BC
:10556000ADF8000004208DF8030069469C4800F067
:1055700057F90120ADF8000003208DF80200042047
:105580008DF803006946964800F04AF92020ADF8EE
:10559000000003208DF8020010208DF803006946FA
:1055A0008F4800F03DF94FF4D050ADF800000320D3
:1055B0008DF8020010208DF803006946884800F03D
:1055C0002FF94FF47050ADF8000010208DF8030053
:1055D00003208DF802006946824800F021F940203E
:1055E000ADF8000003208DF8020014208DF80300B0
:1055F00069467C4800F014F98220ADF800000320D1
:105600008DF8020004208DF803006946754800F00B
:1056100007F90320ADF8000000208DF8030069466B
:10562000704800F0FDF82020ADF8000000208DF853
:10563000030069466C4800F0F3F84FF47070ADF861
:10564000000010208DF803006946674800F0E8F874
:105650001020ADF8000004208DF803006946624870
:1056600000F0DEF84FF20F00ADF8000003208DF8D7
:10567000020048208DF8030069465C4800F0D0F82D
:105680002020ADF8000003208DF8020018208DF8CE
:1056900003006946554800F0C3F84020ADF800000B
:1056A00003208DF8020004208DF8030069464F485E
:1056B00000F0B6F84FF48070ADF8000003208DF8CC
:1056C000020018208DF803006946484800F0A8F849
:1056D0004FF40070ADF8000003208DF802000420A4
:1056E0008DF803006946414800F09AF84FF449608C
:1056F000ADF8000003208DF8020010208DF80300A3
:1057000069463A4800F08CF80120ADF800001420FA
:105710008DF8030003208DF802006946344800F03C
:105720007FF88020ADF8000010208DF803000320E2
:105730008DF8020069462E4800F072F84FF47F4061
:10574000ADF8000003208DF8020028208DF803003A
:105750006946274800F064F80121002000F04CF869
:10576000022024490860002008710C2048710120A3
:1057700088710846FFF7E2FD0221002000F03CF8A6
:1057800004201C490860002008710C204871012089
:1057900088710846FFF7D2FD0721002000F02CF8A1
:1057A000802014490860002008710C2048710120F5
:1057B00088710846FFF7C2FD0421022000F01CF8A2
:1057C00010200C490860002008710C20487101204D
:1057D00088710846FFF7B2FD08BD000030001400D4
:1057E00000080140000C014000100140001401407D
:1057F000001801409400002010B58A0721F003042E
:105800000649130F21440F228C689A4094438C6000
:105810008A68984002438A6010BD00000000014081
:10582000F0B5CB78002503F00F02DB0601D58B78AD
:105830001A430B884FF00F0E13F0FF0F4FF0010CBF
:1058400019D004680E880CFA05F31E409E420ED152
:10585000AF000EFA07F6B44302FA07F7CE783C43DE
:10586000282E00D14361CE78482E00D103616D1CF3
:10587000082DE7D304600B88FF2B1DD94468002551
:1058800005F108060CFA06F30E881E409E420FD161
:10589000AF000EFA07F624EA060602FA07F43443CC
:1058A000CE78282E00D14361CE78482E00D10361F6
:1058B0006D1C082DE4D34460F0BD0000F0B5104D20
:1058C0006B68440D260184B2C0F30157B440C0F3A5
:1058D0000342032F05D0C0020AD503209040834322
:1058E00007E0686823F0706220F07060686002E092
:1058F000A34343F0706201B122436A60F0BD00002F
:1059000000000140806880B2704702460020926823
:105910000A4200D00120704702460020D2680A42A5
:1059200000D0012070474161704701617047C1603C
:105930007047000070B506463546472D00DA47250A
:105940001A48854200DD0546D2220021284602F091
:10595000AFFE441E012C00DA0124601C00EB400065
:10596000134951F8200004EB4401114A52F8211068
:10597000401A04EB440102EB81014968691A48436B
:10598000611C01EB410102EB8101496804EB440217
:10599000074B03EB82025268891A90FBF1F004EB8B
:1059A00044011A4652F82110084470BD54220E00DA
:1059B00094FE010810B504460748844209DA2046DF
:1059C000FFF76CFDC0EBC000044901EB800080686C
:1059D00010BD0020FCE7000078D403003CDC010887
:1059E00070B504460E48844218DA2046FFF756FD8B
:1059F000054600F017FC30B12046FFF7DBFF0546F7
:105A000002F0A8FC70BD2046FFF748FDC0EBC000C7
:105A1000044901EB800040680068F3E70020F1E7EB
:105A200078D403003CDC0108014600200022012953
:105A30001BDB062919DC072911D2DFE801F010046D
:105A400006080A0C0E00012209E0022207E00422E7
:105A500005E0082203E0102201E0202200BF00BF81
:105A6000024B1B68134003B901207047540000200B
:105A700002461146002900DA0021B1F5805F01DB02
:105A800040F6FF714FF47A704843C1F5805390FBA4
:105A9000F3F0704710B54FF4C17002F08BFBB8B152
:105AA00010480468B4F5967F03DB40F2145084423A
:105AB00007DD0D48006820B90121002003F0D4FC67
:105AC0000EE00A4804600121002002F013FE07E006
:105AD0004FF42F70054908600121002002F00AFEF2
:105AE00010BD0000780A0020AC0000203400002027
:105AF000014601F114006422504340F6FF7290FB0E
:105B0000F2F07047024B1970024B1870704700009A
:105B10002E0100202D01002000BFFEE770477047D6
:105B20007047704710B501210148FFF7FEFE10BD18
:105B30000018014002494CF6CC4008607047000054
:105B40000030004002494AF6AA2008607047000071
:105B500000300040014948607047000000300040BC
:105B6000014988607047000000300040014908602A
:105B7000704700000030004010B545F25550FFF767
:105B8000F5FF0520FFF7E6FF40F6C410FFF7E8FF3A
:105B9000FFF7D8FFFFF7CEFF10BD000070B5C64875
:105BA0000078002843D0C5480068CD225043C44A3D
:105BB00002EB800001228168002001F067F80321D8
:105BC0000220FFF79FFF02F019FE04F0BDFF04461C
:105BD000002100F053FF04F0B7FFC4B200230122FC
:105BE0002146184601F08EF904F0AEFFC4B200223F
:105BF0002146104600F0A4FE04210846FFF782FF6C
:105C000000220821022001F0DFFE002209210220EB
:105C100001F0DAFE00220921022001F0D5FE002267
:105C20000921022001F0D0FE0020A349087004F0F1
:105C30008BFFA44901EB001005682846FFF72EFCF6
:105C4000044600F009FBC0F30A0100297ED1C0120E
:105C50002A287BD2DFE800F0151718197A7A7A7AA9
:105C60007A517A7A1A1B1C1D1E7A7A2450167A7A77
:105C7000259126271F202122237A7A7A3C7A287AB6
:105C80007AD900BF00BF00BF00BF00BF00BF00BF88
:105C900000BF00BF00BF00BF00BF00BF00BF00BF0C
:105CA00000BF00BF00BF00BF00220A21022001F098
:105CB0008BFE04F049FF834901EB00100468204685
:105CC000FFF78EFE80490860062080490860F1E0F9
:105CD00000220A21022001F077FE04F035FF794905
:105CE00001EB001004682046FFF77AFE7649086051
:105CF0001B2076490860DDE000BF00220B21022056
:105D000001F062FE05210820FFF7FCFE0022892138
:105D1000012001F059FE6E480078001D6C490870A2
:105D200000228921012001F04FFE69480078001D02
:105D30006749087000223A21012001F045FE6448BD
:105D40000078001D62490870002200E0A5E089216A
:105D5000012001F039FE5E480078001D5C490870A2
:105D600000228921012001F02FFE05210820FFF7E4
:105D7000C9FE0720554908609CE000220B21022043
:105D800001F022FE05210820FFF7BCFE0022892138
:105D9000012001F019FE4E480078001D4C490870A2
:105DA00000228921012001F00FFE49480078001DE2
:105DB0004749087000228921012001F005FE44486E
:105DC0000078001D4249087000222D21012001F0B9
:105DD000FBFD3F480078001D3D49087000228921E5
:105DE000012001F0F1FD3A480078001D38490870A3
:105DF00000228921012001F0E7FD05210820FFF79D
:105E000081FE08203149086054E004F09DFE2D49D0
:105E100001EB001004682046FFF7E2FD2A49086004
:105E200000220B21022001F0CFFD05210820FFF701
:105E300069FE25480068010E0022012001F0C4FD22
:105E400023480078001D2249087000221E4800687F
:105E5000C0F30741012001F0B7FD1D480078001D87
:105E60001B490870002218480088C0F30721012050
:105E700001F0AAFD16480078001D15490870124867
:105E800001780022012001F09FFD05210820FFF785
:105E900039FE1C200D4908600CE000220B21022075
:105EA00001F092FD05210820FFF72CFE092007498B
:105EB000086000BF00BF70BD3701002080010020D6
:105EC000004D0208302A0020C00100209801002067
:105ED0002D01002070B505460C46B548007808280D
:105EE0007BDCB3480078082814DAB2480068B0F5C3
:105EF000FA7F05DA00225F21012001F065FD04E050
:105F000000222021012001F05FFDAB4800780B3812
:105F1000A94908704B2D7BD00CDC2B2D79D004DCEB
:105F20001D2D14D0272D2AD114E12D2D72D02E2D08
:105F3000F9D1C3E08B2D57D004DC4D2D6BD04E2D05
:105F4000F1D16FE08D2D34D08E2DECD118E0984832
:105F50000078082813DA3021954802780078401C30
:105F6000934B18709548815424B90022012001F008
:105F70002BFD04E000222A21012001F025FD15E17E
:105F80008B480078082813DA312189480278007894
:105F9000401C874B18708948815424B90022012085
:105FA00001F012FD04E000222A21012001F00CFD85
:105FB000FCE07F480078082815DA32227C48017816
:105FC0000078401C7A4B18707C48425434B9002247
:105FD0003221012001F0F8FC05E0E8E000222A214E
:105FE000012001F0F1FCE1E071480078082818DA9E
:105FF00033226F4801780078401C6D4B18706F4851
:1060000042544CB900223321012001F0DDFC08E0AC
:106010003BE085E06BE01FE000222A21012001F037
:10602000D3FCC3E062480078082814DA34226048C0
:1060300001780078401C5E4B1870604842542CB9BF
:1060400000223421012001F0BFFC04E000222A21BB
:10605000012001F0B9FCA9E055480078082813DABE
:106060003521534802780078401C514B1870534832
:10607000815424B90022012001F0A6FC04E0002292
:106080002A21012001F0A0FC90E04948007808286E
:1060900013DA3621464802780078401C444B1870C9
:1060A0004648815424B90022012001F08DFC04E00F
:1060B00000222A21012001F087FC77E03C4800788B
:1060C000082813DA37213A4802780078401C384B08
:1060D00018703A48815424B90022012001F074FC60
:1060E00004E000222A21012001F06EFC5EE030482D
:1060F0000078082813DA38212D4802780078401CEF
:106100002B4B18702D48815424B90022012001F036
:106110005BFC04E000222A21012001F055FC45E04F
:1061200023480078082814DA3922214801780078B9
:10613000401C1F4B1870214842542CB900223921B1
:10614000012001F041FC04E000222A21012001F09D
:106150003BFC2BE016480078002826DD1448007828
:10616000401E1349087000201449114A12788854BF
:106170000F480078072809DA00222021012001F0C9
:1061800023FC0D4800780B380B4908700A4800784A
:106190000B380949087000222021012001F014FC6D
:1061A000054800780B380449087000BF00BF70BD77
:1061B00035010020140000202D01002039010020AD
:1061C00010B510210448FFF7B0FB4FF4806103487D
:1061D000FFF7A9FB012010BD00080140001001409D
:1061E000014608480068CD225043074A02EB800070
:1061F000143000EB0110C068006808B1012070473E
:106200000020FCE780010020004D02080146C1EBA0
:10621000C100034A02EB8000008B00F4FE6070476F
:106220003CDC01080146C1EBC100034A02EB8000DF
:10623000007EC0F3400070473CDC01080146C1EB22
:10624000C100044A02EB8000007E00F0010080F0F3
:10625000010070473CDC01080146C1EBC100034A64
:1062600002EB8000806900F4FF2070473CDC0108ED
:106270000146C1EBC100054A52F820004FF6FF72FB
:10628000904201D1012070470020FCE73CDC01086E
:106290000146CD204843054A02EB8000C0680068F3
:1062A00008B1012070470020FCE70000004D020803
:1062B00038B500250820ADF8000010208DF8030047
:1062C00003208DF8020069464A48FFF7A9FA082121
:1062D0004848FFF728FBFCF7DDFE4648FFF712FBB6
:1062E00004130820ADF8000048208DF8030069462B
:1062F0004048FFF795FA0F2C76D10420ADF8000046
:1063000010208DF8030003208DF8020069463948FB
:10631000FFF786FA04213748FFF705FBFCF7BAFEC2
:106320003448FFF7EFFA04130420ADF800004820CA
:106330008DF8030069462F48FFF772FA0F2C4FD1F2
:106340000220ADF8000010208DF8030003208DF826
:10635000020069462748FFF763FA02212548FFF744
:10636000E2FAFCF797FE2348FFF7CCFA0413022069
:10637000ADF8000048208DF8030069461D48FFF77E
:106380004FFA0F2C27D10120ADF8000010208DF816
:10639000030003208DF8020069461648FFF740FA13
:1063A00001211448FFF7BFFAFCF774FE1148FFF70C
:1063B000A9FA04130120ADF8000048208DF803006D
:1063C00069460C48FFF72CFA0F2C00D10FE0E0B221
:1063D00040F010050BE0E0B240F0200507E003E0DC
:1063E000E0B240F0400502E0E0B240F0800528460F
:1063F00038BD00000014014070B500F035F80024ED
:1064000017E0002511E0A107080E294603F0B6F8B1
:10641000002606E000222146012003F0D9FF701C6F
:10642000C6B2402EF6DB681CC5B2082DEBDB601C43
:10643000C4B2022CE5DB00F023F870BD10B548F2C1
:1064400020010748FFF76FFA4FF480410448FFF737
:106450006CFA40210348FFF766FAFFF7CDFF10BD45
:10646000000C01400008014010B53E220021084602
:1064700003F0AEFF3E220121002003F0A9FF10BD72
:1064800010B53F220021084603F0A2FF3F22012160
:10649000002003F09DFF10BD70B505460C466E2030
:1064A0001C490870012D28D11B480068C8280CDA47
:1064B00000201A490870E2B2FE2101F085FAE2B22A
:1064C0002021002001F080FA23E013480068B0F595
:1064D000FA7F1EDD10480068B0F52F7F19DA012021
:1064E0000E490870E2B2F821002001F06DFAE2B224
:1064F0002021002001F068FA0BE0022D09D1E2B260
:10650000F721002001F060FAE2B2FD21002001F045
:106510005BFA70BD2D01002014000020CC0100208A
:1065200000BFFEE77047000010B54FF48031C8028D
:1065300000F0A0F84FF4E06000F092F8284800F076
:1065400051F82620264908700020487001208870E4
:10655000C870084600F046F827202149087000203E
:10656000487001208870C870084600F03BF803208E
:106570001B49087000204870022088700120C870F4
:10658000084600F02FF807201549087000204870D1
:1065900088700120C870084600F024F808201049CF
:1065A00008700020487088700120C870084600F00C
:1065B00019F80A200A4908700020487088700120E4
:1065C000C870084600F00EF8172005490870002032
:1065D000487088700120C870084600F003F810BDAC
:1065E0008D000020F0B50F22C378017801244FF010
:1065F000E0263BB3184B1B6803F4E063C3F5E0638C
:106600001D0AC5F10403EA4045789D408378134094
:106610002B431A018B07DF0E21F003030F49BA4009
:106620005D182968FF23BB4099431A401143296034
:10663000007800F01F018C40400906EB8000C0F894
:106640000041F0BD01F01F008440480906EB8000C6
:10665000C0F88041F0BD00000CED00E000E400E077
:106660000249084302490860704700000000FA052B
:106670000CED00E0024A11400143024801607047FE
:1066800080FFFF1F08ED00E010B50848006820B942
:1066900001200649086003F05BFA02F091FF03F065
:1066A0000FF801F0D3FD0446204610BDA4010020E0
:1066B00070470000014908627047000000000E4268
:1066C00070472DE9F04180460C4615461E4604F100
:1066D000910003F0E3F8074685B104E0324620213B
:1066E000404601F071F938467F1C0628F6DB324639
:1066F00004F19101404603F009FF0FE0324604F136
:106700009101404603F002FF04E03246202140465A
:1067100001F05AF938467F1C0628F6DBBDE8F08107
:10672000704770472DE9F04107460D4690461E46DA
:1067300080240C4800780C380A4908700EE005EAFD
:10674000040028B132463021384601F03DF904E01A
:1067500032463121384601F037F96410002CEED171
:10676000BDE8F0812D0100202DE9F04106460C46E0
:1067700090461D460020244908702A4620213046B4
:1067800001F022F90A2094FBF0F00A2190FBF1F2CB
:1067900001FB12003030C7B22A463946304601F0BC
:1067A00013F90A2094FBF0F100FB11403030C7B21E
:1067B0002A463946304601F007F92A462D2130464F
:1067C00001F002F94FF47A7094FBF0F00A2190FB8B
:1067D000F1F201FB12003030C7B22A46394630468A
:1067E00001F0F2F8642094FBF0F00A2190FBF1F242
:1067F00001FB12003030C7B22A463946304601F05C
:10680000E3F8BDE8F08100002C0100202DE9F047FD
:106810000746884691461E46474800783038464924
:106820000870464D2C6804F00F00FAF788FF824686
:1068300032465146384601F0C7F8C4F30320FAF750
:106840007EFF824632465146384601F0BDF8C4F319
:106850000340FAF774FF824632465146384601F04B
:10686000B3F8C4F30360FAF76AFF82463246514632
:10687000384601F0A9F832462D21384601F0A4F837
:106880002D1D2C6804F00F00FAF759FF824632469E
:106890005146384601F098F8C4F30320FAF74FFF49
:1068A000824632465146384601F08EF8C4F3034022
:1068B000FAF745FF824632465146384601F084F8E1
:1068C000C4F30360FAF73BFF82463246514638462E
:1068D00001F07AF832462D21384601F075F82D1D69
:1068E0002C6804F00F00FAF72AFF82463246514620
:1068F000384601F069F8C4F30320FAF720FF824616
:1069000032465146384601F05FF8C4F30340FAF7C7
:1069100016FF824632465146384601F055F8C4F318
:106920000360FAF70CFF824632465146384601F0C2
:106930004BF8BDE8F08700002D010020E8F7FF1FAD
:106940002DE9F04105460C4616467120494908706C
:10695000494901EB04110868FEF7A0FD8046FFF7E6
:1069600055FC074607F00F0000287AD1381115288A
:1069700077D2DFE800F0760B1C222876762E343AA8
:1069800040464C52585E767664766B0040F27B103F
:1069900001F010FC28B932460021284603F0B6FD6C
:1069A00004E032460F21284603F0B0FD5FE0324696
:1069B0000121284603F0AAFD59E03246022128466B
:1069C00003F0A4FD53E032460321284603F09EFD68
:1069D0004DE032460421284603F098FD47E0324658
:1069E0000521284603F092FD41E032460621284663
:1069F00003F08CFD3BE032460721284603F086FD7C
:106A000035E032460821284603F080FD2FE032466B
:106A10000921284603F07AFD29E032460A2128465A
:106A200003F074FD23E032460B21284603F06EFD8F
:106A30001DE032460C21284603F068FD17E032467F
:106A40000D21284603F062FD11E00AE03246F021F4
:106A5000284600F0B9FF3246F521284600F0B4FF81
:106A600005E032460E21284603F050FD00BF00BF6E
:106A7000BDE8F0812D010020302A002070B50446C9
:106A80000D46074800EB04102A464168002003F039
:106A90003DFD2A460E21002003F038FD70BD0000A8
:106AA000302A00202DE9F04105460C461646002705
:106AB000672001F07FFB06283FD2DFE800F0030CDF
:106AC00016202A3404EB4401234A52F83100F9F726
:106AD00077FD074631E004EB44011F4A02EBC10198
:106AE0004868F9F76DFD074627E004EB44011A4AB0
:106AF00002EBC1018868F9F763FD07461DE004EB6E
:106B00004401154A02EBC101C868F9F759FD07466F
:106B100013E004EB4401104A02EBC1010869F9F7E4
:106B20004FFD074609E004EB44010B4A02EBC101AB
:106B30004869F9F745FD074600BF00BF07EB47006E
:106B4000C0F140000549087032462146284603F04E
:106B5000DDFCBDE8F0810000F83902082D010020BD
:106B600010B500210846FEF7CDFF0022022108469D
:106B700000F02AFF00212020FEF7C4FF002203219D
:106B8000022000F021FF00214020FEF7BBFF002281
:106B90000321022000F018FF00216020FEF7B2FF61
:106BA00000220421022000F00FFF04210020FEF744
:106BB000A9FF00220521022000F006FF0421202069
:106BC000FEF7A0FF00220621022000F0FDFE0421B6
:106BD0004020FEF797FF00220621022000F0F4FE7D
:106BE00004216020FEF78EFF00220721022000F022
:106BF000EBFE10BD10B50020224908702249087034
:106C000000220D21022000F0DFFE20201D49087027
:106C100000220E21022000F0D7FE40201949087002
:106C200000220E21022000F0CFFE602015490870DE
:106C300000220F21022000F0C7FE00201149087039
:106C400004201149087000221021022000F0BCFE2F
:106C500020200C49087000221121022000F0B4FE0F
:106C600040200849087000221121022000F0ACFEEB
:106C700060200449087000221221022000F0A4FEC6
:106C800010BD00002D0100202E01002070B504462B
:106C90000D461646FFF764FF00210846FEF732FF57
:106CA000324629462046FFF7FDFE70BD2DE9F04132
:106CB00080460C4615461E4604F1160002F0EEFD15
:106CC000074685B104E032462021404600F07CFEB4
:106CD00038467F1C0628F6DB324604F11601404692
:106CE00003F014FC0FE0324604F11601404603F0B5
:106CF0000DFC04E032462021404600F065FE384697
:106D00007F1C0628F6DBBDE8F0812DE9F041064640
:106D10000D461746284601F04DFA0446210E3A4624
:106D2000304600F051FE3A46C4F30741304600F0C9
:106D30004BFE3A46C4F30721304600F045FEE1B26F
:106D40003A46304600F040FEBDE8F0812DE9F041C2
:106D500007460C4615461E4605B3324620213846E6
:106D600000F032FE32462021384600F02DFE210E82
:106D70003246384600F028FE3246C4F30741384612
:106D800000F022FE3246C4F30721384600F01CFE14
:106D9000E1B23246384600F017FE1FE0210E3246BF
:106DA000384600F011FE3246C4F30741384600F081
:106DB0000BFE3246C4F30721384600F005FEE1B26F
:106DC0003246384600F000FE32462021384600F0B8
:106DD000FBFD32462021384600F0F6FDBDE8F0818B
:106DE000704700002DE9F04106460C4690461D46CE
:106DF000002029490870294894FBF0F00A2190FBF3
:106E0000F1F201FB12003030C7B22A463946304653
:106E100000F0DAFD42F2107094FBF0F00A2190FBD2
:106E2000F1F201FB12003030C7B22A463946304633
:106E300000F0CAFD4FF47A7094FBF0F00A2190FB49
:106E4000F1F201FB12003030C7B22A463946304613
:106E500000F0BAFD2A462D21304600F0B5FD0A208B
:106E600094FBF0F00A2190FBF1F201FB12003030AC
:106E7000C7B22A463946304600F0A6FD0A2094FBE8
:106E8000F0F100FB11403030C7B22A463946304697
:106E900000F09AFDBDE8F0812C010020A0860100E1
:106EA00070472DE9F04180460C4615461E4604F118
:106EB000100002F0F3FC074685B104E032462021C1
:106EC000404600F081FD38467F1C0628F6DB32463E
:106ED00004F11001404603F019FB0FE0324604F1C3
:106EE0001001404603F012FB04E0324620214046E8
:106EF00000F06AFD38467F1C0628F6DBBDE8F0810D
:106F0000704700002DE9F84F06460D461746984693
:106F1000A34901EB05110868FEF7C0FA8246FFF7A6
:106F20009BF981469E4901EB05110868FEF758FD63
:106F300004464C209B490870C9F30A00002822D15E
:106F40004FEAE9202A281ED2DFE800F0A11D1D1D0E
:106F5000151E2F363D44521D97ABB5BF1D73251D21
:106F6000901DDD1D1DFEC91DD31D1D1D1DFDFC1D1C
:106F70001D4BFB1D1DFA062043463A462146009054
:106F8000304600F0A5FC08E143463A46214630462B
:106F900000F03CFC01E140208249087043463A463B
:106FA0002146304600F05CF9F7E043463A46214678
:106FB000304600F0C9FBF0E043463A4621463046F1
:106FC00000F018FAE9E043463A462146304600F020
:106FD000EBF8E2E043463A462146304600F0B4F989
:106FE000DBE043463A462146304600F065FAD4E0FD
:106FF00040F27B1001F0DEF830B943463A462146B4
:10700000304600F0D1FA13E0A4F52F70C0EB001069
:1070100000EB4000192101EB4000322190FBF1F020
:1070200000F57F7A43463A465146304600F0BCFAB6
:10703000B3E040F27B1001F0BDF830B943463A4668
:107040002146304600F0E2FB0FE0C4EB041000EBF9
:107050004000192101EB4000322190FBF1FA434638
:107060003A465146304600F0D1FB96E043463A4658
:1070700021463046FFF778FB8FE04C2049490870E5
:1070800043463A4621463046FFF71BFB85E04C203D
:107090004449087043463A4621463046FFF706FE0B
:1070A0007BE04C203F49087043463A462146304633
:1070B000FFF7F6FE71E04C203A49087043463A4625
:1070C00021463046FFF72DFB67E04C20354908701C
:1070D00043463A4621463046FFF782FE5DE04C20AB
:1070E0003049087043463A4621463046FFF708FFCC
:1070F00053E04C202B49087043463A46214630461F
:10710000FFF7CFFE49E040F27B1001F053F830B9B1
:1071100043463A462146304600F0AEFA19E0A4F55F
:107120002F70C0EB001000EB4000192101EB400074
:10713000322190FBF1F000F52F7A43463A4604E005
:1071400024E01CE00DE005E012E05146304600F07E
:1071500093FA22E043463A4621463046FFF7E2FAE8
:107160001BE043463A4621463046FFF74FFB14E00A
:1071700043463A4621463046FFF734FE0DE043468B
:107180003A4621463046FFF7CBFA06E043463A46F8
:1071900021463046FFF7DAFD00BF00BFBDE8F88F9B
:1071A000302A00202D0100202DE9F04106460C4632
:1071B00090461D4600202949087042F2107094FB49
:1071C000F0F00A2190FBF1F201FB12003030C7B25F
:1071D0002A463946304600F0F7FB2A462E21304633
:1071E00000F0F2FB4FF47A7094FBF0F00A2190FB70
:1071F000F1F201FB12003030C7B22A463946304660
:1072000000F0E2FB642094FBF0F00A2190FBF1F225
:1072100001FB12003030C7B22A463946304600F032
:10722000D3FB0A2094FBF0F00A2190FBF1F201FB62
:1072300012003030C7B22A463946304600F0C4FB4F
:107240000A2094FBF0F100FB11403030C7B22A460F
:107250003946304600F0B8FBBDE8F0812C01002033
:107260002DE9F04106460C4617461D4600203449DC
:107270000870344894FBF0F000F0FF082B463A46C3
:107280004146002000F088FC42F2107094FBF0F0C0
:107290000A2190FBF1F201FB1200303000F0FF08F0
:1072A0002A464146304600F08FFB2A462E213046C2
:1072B00000F08AFB4FF47A7094FBF0F00A2190FB07
:1072C000F1F201FB1200303000F0FF082A4641467F
:1072D000304600F079FB642094FBF0F00A2190FB2B
:1072E000F1F201FB1200303000F0FF082A4641465F
:1072F000304600F069FB2A462E21304600F064FB40
:107300000A2094FBF0F00A2190FBF1F201FB12003D
:10731000303000F0FF082A464146304600F054FB6A
:107320000A2094FBF0F100FB1140303000F0FF0820
:107330002A464146304600F047FBBDE8F081000098
:107340002C010020A08601002DE9F04107460C46E3
:1073500015461E4625B132462021384600F034FB42
:107360004FF4167094FBF0F00A2190FBF1F201FB50
:107370001200303000F0FF0832464146384600F037
:1073800023FB3C2094FBF0F00A2190FBF1F201FB7F
:107390001200303000F0FF0832464146384600F017
:1073A00013FB32463A21384600F00EFB3C2094FB9A
:1073B000F0F100FB11400A2190FBF1F0303000F0B9
:1073C000FF0832464146384600F0FEFA3C2094FB66
:1073D000F0F100FB11400A2190FBF1F201FB1200D9
:1073E000303000F0FF0832464146384600F0ECFAF3
:1073F000BDE8F0812DE9F04106460C4617461D46D2
:1074000000202C49087042F2107094FBF0F06421C7
:1074100090FBF1F201FB120000F0FF082B463A4608
:107420004146304600F0B8FB4FF47A7094FBF0F020
:107430000A2190FBF1F201FB1200303000F0FF084E
:107440002A464146304600F0BFFA2A462E213046F1
:1074500000F0BAFA642094FBF0F00A2190FBF1F2FC
:1074600001FB1200303000F0FF082A46414630464A
:1074700000F0AAFA0A2094FBF0F00A2190FBF1F246
:1074800001FB1200303000F0FF082A46414630462A
:1074900000F09AFA0A2094FBF0F100FB1140303022
:1074A00000F0FF082A464146304600F08DFABDE85C
:1074B000F08100002C0100202DE9F84307460D461D
:1074C00090461E460020374908702C46B4F52F7FA1
:1074D0000ADBA4F52F74062033464246214600906D
:1074E000384600F0F5F95BE000202E490870C4F53D
:1074F0002F7442F2107094FBF0F00A2190FBF1F22D
:1075000001FB120000F0FF09334642464946384667
:1075100003F0C2F84FF47A7094FBF0F00A2190FB6C
:10752000F1F201FB120000F0FF09334642464946E2
:10753000384603F0B1F8642094FBF0F00A2190FB88
:10754000F1F201FB120000F0FF09334642464946C2
:10755000384603F0A1F80A2094FBF0F00A2190FBD2
:10756000F1F201FB120000F0FF09334642464946A2
:10757000384603F091F80B48007820B932462D21A7
:10758000384600F021FA0A2094FBF0F100FB11408C
:10759000303000F0FF0932464946384600F014FA10
:1075A000BDE8F8832C0100202DE9F04707460D4681
:1075B00090461E462C46B4F52F7F08DBA4F52F74A9
:1075C000334642462146384600F020F94FE000207D
:1075D00028490870C4F52F744FF47A7094FBF0F0CA
:1075E0000A2190FBF1F201FB120000F0FF09334683
:1075F00042464946384603F04FF8642094FBF0F0C9
:107600000A2190FBF1F201FB120000F0FF09334662
:1076100042464946384603F03FF81648007820B9FC
:1076200032462D21384600F0CFF90A2094FBF0F0C5
:107630000A2190FBF1F201FB1200303000F0FF094B
:1076400032464946384600F0BFF932462E213846C8
:1076500000F0BAF90A2094FBF0F100FB1140303041
:1076600000F0FF0932464946384600F0ADF9BDE862
:10767000F08700002C0100202DE9F04707460D4659
:1076800090461E462C46B4F52F7F08DBA4F52F74D8
:10769000334642462146384600F0B8F84FE0002015
:1076A00028490870C4F52F744FF47A7094FBF0F0F9
:1076B0000A2190FBF1F201FB120000F0FF093346B2
:1076C00042464946384602F0E7FF642094FBF0F05A
:1076D0000A2190FBF1F201FB120000F0FF09334692
:1076E00042464946384602F0D7FF1648007820B98E
:1076F00032462D21384600F067F90A2094FBF0F05D
:107700000A2190FBF1F201FB1200303000F0FF097A
:1077100032464946384600F057F932462E2138465F
:1077200000F052F90A2094FBF0F100FB11403030D8
:1077300000F0FF0932464946384600F045F9BDE8F9
:10774000F08700002C0100202DE9F04106460C4690
:1077500017461D4600202C49087042F2107094FB19
:10776000F0F00A2190FBF1F201FB120000F0FF089B
:107770002B463A464146304600F00EFA4FF47A70F6
:1077800094FBF0F00A2190FBF1F201FB120000F0F3
:10779000FF082B463A464146304600F0FDF964208A
:1077A00094FBF0F00A2190FBF1F201FB1200303063
:1077B00000F0FF082A464146304600F005F92A4607
:1077C0002E21304600F000F90A2094FBF0F00A2147
:1077D00090FBF1F201FB1200303000F0FF082A4666
:1077E0004146304600F0F0F80A2094FBF0F100FB2F
:1077F0001140303000F0FF082A464146304600F084
:10780000E3F8BDE8F08100002C0100202DE9F041F3
:1078100006460C4617461D4600202C49087042F2C9
:10782000107094FBF0F00A2190FBF1F201FB1200C2
:1078300000F0FF082B463A464146304600F0ACF9CE
:107840004FF47A7094FBF0F00A2190FBF1F201FB07
:10785000120000F0FF082B463A464146304600F041
:107860009BF9642094FBF0F00A2190FBF1F201FBFC
:10787000120000F0FF082B463A464146304600F021
:107880008BF90A2094FBF0F00A2190FBF1F201FB46
:107890001200303000F0FF082A464146304600F022
:1078A00093F82A462E21304600F08EF80A2094FBE9
:1078B000F0F100FB1140303000F0FF082A4641464D
:1078C000304600F081F8BDE8F08100002C01002076
:1078D0002DE9F04707460C4690461E46089D0020BD
:1078E00037490870062D0FDB364894FBF0F00A216B
:1078F00090FBF1F201FB120000F0FF093346424613
:107900004946384600F048F9052D10DB42F2107068
:1079100094FBF0F00A2190FBF1F201FB120000F061
:10792000FF09334642464946384600F035F9042DF2
:1079300010DB4FF47A7094FBF0F00A2190FBF1F227
:1079400001FB120000F0FF09334642464946384623
:1079500000F022F9032D0FDB642094FBF0F00A21E4
:1079600090FBF1F201FB120000F0FF0933464246A2
:107970004946384600F010F9022D0FDB0A2094FB2F
:10798000F0F00A2190FBF1F201FB120000F0FF0978
:10799000334642464946384600F0FEF8012D0CDBDE
:1079A0000A2094FBF0F100FB1140303000F0FF0999
:1079B00032464946384600F007F8BDE8F087000037
:1079C0002C010020A086010070B506460C46154625
:1079D00026B1012E07D0022E0FD109E029462046FC
:1079E00000F00EF809E02946204600F043F804E0D4
:1079F0002946204600F08AF800BF00BF70BD000095
:107A00002DE9F04105460E46002706B1FF27202D3F
:107A100000DA202500241EE013480078802818DAB8
:107A2000124801781048007801F0A8FDA5F1200067
:107A30000F4B03EBC000005D80EA07020A480078A4
:107A40008111012002F0C4FC07480078401C06495F
:107A50000870601CC4B2082CDEDB03480078801E6E
:107A600001490870BDE8F0812D0100202E010020A1
:107A7000780C02082DE9F04105460F464FF000084A
:107A80000FB14FF0FF08202D00DA202500242DE053
:107A9000002622E01A48007880281CDA194800786D
:107AA0002044C1B21648007801F068FDA5F120001D
:107AB000154B03EB401006EB0413C05C80EA080290
:107AC0000F4800788111012002F082FC0C480078F8
:107AD000401C0B490870701CC6B2102EDADB084837
:107AE0000078103806490870601CC4B2022CCFDB45
:107AF000034800780B3002490870BDE8F0810000AF
:107B00002D0100202E010020801302082DE9F041F4
:107B100006460F464FF000080FB14FF0FF08002453
:107B20002BE0002520E01948007880281ADA184850
:107B300000782044C1B21548007801F01FFD1548B7
:107B400000EBC61005EB4413C05C80EA08020F4846
:107B500000788111012002F03BFC0C480078401CA9
:107B60000A490870681CC5B2202DDCDB0748007884
:107B7000203806490870601CC4B2042CD1DB0348CD
:107B80000078163001490870BDE8F0812D01002011
:107B90002E010020A02F02082DE9F04107460C46D7
:107BA00015461E4614B90B48007850B1012009490A
:107BB000087004F13000C1B232463846FFF704FFC6
:107BC00005E025B1324620213846FFF7FDFEBDE82D
:107BD000F08100002C01002010B504460F48104928
:107BE000096840F821400E480068401C142190FBB1
:107BF000F1F201FB12000A490860084600680949D1
:107C00000968884204D10221012001F02DFC03E023
:107C10000221002000F06EFD10BD0000AC0C002021
:107C2000C4000020C0000020034A516821F44041F4
:107C3000014351607047000000100240044A0029CF
:107C4000516901D0014300E0814351617047000058
:107C500000100240044A0029D16901D0014300E02C
:107C60008143D1617047000000100240044A00299E
:107C7000916901D0014300E08143916170470000A8
:107C80000010024010B500F035F84FF4803000F0DD
:107C9000C3F800F029F91649087008460078012851
:107CA00024D11020FDF784FB0220FDF78DFB00207E
:107CB00000F0A8F8002000F0E5F84FF4806000F034
:107CC000D7F84FF44040FFF7AFFF00214FF480306A
:107CD00000F0E8F8012000F0DFF800BF392000F0E4
:107CE00079F80028FAD0022000F0F4F810BD000066
:107CF0008C0000200B48016841F0010101604168DF
:107D0000094A114041600168084A11400160016858
:107D100021F480210160416821F4FE0141600021CD
:107D200081607047001002400000FFF8FFFFF6FE80
:107D3000224A10B55168224B11F00C0103D00429DE
:107D400003D0082903D0036015E01E4912E05168F2
:107D5000022301F4701103EB9141536813F4803F47
:107D600004D053689B0303D5174B02E0174B00E088
:107D7000144B594301605168154B01F0F00109099A
:107D80005C5C0168E1404160546804F4E064240AEA
:107D90001C5D21FA04F48460546804F46054E40A1D
:107DA0001B5DD940C1605268094B02F44042920BFE
:107DB0001B1F9A5CB1FBF2F1016110BD0010024083
:107DC00000127A0040787D0120BCBE0000093D0011
:107DD0009E4003080246002053090949012B0BD09D
:107DE000022B0BD0D1F8241002F01F020123934084
:107DF0000B4200D0012070470968F5E7096AF3E7F4
:107E000000100240034A516821F0F0010143516023
:107E100070470000001002400B490A6822F48032CB
:107E20000A600A6822F480220A60B0F5803F07D019
:107E3000B0F5802F03D1086840F4A0200860704797
:107E4000086840F48030F9E70010024070470000F5
:107E5000064900220A7001F82029012802D00428CE
:107E600002D1052081F82000704700002010024058
:107E7000034A516821F4E0610143516070470000FA
:107E80000010024003494A6822F4605242EAC000EE
:107E900048607047001002400149086670470000C2
:107EA00000004242034A5368084323F47C131843FA
:107EB00050607047001002400149086070470000A0
:107EC0003C04424202490A6A02430A6270470000C7
:107ED00000100240034A516821F003010143516040
:107EE000704700000010024030B50B4C40F2FF1507
:107EF0003120FFF76FFF20706068401C60602078C1
:107F000010B96068A842F3D13120FFF763FF002861
:107F100000D0012030BD000080020020704700002A
:107F200002490A8882430A80704700000428004002
:107F300010B54FF47A7400BF01214FF0C050FFF725
:107F400089FE0120FEF7B6FB0120FFF781FF2848DC
:107F5000046042F21070844201DA04F5FA7400BF42
:107F60004120FFF737FF18B9214800680028F7D1F2
:107F70004120FFF72FFFE8B90020FFF769FF00203D
:107F8000FEF798FB00214FF0C050FFF763FE4FF45F
:107F900080611848FDF7C9FC4FF4FA701449086075
:107FA00000BF134800680028FBD14FF480611148DE
:107FB000FDF7B9FC4120FFF70DFF0028BCD04FF4BE
:107FC0008070FFF77FFF0120FFF776FF00F0E6F8F3
:107FD00000F0DCF80121084600F05CF800F0D6F86B
:107FE00047F6FF7000F0C2F800F0D0F810BD0000B6
:107FF00018000020000C01400248018841F01001E7
:1080000001807047042800400248018821F01001D7
:108010000180704704280040034800880249091F76
:10802000098840EA014070471C2800400649098839
:10803000054A0140121FC9B21288024202D009B19A
:1080400001207047002070470428004010B501202F
:10805000FFF7ECFFB0B10120FFF762FF01200A49F2
:108060000870FFF7D9FF094988420BD30848007808
:10807000401C07490870FFF7CFFF0449441A204607
:1080800000F064F810BD00000000002080510100E5
:1080900001000020044A0029118801D0014300E0BA
:1080A00081431180704700000028004010B5012175
:1080B0004FF0C050FFF7CEFD0120FEF7FBFA042081
:1080C000F9F752FB4AF2A55188422FD0FFF730FF53
:1080D00000F05CF84AF6C00000F038F800F056F8FE
:1080E0004AF2A5510420F9F745FB00210820F9F7D1
:1080F00041FB00210C20F9F73DFB00211020F9F78E
:1081000039FB00211420F9F735FB00211820F9F77D
:1081100031FB00211C20F9F72DFB00212020F9F76D
:1081200029FB00212420F9F725FB0DE04120FFF772
:1081300051FE08B9FFF7FCFE00F030F801210846B7
:10814000FFF7A8FF00F022F810BD000000B50246BE
:10815000FFF752FF0449100C0880081D02805DF8EB
:1081600004EBFFF751BF00001828004000B502469D
:10817000FFF742FF0449C2F303400880081D028054
:108180005DF804EBFFF740BF082800400248018873
:108190008906FCD570470000042800400448018887
:1081A00021F00801018001880907FCD57047000013
:1081B0000428004010B50446204600F0CBF810BD5E
:1081C00070B54FF4C970FFF7F5FF0546002D01DBD0
:1081D000322D00DB0025681E051E00DA31252C46F5
:1081E00002221848016818480068FAF74BFE00BFE1
:1081F00004F29310FFF7DEFF064600F0FDFF2C208F
:1082000000F0A2FF04F2C510FFF7D4FF064600F00D
:10821000F3FF2C2000F098FF04F2F710FFF7CAFFDD
:10822000064600F0E9FF641E002C00DA3124AC425F
:1082300002D02C2000F088FFAC42D9D1FAF742FEE0
:1082400070BD0000D8000020DC00002070B5204880
:108250000078D0B100BFFEF72BF80446FAF712FF02
:10826000FEF726F80546FAF70DFFFEF721F8064659
:10827000FAF708FFAC42EED1B442ECD10CB10020C9
:1082800070BD002012490870FAE700BFFEF710F831
:1082900004460CB90020F3E7FAF7F4FEFEF708F8FD
:1082A0000546FAF7EFFEFEF703F80646FAF7EAFE90
:1082B000AC42EBD1B442E9D10548047034B14FF47B
:1082C0001670044908600120034908602046D7E77A
:1082D000A4000020F0010020B001002070B5044689
:1082E0000D464FF480411848FDF71FFB24B980214B
:1082F0001648FDF718FB03E080211448FDF715FB35
:1083000025B140211248FDF710FB04E04FF4004175
:108310000D48FDF70AFB20210B48FDF706FB0B4833
:10832000FDF7F0FA0646360A20210748FDF7FBFA6A
:1083300040210748FDF7F7FA4FF400410248FDF7E6
:10834000F2FA304670BD0000000C014000180140F8
:10835000000801402DE9F04706460027B500C5F3A7
:108360000749ADB24FF0030800BF00242946484634
:1083700005F094FAF0B105F063F9A12101EB490190
:10838000C8B205F00DFB0746A7B104F0F5FE0446A0
:1083900004F01AFF04F0F0FE00EB042404F014FFD4
:1083A00004F0EAFE00EB042404F00EFF04F0E4FE07
:1083B00000EB042405F054F927B9A8F1010000F0FE
:1083C000FF0801E04FF00008B8F1000FCDDC2046B7
:1083D000BDE8F08710B51848006820B1012807D023
:1083E000022817D109E01448006804F095FB15E055
:1083F0001148006804F090FB10E010490E4A126822
:1084000031F81200FDF774FB0D490B4A126841F870
:10841000220003E000200849086000BF00BF0648B2
:108420000068401C0449086008460068022801DD15
:108430000020086010BD0000B8000020040C0020DF
:10844000780A0020F0B502460B4600240FE01749D9
:1084500001EB021516490E680968491C144F396072
:10846000A85DF9F777F904EB840100EB41040F48AC
:1084700000EB02100E490968405C984213D00B488B
:1084800000EB02100A490968405C30280BDB074802
:1084900000EB021006490968405C392803DC0448F7
:1084A00000681328D3DB2046F0BD0000D41D002057
:1084B000EC00002070B505460E46002404E0FF20C5
:1084C00000F092FF2855641CB442F8D3012070BD1F
:1084D00010B580210148FDF726FA10BD00140140B7
:1084E00010B580210148FDF720FA10BD00140140AD
:1084F00010B580210348FDF718FA80210148FDF7E7
:1085000012FA10BD0010014010B510210148FDF70E
:108510000AFA10BD0014014010B510210148FDF702
:1085200004FA10BD0014014010B54FF40061024878
:10853000FDF7F9F910BD0000000C014010B54FF433
:1085400000610248FDF7F1F910BD0000000C014088
:1085500010B540210148FDF7E6F910BD00100140BB
:1085600010B540210148FDF7E0F910BD00100140B1
:1085700010B54FF480710248FDF7D5F910BD000029
:108580000010014010B54FF480710248FDF7CDF99D
:1085900010BD00000010014010B54FF4006102480A
:1085A000FDF7C1F910BD00000014014010B54FF4F3
:1085B00000610248FDF7B9F910BD00000014014048
:1085C00010B54FF400710248FDF7ADF910BD000081
:1085D0000010014010B54FF400710248FDF7A5F9F5
:1085E00010BD00000010014010B54FF4806102483A
:1085F000FDF799F910BD00000014014010B54FF4CB
:1086000080610248FDF791F910BD0000001401409F
:1086100010B54FF400610248FDF785F910BD000068
:108620000008014010B54FF400610248FDF77DF9E4
:1086300010BD00000008014010B54FF40051024881
:10864000FDF771F910BD0000000C014010B54FF4AA
:1086500000510248FDF769F910BD0000000C01400F
:1086600010B54FF480510248FDF75DF910BD0000D0
:108670000008014010B54FF480510248FDF755F94C
:1086800010BD00000008014010B54FF480510248B1
:10869000FDF749F910BD0000000C014010B54FF482
:1086A00080510248FDF741F910BD0000000C014067
:1086B000F0B507460C461646B44201D12046F0BD3F
:1086C000A01900EBD0714D1005EB4500084901EBF6
:1086D00080004068B84205DD3246691C3846FFF725
:1086E000E7FFECE72A4621463846FFF7E1FFE6E7D9
:1086F00094FE010870B502460020002317E000EB4D
:108700004004304D55F82440944206D100EB40041B
:1087100005EB840464688C4206D000EB4004294DCC
:1087200005EB8404A4680CB9012300E0401C19285F
:1087300001DA002BE3D0E3B300EB4004214D05EB5D
:108740008404A468022C3BD123E0441C04EB4404C1
:108750001C4D55F8244000EB40051A4E46F82540C4
:10876000441C04EB4404354605EB8404646800EBC8
:10877000400506EB85056C60441C04EB440435465B
:1087800005EB8404A46800EB400506EB8505AC60AE
:10879000401C1828D9DB002400EB4005094E46F8A0
:1087A000254000EB400506EB85056C6000EB4005BD
:1087B00000E005E006EB8505AC600124024D2C705D
:1087C00070BD0000D80A002037010020002010E012
:1087D000002100EB4002084B03EB8202916000EBAA
:1087E000400243F8221000EB400203EB820251608A
:1087F000401C1928ECDB7047D80A00200021074AEA
:108800001170002004E00021054A1154411CC8B237
:108810000828F8DB0021034A117070473501002059
:108820003901002038010020002008E00021054A1D
:1088300042F82010044A1160044A1160401C1428B8
:10884000F4DB7047AC0C0020C0000020C400002006
:1088500070B50E480068FCF7FBFD04460B48006845
:10886000FCF7D8FD054601222946204601F052FDBD
:1088700006490968491C054A08461160FDF7F8FCDD
:1088800010B100200149086070BD000020000020E8
:1088900070B539A13948F7F746FE394908600846EE
:1088A0000068002867D04FF480613648FDF73DF836
:1088B00001203549087000F0D3FE03220421084648
:1088C00000F0EAFE05220621042000F0E5FE2AE081
:1088D000002400252D48005D2A2822D008E02B48DE
:1088E000005D05EB850100EB4100A0F13005641C43
:1088F0002648005D3D28F2D1641C002608E023488C
:10890000005D06EB860100EB4100A0F13006641C1F
:108910001E48005D0A28F2D100223146284601F0A7
:10892000F9FCFDF70FF916481E2102681748F7F702
:1089300085FD0028CCD1FDF705F911480068F7F74F
:1089400019FEFDF7FFF812490C4803F097FAFDF7FE
:10895000F9F841F288300F49086001E0FDF7F2F8BC
:108960000C4800680028F9D107490870FDF744FD5C
:1089700001200949087070BD7200000070400308B2
:1089800074020020000C0140D0000020A849002003
:1089900085400308180000203701002070B5E5E08D
:1089A00000F0ACFB044674480078062870D2DFE87B
:1089B00000F00314384C70B3012C0DD1C8206F495E
:1089C000086001206C49087000206D4908606D49FD
:1089D0000860204600F0DEFBC7E0204600F0DAFB2E
:1089E0002C2C16D101266520FFF7E4FB06466548CE
:1089F0000068B04202D06348006818B902205E499E
:108A0000087002E000205C49087000205E490860A0
:108A100006E021465B480068F8F786FE5949086081
:108A2000A3E0204600F0B6FB2C2C06D103205249CF
:108A3000087000205549086006E021465248006849
:108A4000F8F772FE504908608FE0204600F0A2FB64
:108A5000022C15D104204849087000204C490860B8
:108A60004C490860002508E000214B48484A12683C
:108A700000EB02104155681CC5B2102DF4DB06E076
:108A8000214642480068F8F74FFE404908606CE014
:108A900067E0204600F07EFB032C06D10520364916
:108AA000087000203D49086035E02C2C20D1384862
:108AB0000068401C3649086008460068642803DBEB
:108AC00008460068401E0860002032490860002502
:108AD00008E0002030492E4A126801EB0211485587
:108AE000681CC5B2102DF4DBC8202449086012E0D0
:108AF00029482749096800EB0110264909684454B0
:108B000024480068401C2349086008460068122871
:108B100001DD1220086028E0042C13D11F480068F2
:108B200017490968884209D14FF416701C4908603A
:108B300000F038F800201049087011E000200E49BC
:108B400008700DE0154800680001144908602046CF
:108B5000F9F7E0FD1149098889B208430F49086017
:108B600003E000200449087000BF00BF00F0DEFAF7
:108B700000287FF415AF70BD03010020F400002031
:108B8000F8000020D8000020DC000020E0000020D9
:108B9000E4000020E8000020D41D0020FC0000209C
:108BA000F00000202DE9F047FC4800680E2878D03E
:108BB00009DC0C2849D2DFE800F048174849788BD7
:108BC000CC484848FEFD65286CD006DC0F286AD0EA
:108BD000102869D0642838D1B2E1662876D0672899
:108BE00075D06828F7D129E20222ED480168ED48E6
:108BF0000068FAF747F9002400BF0020EA4908603E
:108C000000212046FFF71EFC80464046FCF746FC4C
:108C1000002806DB4046FCF7E3FE054600F0ECFAD0
:108C200005E02D2000F090FA312000F08DFADF48A9
:108C30000068844202DA2C2000F086FA641CDB48CB
:108C400000688442D9DDFAF73DF916E20222D448E1
:108C50000168D4480068FAF715F9D5480078D54975
:108C60000978884206D12D2000F06EFA312000F0FC
:108C70006BFA13E0CF4805780CE0681CC5B2142DE0
:108C800000DB0025CC4951F8250000F0B5FA2C2076
:108C900000F05AFAC6480078A842EED1FAF712F965
:108CA000EBE109E196E134E146E1C1480078C149D0
:108CB00008700222BA480168BA480068FAF7E2F878
:108CC000302000F041FAFAF7FDF8D6E192E195E1A3
:108CD00000250222B2480168B2480068FAF7D2F8CB
:108CE000B648007830B92D2000F02EFA312000F07F
:108CF0002BFA1BE016E0B24951F8350000F07CFA7F
:108D00002C2000F021FAAE4901EBC501486800F0C3
:108D100073FA681CC5B2A9480078854202DA2C2093
:108D200000F012FAA54800788542E4DBFAF7CAF8A9
:108D3000002508E00020A24941F8350001EBC501FB
:108D40004860681CC5B2782DF4DB00209B49087090
:108D500093E1002502229248016892480068FAF7E0
:108D600091F89848007830B92D2000F0EDF93120C5
:108D700000F0EAF91BE016E0934951F8350000F0E5
:108D80003BFA2C2000F0E0F98F4901EBC50148685F
:108D900000F032FA681CC5B28A480078854202DACF
:108DA0002C2000F0D1F9874800788542E4DBFAF7FF
:108DB00089F801E07FE010E0002508E0002082490A
:108DC00041F8350001EBC5014860681CC5B2782D3B
:108DD000F4DB00207B4908704FE10024A1467B486A
:108DE0000078002854D100BF002600206E4908609A
:108DF0003D212046FFF726FB80466B480068401C5B
:108E0000694908604046FCF749FB002839DB4046C9
:108E1000FCF744FB40B900212046FFF713FB064650
:108E2000304600F08FFB2EE04046FCF737FB1B2856
:108E300029D000212046FFF705FB06464046FCF7F7
:108E40002DFB0546FDF7FAF9E8B14046FCF726FB95
:108E50000546FCF7F3FAB04202DD49F0020912E0E0
:108E60004046FCF71BFB0546FCF7DEFAB04202DA8F
:108E700049F0040907E000223146404601F04AFA71
:108E800001E049F00109641C484800688442ABDDF8
:108E90004348006870B114224148016841480068A5
:108EA000F9F7F0FF4949097809EBC10000F0A4F98E
:108EB000FAF708F8E1E0E0E00024002717E00020DE
:108EC0003949086000212046FFF7BCFA404941F8C3
:108ED0003700641C00203449086000212046FFF759
:108EE000B1FA3B4901EBC7014860641C7F1C2F4865
:108EF00000688442E3DB09E00020354941F837008F
:108F0000002238467F1C01EBC0004260192FF3DBC2
:108F1000B3E000202449086000210846FFF792FAD8
:108F200080464046FCF75CFD012804D10122022165
:108F3000404601F0EFF9A0E000201B4908609CE0EA
:108F400000201949086000210846FFF77BFA804697
:108F500000201549086000210120FFF773FA06463A
:108F6000FA2E00DDFA2602220D4801680D4800683D
:108F7000F9F788FFC24600250AE01AF8010B00F055
:108F80003BF9701EA84202DD2C2000F0DDF86D1CBC
:108F9000B542F2DBF9F796FF6FE00000E000002039
:108FA000D8000020DC000020EC000020E4000020BD
:108FB0002500002024000020A8020020010100203C
:108FC000F802002002010020B80600200401002061
:108FD000FC0C002000202A49086000210846FFF709
:108FE00031FA284908600846006810B10120264976
:108FF000087042E00020244908703EE0002020492B
:10900000086000210846FFF71DFA18B1A0F2E7300A
:1090100090B902E0FFF7D4F80EE0F8F7CBFC02229B
:109020001A4801681A480068F9F72CFF002000F080
:10903000E3F8F9F747FF00BF00BF1EE00222134824
:10904000016813480068F9F71DFF122000F0D4F8FA
:109050002C2000F079F86420FFF7ACF8054600F00A
:10906000CBF82C2000F070F86520FFF7A3F8054638
:1090700000F0C2F8F9F726FF00BF00BFBDE8F08797
:10908000EC000020CC000020D0000020D800002000
:10909000DC00002010B5002011490860114908606B
:1090A0001149086011490860114908704FF41640D1
:1090B0001049086000208880C880088188810C20C1
:1090C00048810D4800F068FF012240F225510A480E
:1090D00000F049FF0121084800F01CFF10BD00000E
:1090E0000C010020080100201401002010010020C4
:1090F00003010020C40D00200044004000BF0848C8
:109100000068084A12689042F9D005480068401C7F
:10911000C0F30A01024801600348405C7047000048
:109120000C01002008010020D40D00200448006834
:1091300004490968884201D0012070470020FCE7FB
:10914000080100200C01002070B505460D4800689C
:10915000401CC0F30A0400BF0B4800688442FBD0E7
:109160000A48055507480460284600F013F8012214
:1091700040F22771064800F0F6FE0121044800F095
:10918000C9FE70BD1001002014010020D41500207C
:109190000044004007490988C1F307214140064ABD
:1091A00032F82110034A127881EA022189B2014A79
:1091B00011607047F80000207808020810B50446D6
:1091C00004F13000C4B2392C01DDE01DC4B22046E8
:1091D000FFF7BAFF10BD000010B50446002C02DDF9
:1091E0000120044908700348007810B12046FFF7B9
:1091F000E5FF10BD0001002070B5044600203E4987
:109200000870002C00DA00243C4894FBF0F00A219E
:1092100090FBF1F201FB1200C5B22846FFF7DCFF1C
:10922000374894FBF0F00A2190FBF1F201FB1200A9
:10923000C5B22846FFF7D0FF324894FBF0F00A2170
:1092400090FBF1F201FB1200C5B22846FFF7C4FF04
:109250002D4894FBF0F00A2190FBF1F201FB120083
:10926000C5B22846FFF7B8FF284894FBF0F00A2162
:1092700090FBF1F201FB1200C5B22846FFF7ACFFEC
:1092800042F2107094FBF0F00A2190FBF1F201FB26
:109290001200C5B22846FFF79FFF4FF47A7094FB87
:1092A000F0F00A2190FBF1F201FB1200C5B2284652
:1092B000FFF792FF642094FBF0F00A2190FBF1F29B
:1092C00001FB1200C5B22846FFF786FF0A2094FB77
:1092D000F0F00A2190FBF1F201FB1200C5B2284622
:1092E000FFF77AFF0A2094FBF0F100FB1140C5B2B2
:1092F0002846FFF763FF70BD0001002000CA9A3BBB
:1093000000E1F5058096980040420F00A08601001C
:1093100010B50446C4F30330FFF750FFC4F3032035
:10932000FFF74CFFC4F30310FFF748FF04F00F00F2
:10933000FFF744FF10BD000010B540210248FCF7C4
:10934000F4FA02F071F810BD000C014010B5402194
:109350000248FCF7E8FA02F067F810BD000C014083
:1093600010B580210748FCF7E0FA80200649088004
:10937000032088700420C8700248FCF751FA02F0FC
:1093800053F810BD000C01402401002010B58020CE
:1093900007490880032088701420C8700548FCF72E
:1093A0003FFA80210348FCF7BEFA02F03DF810BDF9
:1093B00024010020000C014070477047704770473F
:1093C000704710B50446204600F00EF810BD70B589
:1093D00005460E46002403E0285D00F005F8641CF5
:1093E000B442F9D3012070BD2DE9F04105462E4667
:1093F0000024002725E006F0800028B94FF48051B2
:109400001248FCF790FA04E04FF480510F48FCF743
:109410008CFA7006060E4FF480610C48FCF785FA52
:109420006006040E4FF400610848FCF76EFA08B1BC
:1094300044F001044FF480610448FCF774FA781C8E
:10944000C7B2082FD7DB2046BDE8F08100100140ED
:10945000014609B1102001E04FF48010014A10606C
:10946000012070471008014070B50246002000231B
:1094700017E000EB40042F4D55F82440944206D1EC
:1094800000EB400405EB840464688C4206D000EBDA
:109490004004284D05EB8404A4680CB9012300E0C6
:1094A000401C192801DA002BE3D00BB300EB400479
:1094B000204D05EB8404A468022C1AD11E4C2468AC
:1094C000B4B900EB400445F8242000EB400405EB60
:1094D00084046160012400EB4005164E06EB85050F
:1094E000AC60164C2468112C22D10124144D2C7030
:1094F0001EE000EB40040F4D05EB8404A468012C32
:1095000016D000EB400445F8242000EB400405EBA6
:1095100084046160012400EB4005064E06EB8505DE
:10952000AC60064C2468112C02D10124044D2C702F
:1095300070BD0000D80A0020A00000209801002083
:109540003701002010B50446FEF7F2FCFEF71EFEC0
:10955000C4EB04118800FEF7F9FDFEF717FE4AF28E
:10956000A5510420F8F706F9FEF756FD3C21B0FBA3
:10957000F1F00149086010BD3000002070B50446CC
:109580000D4600F030FE04F03F0000F14002A11152
:10959000002000F01DFF00F026FE05F1B802A11129
:1095A000002000F015FF00F01EFEC022002108463A
:1095B00000F00EFFC0220121002000F009FF70BD65
:1095C00070B50025202600216C20FCF79BFA21486D
:1095D000006800283DD14FF496701E4908600024B1
:1095E0001CE004EB44001C4901EB8000406898B18A
:1095F00004EB440001EB80008068022802D1012DB9
:1096000000DA012504EB4400134901EB8000806877
:10961000012802D1022500E01924641C192CE0DB8A
:10962000012D02D0022D0ED101E096260BE00B4851
:10963000007820B9962601200849087002E0002031
:109640000649087000BF00BF012231461046FEF7F0
:10965000BBF970BD90010020D80A0020BC01002099
:1096600010B5FCF7C9FEFCF70BFF00200449087099
:1096700004490870012204A1104600F09BFF10BDB0
:109680002D0100202E0100202020204452414D4D6C
:10969000202020200000000070B504460D4616462C
:1096A00005490D7005490C7006F1AC010022104609
:1096B00000F02CFF70BD00002E0100202D010020C5
:1096C0002DE9F0412148006800283CD14FF4AF70EB
:1096D0001E4908601E48007818B901201C4908700E
:1096E00002E000201A4908704FF4BD70FEF762FDD9
:1096F0000446012C01DA3C2604E03C2090FBF4F007
:10970000801EC6B200251CE012480068401EA84218
:1097100004D10F48007808B9E32700E0DF27C5EB44
:109720000510C00090FBF4F000EB0608072140464E
:10973000FCF7E8F9002239461046FEF745F9681CA7
:10974000C5B2A542E0DBBDE8F08100003001002099
:10975000BE0100203800002070B5FCF791FE00200B
:109760004249087042490870012242A1104600F0A7
:1097700021FF10203D49087004203D490870002257
:1097800040A1104600F016FF06203949087022203B
:10979000364908706420FEF70DFD0446002256216C
:1097A0001046FEF711F93B4894FBF0F03030C5B29B
:1097B000002229461046FEF707F942F2107094FB8A
:1097C000F0F00A2190FBF1F201FB12003030C5B23B
:1097D000002229461046FEF7F7F800222E211046F7
:1097E000FEF7F2F84FF47A7094FBF0F00A2190FB48
:1097F000F1F201FB12003030C5B2002229461046BA
:10980000FEF7E2F8642094FBF0F00A2190FBF1F2FD
:1098100001FB12003030C5B2002229461046FEF787
:10982000D3F800222E211046FEF7CEF80A2094FB32
:10983000F0F00A2190FBF1F201FB12003030C5B2CA
:10984000002229461046FEF7BFF80A2094FBF0F1EB
:1098500000FB11403030C5B2002229461046FEF709
:10986000B3F842F210700C49086070BD2D01002061
:109870002E0100202020204452414D4D2020202048
:10988000000000002020204D6973742D54696D651F
:1098900020202000A08601001400002070B504469E
:1098A00000256720FEF786FC06283FD2DFE800F09F
:1098B000030C16202A3404EB44011E4A52F83100EE
:1098C000F6F77EFE054631E004EB4401194A02EB4F
:1098D000C1014868F6F774FE054627E004EB440131
:1098E000144A02EBC1018868F6F76AFE05461DE0DE
:1098F00004EB44010F4A02EBC101C868F6F760FEB1
:10990000054613E004EB44010A4A02EBC101086971
:10991000F6F756FE054609E004EB4401054A02EB62
:10992000C1014869F6F74CFE054600BF00BF284656
:1099300070BD0000F839020810B500F035F810BD10
:109940004FF0E021012804D0801C06D0002088615F
:109950007047086940F0010002E0086920F001004A
:10996000086170474FF0E0210028086902D040F0FC
:10997000020001E020F002000861704710B541F6D6
:109980006A0000F00DF80120FFF7ECFF0120FFF75F
:10999000D7FF14200149086010BD0000140000200A
:1099A0004FF0E0214861704710B54E48006820B183
:1099B0004C480068401E4B4908604B48006828B17D
:1099C00049480068401E4849086003E04FF47A7037
:1099D000454908604548007870B143480068C8218F
:1099E00090FBF1F201FB1200642805DD4FF4807159
:1099F0003F48FBF79AFF04E04FF480713C48FBF7C7
:109A000092FF3C48006820B13A480068401E39493E
:109A100008603948006820B137480068401E364960
:109A200008603648006820B134480068401E334959
:109A300008603348006820B131480068401E304952
:109A400008603048006820B12E480068401E2D494B
:109A500008602D48007820B12B480078401E2A4924
:109A600008702A48007820B128480078401E27490D
:109A700008702748007820B125480078401E244906
:109A800008702448007820B122480078401E2149FF
:109A900008702148006828B11F480068401E1E4910
:109AA000086002E000201D4908701D48006828B1C8
:109AB0001B480068401E1A49086002E0002019494E
:109AC00008701948006820B117480068401E164900
:109AD00008601648006820B114480068401E134909
:109AE000086010BD1801002014000020D0000020E4
:109AF0000008014018000020640200206C020020D1
:109B000070020020680200200200002003000020F4
:109B10000400002005000020F400002003010020C4
:109B2000580200201A02002030010020900100207D
:109B3000704770477047704770477047704770476D
:109B40007047704770477047704770477047000014
:109B50002DE9F0419448007808B1FDF74BF800205A
:109B60009149087000212820FBF7CCFF0123002237
:109B70008E4801681846FDF7E7FB4FF4C170FEF709
:109B800019FB40B303210420FBF7BCFF00221D2179
:109B9000104600F0BBFC86480068FBF722FC8046BC
:109BA00000231A4641461846FDF7FEFC40F27B10A2
:109BB000FEF700FB28B900221146104600F0A6FC73
:109BC00004E000220F21104600F0A0FC002220211A
:109BD0001046FDF7F9FE04210846FBF793FF754890
:109BE0000068002870D00022B221104600F08EFCE0
:109BF000704800680B284DD2DFE800F04C060D14C9
:109C00001B222930373E4500002240F287111046C2
:109C1000FDF77BF83EE000224FF4C4711046FDF7DB
:109C200074F837E0002240F289111046FDF76DF814
:109C300030E000224FF4C5711046FDF766F829E0C8
:109C4000002240F28B111046FDF75FF822E000225F
:109C50004FF4C6711046FDF758F81BE0002240F2A1
:109C60008D111046FDF751F814E000224FF4C77132
:109C70001046FDF74AF80DE0002240F28F11104621
:109C8000FDF743F806E000224FF4C8711046FDF7D7
:109C90003CF800BF00BF002220211046FDF794FED3
:109CA00044490968491E01EBC10101EB410101F181
:109CB0006C00FEF77FFA012807D002280BD003289A
:109CC0000FD0042819D112E018E00022B421104668
:109CD00000F01CFC11E00022B521104600F016FC3B
:109CE0000BE00022B621104600F010FC05E0002237
:109CF000B721104600F00AFC00BF0DE02E480068B6
:109D000028B10022B821104600F000FC04E0002237
:109D1000B921104600F0FAFB04E000222021104691
:109D2000FDF752FE254800787828F6DD4FF4BD7027
:109D3000FEF740FA0446092C01DD092600E0E6B2F0
:109D4000012C01DA3C2704E03C2090FBF4F0401E9B
:109D5000C7B2002513E0C5EB0510C00090FBF4F07E
:109D600000EB070806214046FBF7CCFE05F1310069
:109D7000C1B200221046FDF727FE681CC5B2B542ED
:109D8000E9DB0A2C0DD106216E20FBF7BBFE002279
:109D900031211046FDF718FE002230211046FDF754
:109DA00013FEBDE8F08100003701002030000020E4
:109DB0003400002038000020880000202D01002001
:109DC000704770477047000070B540F227711E4819
:109DD00000F0AAF8C8B11D4800681D49096888420A
:109DE0000CD01B480068401CC0F30A041948015DF0
:109DF000154800F01BF91648046005E0002240F207
:109E00002771114800F0AFF800BF40F225510E480D
:109E100000F08AF8B8B10C4800F004F9C5B20E4859
:109E20000068401CC0F30A040B4804600B4800683B
:109E3000844202D101200A4908700A48055564206D
:109E40000949086000BF70BD0044004010010020B7
:109E500014010020D4150020080100200C0100206E
:109E600004010020D40D0020F400002070B540F261
:109E700027711F4800F058F8C8B11E4800681E49F5
:109E8000096888420CD01C480068401C00F01F0480
:109E90001A48015D164800F0C9F81748046005E04B
:109EA000002240F22771124800F05DF800BF40F236
:109EB00025510F4800F038F8C0B10D4800F0B2F855
:109EC000C5B20F480068401CC0F308040C48046089
:109ED0000C480068844202D101200B4908700B48ED
:109EE00005554FF47A700A49086000BF70BD000044
:109EF000004800401002002014020020602F0020C3
:109F0000080200200C0200201B020020602D00200F
:109F1000580200200029818902D041F4005101E05B
:109F200021F400518181704770B501F01F060122B4
:109F30000025C1F3421302FA06F4012B0FD0022BC5
:109F40000FD0838A4FEA11210088234202FA01F2DE
:109F500000EA020001D000B10125284670BD8389C6
:109F6000F0E7038AEEE710B5C1F3421301F01F04D6
:109F70000121A140012B07D0022B07D01430002A69
:109F8000026805D00A4304E00C30F8E71030F6E729
:109F90008A43026010BD000030B50446008A85B0D7
:109FA0000D464CF6FF710840E98801432182A189E2
:109FB0004EF6F3100140A8882A8910436A890A43A3
:109FC0001043A081A08A4FF6FF410840A9890143B0
:109FD000A1826846FDF7ACFE1148844201D1039886
:109FE00000E00298642200EBC00101EB0010296838
:109FF0006FF018058900B0FBF1F0B0FBF2F1090138
:10A000000B096B4300EB8300322303EB0010B0FB22
:10A01000F2F000F00F000843208105B030BD0000D1
:10A02000003801408088C0F308007047C1F3080180
:10A03000818070477047704770470120704700006B
:10A040002D2802D08D2842D12EE02249096804290A
:10A0500014DA20490968491C1E4A11601E49096822
:10A06000126811441D4A02EB01110968491CD1B95B
:10A0700018490968491E174A116014E01649096811
:10A08000491C154A116011460968124A12681144A8
:10A09000124A02EB01110968491C21B90E490968ED
:10A0A000491E0D4A116012E00A49096829B109499F
:10A0B0000968491E074A116008E007490968002934
:10A0C00004DD05490968491E034A116000BF00BF4D
:10A0D000704700002801002084010020302A002061
:10A0E0004FF6FF72904216D042F21072904212DB8D
:10A0F000520090420FDA084A1278521CD1B2142949
:10A1000000DB0021054A1278914204D0044A42F84B
:10A110002100014A11707047250000202400002012
:10A12000A802002000BFFEE770B502460020002311
:10A1300017E000EB4004174D55F82440944206D137
:10A1400000EB400405EB840464688C4206D000EB0D
:10A150004004104D05EB8404A4680CB9012300E011
:10A16000401C192801DA002BE3D093B100EB400426
:10A17000084D05EB8404A468012C0AD1022400EBED
:10A180004005044E06EB8505AC604FF49674024D15
:10A190002C6070BDD80A0020A000002010B50D4A28
:10A1A00012680D4B1B681A4402EB42020B4B03EB87
:10A1B00082025168074A1268074B1B681A4402EB77
:10A1C0004202064B53F82200FFF7AEFF012004497C
:10A1D000087010BDD001002028010020D80A0020FE
:10A1E00037010020704770B500BF00210846FEF718
:10A1F00075F8C5B201210020FEF770F8C4B2802DB9
:10A2000002D00DB1FCF73CF9802C02D00CB1FCF768
:10A2100037F905F080000028E7D104F0800000281D
:10A22000E3D170BD10B515E0FBF78CFC0D4800685C
:10A23000C82190FBF1F201FB1200642805DA4FF40B
:10A2400080610948FBF771FB04E04FF48061064828
:10A25000FBF769FB0348006818B1FDF7F7FF00281A
:10A26000E2D010BD14000020000C01402DE9F041A7
:10A2700007460D4690461C46069E01201A49087066
:10A28000E2B220210020FDF79FFB04201649087050
:10A29000E2B220210020FDF797FB012D02D0022D14
:10A2A0000CD105E0E2B2BA21002000F02FF905E060
:10A2B000E2B2BB21002000F029F900BF00BF04E09A
:10A2C000E2B220210020FDF77FFB074800787828C4
:10A2D000F6DB772004490870E2B220210020FDF768
:10A2E00073FBBDE8F08100002D01002070B505462C
:10A2F0000C462846FDF75EFFA04209D029462046BD
:10A3000000F0C0F82846FBF7ADF80646FFF7E8FE78
:10A3100070BD00002DE9F04105460C461646154873
:10A32000854225DA2846FBF7B9F80746FBF77AFF9E
:10A33000A0B12846FBF73EFB0746FDF73BFFA042D6
:10A3400016D02846FBF736FB07463946204600F074
:10A3500099F86EB12846FFF7C3FE09E02846FBF7DF
:10A360009DF8C0EBC000044901EB80004068046028
:10A37000BDE8F08178D403003CDC01082DE9F04110
:10A3800005460F4616464FF4C970FDF713FF044605
:10A39000002C01DB322C00DD002404F2931029464E
:10A3A000FFF7A4FF04F2C5103946FFF79FFF04F240
:10A3B000F7103146FFF79AFF641C322C00DB0024B3
:10A3C00021464FF4C970FFF791FFBDE8F08100000E
:10A3D000F8B505460E4617464FF480412648FBF770
:10A3E000A2FA25B980212548FBF79DFA03E08021D8
:10A3F0002248FBF79AFA26B140212148FBF795FA4B
:10A4000004E04FF400411C48FBF78FFA20211A4862
:10A41000FBF78BFA4FF47F40ADF8000010208DF869
:10A42000030003208DF8020069461448FBF7F8F991
:10A430001248FBF767FA0446E4B244EA0724A1B2E3
:10A440000E48FBF774FA20210B48FBF76CFA402109
:10A450000B48FBF768FA4FF400410748FBF763FA33
:10A460004FF47F40ADF8000028208DF803006946C6
:10A470000248FBF7D5F9F8BD000C01400018014077
:10A48000000801402DE9F047074688464FEA880654
:10A49000C6F3074AB6B23D464FF0030903F0BCF9D4
:10A4A00000BF00243146504603F0F8F9A0B1280E51
:10A4B00003F076FA044624B1C5F3074003F070FABE
:10A4C000044624B1C5F3072003F06AFA04461CB120
:10A4D000E8B203F065FA044603F0C2F824B9A9F122
:10A4E000010000F0FF0901E04FF00009B9F1000F91
:10A4F000D7DC03F087F904480068401C0249086073
:10A500002046BDE8F08700001C01002070B505461C
:10A510000C4616466720FDF74DFE062845D2DFE8BB
:10A5200000F0030D18232E3904EB4400204A52F8A2
:10A5300030103246284600F03DF836E004EB440087
:10A540001B4A02EBC00032464168284600F032F850
:10A550002BE004EB4400164A02EBC000324681684F
:10A56000284600F027F820E004EB4400104A02EBF4
:10A57000C0003246C168284600F01CF815E004EB24
:10A5800044000B4A02EBC00032460169284600F045
:10A5900011F80AE004EB4400054A02EBC000324621
:10A5A0004169284600F006F800BF00BF70BD0000FA
:10A5B000F83902082DE9F04106460C46174666E0D8
:10A5C000207823285DD1641C2078A0F13005641C1C
:10A5D000207805EB850100EB4100A0F13005641CFB
:10A5E0000B2D4DD2DFE805F04C060D141B2229304F
:10A5F000373E45003A4640F287113046FCF785FB6E
:10A600003EE03A464FF4C4713046FCF77EFB37E03B
:10A610003A4640F289113046FCF777FB30E03A4683
:10A620004FF4C5713046FCF770FB29E03A4640F222
:10A630008B113046FCF769FB22E03A464FF4C671B5
:10A640003046FCF762FB1BE03A4640F28D11304683
:10A65000FCF75BFB14E03A464FF4C7713046FCF759
:10A6600054FB0DE03A4640F28F113046FCF74DFBAB
:10A6700006E03A464FF4C8713046FCF746FB00BF8F
:10A6800005E014F8011B3A463046FDF79DF92078A5
:10A69000002895D1BDE8F0812DE9F04107460C4630
:10A6A00015461E461148007838B104F13000C1B299
:10A6B00032463846FDF788F916E07CB101200B4997
:10A6C000087032462D213846FDF77EF904F130003E
:10A6D000C1B232463846FDF777F905E025B132467A
:10A6E00020210020FDF770F9BDE8F0812C01002049
:10A6F00070B504461148AFF30080114904EBC40063
:10A7000001EB8004002620884FF0FF3581070029E7
:10A7100006D00ADA8006204604D501F072F903E07B
:10A720002C4604E000F0ECFE30B126800024034803
:10A73000AFF30080204670BD2680F1E700000000E6
:10A740001424002010B504460C48AFF300800C49D7
:10A7500004EBC40001EB80042088810703D080064D
:10A7600003D5A46805E0002403E0204600F0C1FE04
:10A7700064680248AFF30080204610BD000000006E
:10A78000142400202DE9F84306460F466648AFF32F
:10A790000080684601F048FC04004FF0FF3575D09A
:10A7A0000146304601F08EFC814620690028F6D033
:10A7B00017F00C0004D004280AD0082866D103E062
:10A7C000208840F0010006E0208840F0040020804E
:10A7D000208840F00200208017F0060F04D0484681
:10A7E00001F010FC002851D12088DFF8408180065C
:10A7F0004FF000064BD52146484600F015FF0128D2
:10A8000003D02088C00772D133E000214848C446F5
:10A810001BE000BFB0F800805FEA887213D00269C5
:10A8200023699A420FD1A0420DD0C28AE38A9A428C
:10A8300009D1026A236A9A4205D15FEA887270D40C
:10A84000228892076DD4491C2430BCF80020914224
:10A85000E0DB208810F0050F06D0B9075AD500BFFD
:10A8600040F00B00208055E02146484600F077FE7E
:10A87000E8B3208810F0060F04D02146484600F0C7
:10A8800043FEA0B3B80745D52088E9E743E0B80701
:10A8900041D42146484600F02AFE012803D02088F2
:10A8A000C0073ED130E000212148424617E000BFFA
:10A8B000B0F800C05FEA8C730FD003692769BB4210
:10A8C0000BD1A04209D0838AA78ABB4205D15FEA97
:10A8D0008C7326D423889B0723D4491C24301388E7
:10A8E0009942E5DB2088410705D5204600E018E0C5
:10A8F00000F0FFFD0EE0C00702D0E069206209E031
:10A90000204600F0F0FD60B1A6822146484600F0E6
:10A91000E8FD30B1009D0448AFF300802846BDE853
:10A92000F8832680F7E7000000000000A039020845
:10A93000142400202DE9F04107460E461546134821
:10A94000AFF3008045F00044CEB1114907EBC700DA
:10A9500001EB800001888A0711D001F00F02022A62
:10A9600006D089062A46314605D500F06BFF04E083
:10A970004FF0FF3403E000F0BDFD00B12C1A034896
:10A98000AFF300802046BDE8F08100000000000029
:10A990001424002070B504460D460E48AFF3008025
:10A9A0000D4904EBC40001EB80004FF0FF34018837
:10A9B0008A070AD08906294602D500F0E5FF01E0A2
:10A9C00000F09CFD012800D100240248AFF3008074
:10A9D000204670BD00000000142400202DE9F04145
:10A9E00007460D4616461148AFF300804FF0FF347E
:10A9F000B5B10F4907EBC70001EB800001888A075A
:10AA00000ED001F00F02012A0AD0890632462946EB
:10AA100002D501F071F801E000F074FD00B10024EE
:10AA20000248AFF300802046BDE8F081000000003E
:10AA30001424002030380A2801D201207047002059
:10AA4000704710B50446B4F5004F01DD002010BD7D
:10AA50002046FFF74DFEFAE700BFFEE710B50446BB
:10AA6000B4F5004F01DD002010BD2046FFF76AFE5F
:10AA7000FAE70146B1F5004F01DD012070470020E3
:10AA8000FCE7000070B504460D460EA12046F5F720
:10AA900083FE10B948F2010070BD0CA12046F5F705
:10AAA0007BFE10B948F20200F6E70AA12046F5F74E
:10AAB00073FE10B948F20300EEE729462046FFF77F
:10AAC00061FEE9E7535444494E0000005354444F9B
:10AAD0005554000053544445525200002DE9F041B2
:10AAE00004460D4616461F46B4F5004F03DD4FF0F1
:10AAF000FF30BDE8F081324629462046FFF71AFFB5
:10AB0000F7E770B504460D46B4F5004F02DD4FF08F
:10AB1000FF3070BD29462046FFF73CFFF9E72DE9DD
:10AB2000F04104460D4616461F46B4F5004F03DDBE
:10AB30004FF0FF30BDE8F081324629462046FFF74E
:10AB40004DFFF7E7704700000021094A1268094BE2
:10AB50001B68D01800E0491C074A02EB011212687A
:10AB6000521C002AF7D1884200DB401A70470000CF
:10AB70008401002028010020302A00202DE9F84F10
:10AB800005464FF00009C86900900C460127C846E9
:10AB90004E46284600F0E9F8012808D12846F5F786
:10ABA0000FFD0C300D21B0FBF1F0401CC7B2206945
:10ABB000009901F052FB82460025206990F87B1035
:10ABC00019B1B5F5007F56D02AE0818FA94227D16F
:10ABD000016C009A0025914200D900916946009EBF
:10ABE00002F0CAFC002847D02069009901F04AFE13
:10ABF00088B1009601226946206900F048F80028D3
:10AC00003AD02069009900F043F9002834D04FF081
:10AC10000008009E34E02069009900F05BF982464C
:10AC20000AEB1511206902F031FB002824D02069BD
:10AC3000C16D05F00F0001EB4010007838B1FF281E
:10AC400005D0E52803D04FF000096D1CB5E7B9F138
:10AC5000000F02D1009E1FFA85F809F10101C9B267
:10AC60008946E5280AD0206990F87B0040B1C7F5F5
:10AC70000070A84204D20020BDE8F88FB942E4D1A8
:10AC80002169A1F87880206946670120F4E72DE961
:10AC9000F041154607460C460E6801F00DFB0028F2
:10ACA00018D0384601F059FA02463846216802F0B9
:10ACB00005FF00280ED035B131463846226802F033
:10ACC000FDFE002806D00021384600F005F80028D7
:10ACD00000D00120BDE8F08170B50446806C0D46BF
:10ACE000A8423ED094F85010012928D166697EB15F
:10ACF000216889060CD5617F022906D00022014611
:10AD00003046E36C01F027FA14E0218C4218F6E794
:10AD10006268E16CD36801229847002820D0607FE8
:10AD2000022809D16268218CA06CD3680844E16CC8
:10AD300001229847002813D0002084F8500085B1E4
:10AD400094F85100218C6268484328449368E16C70
:10AD500001229847012806D04FF0FF30A064002060
:10AD600070BD012070BDA564FBE72DE9F04100270F
:10AD70000446B8463D463E4625E002F025FD38B380
:10AD80002078202824D02E2814D0A0F16101192980
:10AD900002D92031192907D8B8F1000F03D088EA69
:10ADA0000001890614D480464FB13046761C022833
:10ADB0000ED806E067B9641C0026012703E0082DC1
:10ADC00006D26D1C641C20780028D6D10C2D02D32D
:10ADD0000120BDE8F0810020FBE7012302F0BCBAAE
:10ADE000F8B5C1690446009100293DD0206900F002
:10ADF00071F8074600252069818FA9420FD10025EF
:10AE0000694602F0B9FB00282FD02069009901F0B3
:10AE100039FD58BB2069009900F05CF8074607EB44
:10AE20001511206902F032FA00281ED0206905F0C1
:10AE30000F01C06D00EB411630782E2809D10CA10E
:10AE40003046F5F7A9FC68B10DA13046F5F7A4FC32
:10AE500040B1307850B1E52804D0F07A0F2803D003
:10AE6000000701D56D1CC6E70020F8BD0120F8BD24
:10AE70002E20202020202020202020100000000054
:10AE80002E2E202020202020202020100000000036
:10AE900070B5054600F01EF806464FF40071E86DE7
:10AEA000F5F730FC002406E03119284602F02AFDAF
:10AEB00000280AD0641CA87FA042F5D800212846AB
:10AEC00002F020FD002800D0012070BD10B5FBF776
:10AED00093FA10BD838E82691A44037F032B01D03D
:10AEE000C38E1A44807F891E00FB012070472DE924
:10AEF000F0410446007F0025012806D0022838D002
:10AF0000032857D00020BDE8F08102262CE031460E
:10AF1000204601F0B8F9804601462046FFF7DCFEE6
:10AF2000002867D006EB4600C0F34800B0F5FF7F6D
:10AF300004D8E16C084401F02DFC0CE0E06C08F151
:10AF4000010190F8FF712046FFF7C6FE88B3E06C60
:10AF5000007847EA0020F10701D0000901E0C0F3C2
:10AF60000B0000B96D1C761C206B801CB042CED843
:10AF700040E00221204601F086F9074601462046BE
:10AF8000FFF7AAFEA8B102260FE016F0FF0F05D1C9
:10AF90007F1C39462046FFF79FFE50B1E06CF1B2AE
:10AFA00030F8110000B96D1C761C206B801CB0427B
:10AFB000EBD81FE00221204601F065F90746014663
:10AFC0002046FFF789FEA8B102260FE0700605D1E2
:10AFD0007F1C39462046FFF77FFE58B1E06C06F033
:10AFE0007F0150F8210000B96D1C761C206B801C7D
:10AFF000B042EBD8284686E72DE9F04389B00E46EB
:10B00000904699460546FFF7B0FE88B301271B4CD2
:10B010001CE04246314604A8FFF7DFFE28B1A742F4
:10B0200014D9002009B0BDE8F083694604A800F0F7
:10B03000ACF90028F6D0684601F040FC02463146E3
:10B04000284600F01DF80028ECD007E03A467F1CA7
:10B0500004A9284601F0BEFA0128DAD04B46424640
:10B060003146684600F0B0F80028DBD00120D9E76F
:10B07000FFE76946284600F088F9E4E73E420F0002
:10B080002DE9F74F086982B00C46416F0091B0F886
:10B0900078504FF0000B0298F5F792FA814620693C
:10B0A000009901F0DAF88246D846464E7DE02069E4
:10B0B00090F87B1031B1B5F5007F1DD1002005B0AF
:10B0C000BDE8F08F818FA94216D1016C009A00254E
:10B0D000914200D9009101226946FFF7D8FD00286E
:10B0E000EDD020690099FFF7D3FE0028E7D0206952
:10B0F0000099FFF7EFFE82460AEB151101912069D6
:10B1000002F0C4F80028DAD0206905F00F010D2202
:10B11000C06DBBF1000F00EB411109F10C00B0FB59
:10B12000F2F0C0B2087001D0002200E040221043CB
:10B130000870049A4A73A1F81A800F2200F01F00C9
:10B14000CA72401E00EB800202EBC000029A4FF070
:10B15000010B131800204A1C1F5C4FB116F800C0E9
:10B1600001F80C70375C401C0D2807F80280F3D3FF
:10B17000002305E0375CCB55375CBB54FF23401CF4
:10B180000D28F7D3B9F10C0F02D9A9F10D0000E099
:10B1900000208146E843000706D101222069019979
:10B1A00002F034FD00288AD06D1CB9F1000F7FF445
:10B1B0007EAF2169009848672069A0F87850012087
:10B1C0007DE700004A4103082DE9FC5F06460D4675
:10B1D0009A46012A0DD0002081462869416F0091CE
:10B1E000B0F8787090F87B2042B1B7F5007F02D0BC
:10B1F00018E00120F0E70020BDE8FC9F828FBA42F2
:10B2000010D1026C00278A4200D9009201226946BF
:10B21000FFF73DFD0028EFD028690099FFF738FEC1
:10B220000028E9D02869009901F017F800EB171100
:10B230008B46286902F02AF80028DDD0286907F03B
:10B240000F01C06D00EB41140020315C2154401C03
:10B250000B28FAD35FEA0A004FF0000837D0064601
:10B26000C07AE07284F80C8084F80D80F089E08167
:10B27000308A208200F0DBFF014604F1120002F068
:10B28000C1F9B08AA08201F06DFA014604F11600FE
:10B2900002F0B8F9608A2083708B6083F069E06106
:10B2A000F0696860F069C5E9020806F11A0001F06A
:10B2B00071FA044606F1140001F06CFA04EB004048
:10B2C000E86101225946286902F0A0FC56E084F8A2
:10B2D0000C8084F80D8001F045FA014604F10E005F
:10B2E00002F090F900F0A3FF014604F1100002F013
:10B2F00089F9208A6082E189E1822083C4F81C8078
:10B30000C5F80C80C5F80480C5F80880B9F1000FB5
:10B310001ED01020E072009901912869006C8842CB
:10B3200000D90190002201A92869FFF7B0FC00288C
:10B330003FF462AF0198E861010C04F1140002F0DF
:10B3400061F9019881B204F11A0002F05BF907E09B
:10B350002020E072A4F81480A4F81A80C5F81C809C
:10B3600001225946286902F051FC0028E0D0B9F1C9
:10B37000000F05D028690199FFF78AFD0028D7D072
:10B38000EF8200982862012036E72DE9F04100277E
:10B3900004460D46384620212954401C0B28FBD377
:10B3A0000021295420786178A2782E2806D111B185
:10B3B0002E2902D002E0287031E0AAB100262078C0
:10B3C00068B32E2813D020280AD002F0F4F9A0F197
:10B3D0006101A855192902D820F02000A855761C33
:10B3E000641C082EEBD304E02870687017E0012776
:10B3F000641C0826207890B12E2813D020280BD06A
:10B4000057B102F0D8F9A0F16101A855192902D865
:10B4100020F02000A855761C641C0B2EEAD30120D6
:10B42000BDE8F0810127F7E70649096809B9052158
:10B4300001E04FF4FA61084600BF0100A0F10100ED
:10B44000FBD17047200100202DE9F8430546006933
:10B4500090F87A60416F0091B0F8784000F0FDFEFE
:10B4600007463AE0286990F87B1029B1B4F5007FCF
:10B4700015D10020BDE8F883818FA1420FD1016C66
:10B48000009A0024914200D90091694602F074F8B4
:10B490000028EFD028690099FFF71CFD074607EB4D
:10B4A00014118846286901F0F1FE0028E2D02869CD
:10B4B00004F00F01761EC06DF6B200EB4110E521DD
:10B4C0000170E043000700D036B9012241462869E7
:10B4D00002F09CFB0028CDD0641C002EC2D10120BC
:10B4E000C8E7002070470020704700207047002008
:10B4F0007047704700207047002070470020704759
:10B50000002070470020704770B505460C4608695A
:10B51000142100F049FD002820D028785C2800D1B3
:10B520006D1C2878002819D00020E06101222146F6
:10B53000284600F09FF8002810D0206921467C3072
:10B54000FFF71CFB002809D0206900237C301A4635
:10B550002146FFF751FD002800D0012070BD70B5D5
:10B5600005460C460869142100F01EFD002838D05D
:10B5700028785C2800D16D1C2878002831D0002064
:10B580000246E0612146284600F074F8002828D0E1
:10B59000206990F87C1029B17C300022214600F00F
:10B5A0001DFC02E02046FFF71BFC002819D02046B6
:10B5B000FFF74AFF002814D0E169206902F05EF825
:10B5C00000280ED02069017F032909D102F0EAFA90
:10B5D000002806D00021206902F094F9002800D04C
:10B5E000012070BD70B504460E4615460421106951
:10B5F00000F0DAFC002816D020785C2800D1641C0A
:10B60000207800280FD000200246E8612946204615
:10B6100000F030F8002806D02946304600F0FAFE47
:10B62000002800D0012070BD70B505460C460869A1
:10B63000042100F0B9FC00281BD028785C2800D138
:10B640006D1C2878002814D0002632462146284652
:10B65000E66100F00FF800280BD0206900227C3052
:10B66000214600F0BBFB002803D06675E069A061AD
:10B67000012070BD2DE9F047002706460D46914692
:10B68000B84620E0286901227C30294600F0A6FB5C
:10B69000C0B95FEA09002DD00127286929467C300E
:10B6A000FFF76CFA002825D0286900237C3001229E
:10B6B0002946FFF7A1FC00281CD0284602F07CF99F
:10B6C000002817D0264429697C3100242046325DA9
:10B6D0005C2A06D0222A04D04AB10A54401C641CB9
:10B6E000F5E7641C01F80080002FD6D1CAE701F805
:10B6F00000800120BDE8F0872DE9F0414FF0FF35D3
:10B7000000F148048564806860604FF0000626728E
:10B71000667200F5007100F58060E560C4E905100F
:10B72000267766774FF00208C4F82480A4F1480415
:10B730004FF0300104F11800F5F706F8002120461B
:10B7400001F0A4FD08B3E06D00F5FF7001F022F8F0
:10B75000A0F52A41553918D1E06D0178E9290AD0C0
:10B76000EB2902D18178902905D000F5E37001F032
:10B7700016F8A06100E0A661204600F000FD38B197
:10B78000E18DB1F5007F40D104E00220BDE8F081F9
:10B790000320FBE7A07F08280DD006DC01280AD093
:10B7A000022808D0042830D105E0102803D0202832
:10B7B00001D0402829D1B4F822C0BCF1000F24D018
:10B7C000627F012A01D0022A1FD1238C666AB3420C
:10B7D0001BD8A78D02FB03C305EB471505F50075C4
:10B7E00095FBF1F15A18B21AA262B2FBF0F2226391
:10B7F000A386E1864002A0634009A08740F6F57069
:10B80000824204D20120207716E00420BEE74FF6E2
:10B81000F570824202D284F81C800DE0032020776C
:10B82000204600F0B7FD38B92046FFF760FBA06660
:10B83000204602F0B7F908B10020A7E70520A5E7E8
:10B84000012070472DE9F0470446008889461746D5
:10B85000C00613D40421206900F0A6FB50B1E068B3
:10B86000A168C2198A4201D90F1A07D0C0F308068D
:10B8700000253AE0208840F0100020800020BDE83C
:10B88000F087A1692069FFF725FB627D8118206997
:10B89000837F9A1A01F0A2FC0028F0D0A7EB0508DC
:10B8A00008EB0600B0F5007F01D9C6F500782069E5
:10B8B0004246C06D811909EB0500F4F7ACFE06EBBA
:10B8C0000800C605F60D0FD1607D401CC1B2617540
:10B8D0002069827F914207D10021617504F118012E
:10B8E00001F04AFE0028CAD04544BD42C9D3E068F1
:10B8F0002844E0602846C2E770B506460C46154667
:10B900001421106900F050FB002839D030785C28F1
:10B9100000D1761C20785C2800D1641C307880B37C
:10B92000207870B300200246E86129463046FFF7D0
:10B93000A1FE002824D0286990F87C0080B1002660
:10B94000324629462046FFF748FA01281AD02869CE
:10B9500000227C30294600F041FA002810D007E090
:10B960000126324629462046FFF737FA012809D03A
:10B9700032462946204601F0B2FC002800D00120C2
:10B9800070BDFFE70020FBE72DE9F0410446008889
:10B990000D46C00602D50020BDE8F08104212069D3
:10B9A00000F002FB40B3A068A84200D2054620691F
:10B9B000690A827FB1FBF2F302FB13116175E7693B
:10B9C000A761806BB5FBF0F656B104F1180841464B
:10B9D000A769206901F0D0FD0028DDD0761EF6D1E0
:10B9E000A169206900F04EFF18B12069807F607561
:10B9F000A7610120E560CFE7208840F0100020809B
:10BA0000C9E7F0B50446008889B0C0065FD41421A8
:10BA1000206900F0C9FA002855D0D4E9010181421B
:10BA20004CD9491E2046FFF7AFFF002850D02069AF
:10BA300000F093FB0246A169206902F03FF800285C
:10BA400046D06946204601F006FC002840D0E06957
:10BA5000000CADF81400E069ADF81A00A06807907A
:10BA600000F080FE01460DF1160001F0CBFD00F064
:10BA7000DEFB014606A801F0C5FDBDF81800ADF8D3
:10BA800012006F46E58A216A206900F0E6FB00EBB0
:10BA900015110E46206901F0F9FBC0B1206905F0CF
:10BAA0000F012022C06D00EB41103946F4F7F8FD7C
:10BAB00001223146206902F0A9F840B12069017FD6
:10BAC000032907D00AE0208840F0100020800020E1
:10BAD00009B0F0BD02F066F80028F9D00021206915
:10BAE00001F010FF0028F3D000212069FFF7F4F8DF
:10BAF0000028EDD00120EBE72DE9F74F0446008840
:10BB000082B01746C00603D5002005B0BDE8F08F0F
:10BB10001421206900F048FA60B121884FF40079BF
:10BB200009EA811B04F11800E1694FF0000A009056
:10BB300029B10EE0208840F010002080E4E7206961
:10BB4000009900F0B9FB0028DFD0A069E06184F81B
:10BB500015A0E0680025C0F308064CE02069617D6F
:10BB6000827F914218D1E168A2682944914203D2B0
:10BB7000009901F001FD0BE0D4F81880009900F065
:10BB80009BFB0028C1D04146A269206901F096FFC5
:10BB90000028BAD084F815A0A1692069FFF79AF9A6
:10BBA000617D084401900EB95F4505D22069019975
:10BBB00001F06CFB0028A8D0A7EB050808EB0600F5
:10BBC000484501D9C6F500780398424641192069D5
:10BBD000C06D3044F4F71FFD2069019901F092FE19
:10BBE000002892D006EB0800C605F60D02D1607D54
:10BBF000401C60754544BD42B0D3E0682844E06015
:10BC0000A168884200D9A06001207EE72DE9F05F9D
:10BC100005460C466848AFF30080002000F004FAA7
:10BC2000060055D00146284600F04CFA824630699D
:10BC300000284DD000205146024604E0401C5C2BF9
:10BC400000D10246491C0B78002BF7D10AEB020009
:10BC500083465AA1F4F7A0FD00B32A21584600F00C
:10BC60006DFA05465846F4F7ABFC8046681C1AD0BE
:10BC70004FF001090BEB050051A1F4F78DFD18B150
:10BC8000A8EB0500A0F101008046308880060DD5A4
:10BC9000324621465046FFF7A5FC0BE000254FF049
:10BCA0000109A846F1E74FF00009EEE731462046CA
:10BCB000FFF71BFC60B1002084F8FF00B9F1000F12
:10BCC00008D055EA08001FD0CDB35946002349E0FB
:10BCD00001242EE023465A4610E05B1C12F8011B9B
:10BCE000A0F16107192F01D820F02000A1F1610710
:10BCF000192F01D821F020018842C6D118780028D8
:10BD0000EBD111780029E8D13088800603D5307D49
:10BD100084F8060109E0002084F80601F082B4F8F6
:10BD20000401B0823046FFF7E4FB7068C4F80001FC
:10BD300000242148AFF300802046BDE8F09F13E0C7
:10BD400011F8012BE05CA2F16107192F01D822F054
:10BD50002002A0F16107192F01D820F020008242B3
:10BD600093D15B1CAB42EBDBB8F1000FCCD020468B
:10BD7000F4F726FC844605EB0801614585DC0BEBF6
:10BD800005035B1CACEB080212E000BF13F8010BCB
:10BD9000A15CA0F16107192F01D820F02000A1F1CA
:10BDA0006107192F01D821F020018842A5D1521C2A
:10BDB0006245EBDBA8E70000000000002A2E2A0005
:10BDC0002E2A00000168002901DCF4F77ABF491E21
:10BDD000016041684A1C426008787047002301F006
:10BDE000BBBA0000F0B5044689B01A48AFF3008032
:10BDF00000F0AAF8BCB10020ADF80000049069463C
:10BE0000204600F05FF9049808B3BDF8000000F088
:10BE10002001049800F0CEFC04460E48AFF30080E9
:10BE200009B02046F0BD00240B4D26460B4F0AE01A
:10BE3000E87900F00401286800F0BCFCA04200DDB5
:10BE40000446761C083538888642F1DBE5E7032492
:10BE5000E3E7000000000000BC390208A239020834
:10BE60008A68002A01DCF5F71FB9521E8A604A6809
:10BE7000C0B2531C4B60107070470000F0B5044610
:10BE800095B00F462F48AFF30080002000F0CCF8AB
:10BE900005004ED00146204600F014F906462869F8
:10BEA00080B3288880062ED53046F4F789FB441EDF
:10BEB00006D4305D5C2802D0641EFAD500E06CB177
:10BEC000621C31466846F4F7A6FB0DEB0401002026
:10BED000487039466846F4F792FB07E03846F4F7B5
:10BEE0006FFB024639466846F4F795FB29466846DB
:10BEF000FFF79AFB01281CD02A4639463046FFF747
:10BF0000FBFC14E015E029463846FFF7F0FA01285B
:10BF10000FD029463046FFF7EAFA50B1284600F024
:10BF2000A7F8012805D029463846FFF7E5FA012889
:10BF300006D001240348AFF3008015B02046F0BDC1
:10BF40000024F7E70000000070B5124C20780028AC
:10BF50001ED100F041F800220F4811460F4B05E0BA
:10BF6000C5796D0750F8085B521C29601D88AA42EC
:10BF7000F6D300200A4B0B4A05E000BF00EBC005DA
:10BF8000401C23F825101588A842F7D30120207003
:10BF900070BD000088020020BC390208A2390208E6
:10BFA00014240020A039020810B50446006881431B
:10BFB00001D0002010BD000706D46068002142694E
:10BFC00008469047C00701D0012010BD206820F02E
:10BFD00006002060EDE7000007480021A0F5806220
:10BFE000C0E90221054A426000F5C073044A9A6024
:10BFF0004161018270470000A4280020A439020892
:10C00000D839020860B1017851B1012100E0491C22
:10C01000425C002AFBD1084410F8010C5C2801D0D6
:10C02000002070470120704770B5064600240A4D75
:10C030000A4804E02988890706D02435641C018851
:10C040008C42F7DB002070BD24212846F4F77CFBEE
:10C0500006B13460284670BD14240020A0390208BF
:10C06000004870470101DB074FF440207047000093
:10C0700030B500221149124B1AE00C88A40715D0E4
:10C08000814213D00C690569AC420FD10488A40623
:10C0900009D5CC8AC58AAC4208D10C6A056AAC4283
:10C0A00004D1012030BD8C8A858AF8E7521C2431E6
:10C0B0001C88A242E1DB002030BD000014240020D7
:10C0C000A0390208F0B51B4A1B4CE8B10378DBB17C
:10C0D00023F0200643783A2B03D085783A2D03D0FD
:10C0E00012E03023801C01E073B1C01C002507E082
:10C0F0001779B74202D157799F420AD06D1C083296
:10C100002788BD42F4DBF0BD00230EE0D579ED07B2
:10C1100009D013680B61D2795207F4D50A8842F02E
:10C1200020020A80F0BD5B1C08322588AB42EDDBA3
:10C13000F0BD0000BC390208A2390208002205E067
:10C140008B4201D110467047401C521C0378002BD3
:10C15000F6D1581E704700207047007F012805D097
:10C16000022806D0032807D00020704740F6FF7051
:10C1700070474FF6FF7070476FF07040704710B512
:10C180000446816901F082F8002809D0E06D00F5CD
:10C19000FF7000F0FFFAA0F52A41553901D00020C8
:10C1A00010BDE06D417BA1770B3000F0F3FAE08524
:10C1B000E06D0E3000F0EEFA6084E06D017C617796
:10C1C000113000F0E7FAA085E06D133000F0E2FADC
:10C1D0006062E06D163000F0DDFA2084616AE9B932
:10C1E000B8B9E06D283000F0D5FAE087E06D2C306A
:10C1F00000F0D5FA2064E06D303000F0CBFAA4F8FE
:10C200004400E06D323000F0C5FAA4F84600606AE0
:10C2100020B9E06D203000F0C2FA6062208C20B9B5
:10C22000E06D243000F0BBFA2084012010BD10B571
:10C23000FFF716FF10F01F0100D10121C0F3032208
:10C240000C2A00D802B9012241EA4211442202EB31
:10C25000104041EA402080B210BD10B5002280F8A5
:10C260007B2059B90267017F032906D0828E81693C
:10C270001144012280F87B2003E0016CFEF72AFEC6
:10C280000146084610BD027F012A04D0022A06D0CA
:10C29000032A0AD105E001EB4101890A02E0090AFB
:10C2A00000E0C909028C8A4201D8002070478269E7
:10C2B000408C1044084470472DE9F04105460E4675
:10C2C000C46E5CE021462846FFF7DDFF804601464C
:10C2D0002846FEF701FD002838D0287F012804D029
:10C2E000022823D0032830D127E004EB4400C0F318
:10C2F0004800B0F5FF7F04D8E96C084400F04AFA22
:10C300000DE0E86C08F1010190F8FF712846FEF796
:10C31000E3FC00281AD0E86C007847EA0020E10727
:10C3200001D000090FE0C0F30B000CE0E96C20061F
:10C3300001EBD05000F02EFA05E0E96C600601EB4D
:10C34000D05000F02CFA18B118E00020BDE8F081C0
:10C350000E48002102880E4809E003889F0604D594
:10C360009B0702D58369A34208D02430491C91421F
:10C37000F3D33460641C0120EC66E7E7641C286B8F
:10C38000801CA0429ED8EC66DFE70000A0390208BE
:10C390001424002010B504468069B4F84410014408
:10C3A000204600F073FF002829D0E06D00F5FE70F4
:10C3B00000F0F5F91449884220D1E06D00F0EFF962
:10C3C000124988421AD1E06D00F5F27000F0E7F9E9
:10C3D0000F49884212D1E06D00F5F47000F0DFF9EA
:10C3E000216B81420AD3A066E06D00F5F67000F083
:10C3F000D6F9022802D3216B814201D2002010BD60
:10C40000E066012010BD0000000055AA52526141B3
:10C41000727241612DE9FF5F054600200E460290D1
:10C4200001900390C969814600913069FFF715FFBB
:10C43000B5F8047182464FF0000B306990F87B002C
:10C44000E0B1B7F5007F10D01CE07F1A016C009AB4
:10C45000914200D90091694601F08EF8002805D07C
:10C460003069009900F00EFA18B1002004B0BDE860
:10C47000F09F30690099FEF72DFD82463069818F6B
:10C48000B942E2D909F101090AEB1711306900F04C
:10C49000FDFE0028EAD0306907F00F01C06D00EB07
:10C4A000411420780028E1D0E5285AD0E17A0F29FC
:10C4B00002D0080755D407E0400605D501200390B7
:10C4C0000190607B029011E0039878B30F290BD0A4
:10C4D00000200390204600F0F1F90199002975D061
:10C4E0000299884248D001E00198D0B3617B02985C
:10C4F000814202D00020019068E02078344B00F0A7
:10C500001F00401E00EB800101EBC00805EB080195
:10C5100000201A5CA25C0A54401C0D28F9D3207834
:10C5200008F10D08400601D505F808B0E07A00F0E2
:10C530003F000F284AD0072100E0491E605C2028F8
:10C54000FBD0491C002002E0225C2A54401C884297
:10C55000FAD3217A20290DD02E212954401C0821FC
:10C5600003E033E02A54491C401C625C202A01D0BD
:10C570000B29F7D305F800B005F58275298801EB82
:10C5800009002880E07A307504F11C0000F007F9FA
:10C590007060B06004F1160000F0FCF8C10A297167
:10C5A000C0F34511C0066971800EA87104F118002E
:10C5B00000F0F0F800F01F01E971C0F34311400AE8
:10C5C000297200F2BC70688101204FE77F1C34E7BC
:10C5D0004A4103082DE9F84F834660480E46154648
:10C5E0004FF0000A4FF6FF78824201DD062713E084
:10C5F00042F20F70854201DD05270DE0B5F57A7F27
:10C6000001DB042708E0632D01DD032704E0092D89
:10C6100001DD022700E00127002003E02E2900D1E0
:10C620008046401C1BF800100029F7D105B94F1EA9
:10C630004FF00009C7F107004C46009018E000BF1A
:10C640001BF809A0BAF1200F10D0BAF12E0F0DD0AF
:10C65000BAF1000F11D0AAF16100192801D82AF00F
:10C66000200A504601F0A7F83055641C09F1010971
:10C67000C14502D20098A042E2D8EDB37E203055E9
:10C68000641C072F46D2DFE807F04542352A1E1208
:10C69000040032483249401C95FBF0F0414305EB61
:10C6A0004115092800D9092030303055641C42F268
:10C6B000107095FBF0F06FF41C7141433030305531
:10C6C00005EB0115641C4FF47A7095FBF0F06FF0E8
:10C6D0007C0141433030305505EBC105641C6420BA
:10C6E00095FBF0F06FF0180141433030305505EB09
:10C6F0008105641C0A2000E00CE095FBF0F041424B
:10C70000303001EB8101305505EB4105641C3035BB
:10C710003555641CBAF1000F1AD02E203055641C18
:10C72000A8F57F414046FF3912D0451C071D0DE09A
:10C730001BF8050060B1A0F16101192901D820F0B2
:10C74000200001F038F83055641C6D1CBD42EFD359
:10C75000002030550120BDE8F88F00009F860100C1
:10C76000CBF3FFFF10B5FFF77FFCC0F344011D2999
:10C7700000D90021C0F305223B2A00D90022C0F3D2
:10C78000044041EA4211172800D9172041EAC0208D
:10C7900080B210BD4178007840EA01207047C1782E
:10C7A0008278090641EA02414278007841EA022192
:10C7B0000843704710B5044640680022B1B318B171
:10C7C0002068C00702D00BE0032010BD2260606823
:10C7D00001680020884750B3206840F001012160C3
:10C7E000206820F01E01216060680021426908462F
:10C7F0009047010603D5206840F0180106E0C10704
:10C8000038D0800703D4206840F0100121606068B0
:10C8100001680120884750B1206840F0020120469D
:10C820002160FEF769FF18B1022010BD0AE021E087
:10C83000206840F0040120462160FFF701F8F0B9BC
:10C840000420F2E768B12068C0070AD12260D4E969
:10C850000120E1691268904760B1206840F0010052
:10C860002060206840F004002060616821B1896880
:10C8700011B104E00120D8E740F010002060002052
:10C88000D3E70000007F012804D0022805D0032848
:10C890000FD107E040F6F87001E04FF6F8708142E2
:10C8A00005D206E021F070400349884201D30120FF
:10C8B0007047002070470000F8FFFF0F024600207D
:10C8C0000146C30700D0802303EB5000535C491C92
:10C8D0001844C0B20B29F4D370470000FBF7D2F91B
:10C8E000F9F722FEF8F7EEFDF6F716FBFCF7D2FBA0
:10C8F000FDF744F8F4F7B6FDF9F714F9FBF7D6FBAA
:10C90000F9F73AF9F9F79AFDF5F7BEFCF5F7BCFC33
:10C910000020624908600520614908604FF41670E4
:10C920006049086000206049087060490860012083
:10C930005F490870F5F7F8FC6820FBF73BFC0446FC
:10C9400040F2E7325B4801682046FDF717FD42F2EE
:10C95000D8716420FDF7CAFCF5F7D4FD4FF42F70B1
:10C9600055490860FCF7F8FEF5F720F9FDF75AFC89
:10C97000F5F7BAF900210A20FDF7B8FC00210B20D9
:10C98000FDF7B4FC00210C20FDF7B0FCFBF74CFFD9
:10C9900001204A4908604FF42F70494908604860F7
:10C9A0007BE0FBF7FBFFF4F739FE3D48006810B968
:10C9B000012044490870FBF70DFD3C4800683B49E5
:10C9C0000968491C394A1160062835D005DC45D272
:10C9D000DFE800F013161924272F092835D004DCCE
:10C9E00007282CD0082839D12CE00A2830D0A0F50F
:10C9F00098508838002831D12DE0F5F795FC31E0CA
:10CA0000F5F732F92EE0F9F745F8274800780128C4
:10CA100003D141F288302549086023E0F5F706FC90
:10CA200020E01F48006818B142F210701F490860EA
:10CA300018E0F5F7D3FD15E0F5F752FA12E0F5F737
:10CA40007FFB0FE0F5F79CF90CE0F4F7DBFF09E062
:10CA5000F5F70CF906E0F5F793FA03E00020134927
:10CA6000086000BF00BF18480068B0F5FA7F05DA1B
:10CA70004FF480611548F8F758FF04E04FF48061E7
:10CA80001248F8F750FFF6F72FFCF5F73BFDF5F7E6
:10CA9000FBFBF5F70BF8F9F755F882E7500000209B
:10CAA000AC000020F0000020340100200C00002029
:10CAB000000000203000002034000020480000204A
:10CAC000780A00201000002014000020000C014013
:10CAD000014A00F05FB80000242A0020014900F05C
:10CAE00066B80000242A0020014900F05DB900006A
:10CAF000242A0020014B00F067B90000242A0020FE
:10CB0000014900F08DB90000242A0020014B00F0FB
:10CB100093B90000242A00202DE9F0410746184966
:10CB2000184A126831F81200F8F7A2FF0646F8F723
:10CB300001FF054614481349096850F821002C1AD2
:10CB4000002C00DA64420A2C0EDB10480D490968FB
:10CB5000405C401CC0B20D490A4A126888546428DF
:10CB600002DC0B48006848B107480649096840F8EC
:10CB7000215000200549034A12688854BDE8F0811D
:10CB8000040C0020B8000020780A0020BC0000201F
:10CB9000AC00002018B1022807D000207047906830
:10CBA000C06900B1004780207047506870472DE988
:10CBB000F8430C4610B101287DD104E08868006874
:10CBC0008047BDE8F883A068816901208847A06894
:10CBD00041694FF4C87088470025A0688168FF202C
:10CBE00088476D1C102DF8D3A06881690020884704
:10CBF000002223461146104600F04CF90546002657
:10CC0000012D07D0A0688168FF208847761C054663
:10CC1000642EF5D3A068816901208847012DCBD10E
:10CC2000A068416944F62060884700202070A06811
:10CC300081690020884704268DF8006023466A46F3
:10CC40004FF4D571082000F025F901280FD19DF887
:10CC5000000060B99DF8010048B99DF80200012864
:10CC600005D19DF80300AA2801D103202070A068F7
:10CC700081690120884700254CF25038A0688169FD
:10CC800000208847002223461146372000F002F991
:10CC90000746A06881690120884778071AD4012FC8
:10CCA00015D1A0688169002088472078032815D015
:10CCB0000020810700E06EE023460022292000F0DA
:10CCC000E9F80746A06881690120884747B16D1CD3
:10CCD0004545D3D32078032807D01EE00120E8E79C
:10CCE0002078032801D0022033E0A0688169002069
:10CCF00088478DF8006023466A4600213A2000F0FC
:10CD0000C9F80546A0688169012088472DB99DF8BA
:10CD10000000400601D526701CE02078D0B900251F
:10CD20004746A068816900208847002223461146B3
:10CD3000012000F0AFF80646A0688169012088470D
:10CD4000012E01D03EBB03E06D1CBD42E9D322E0C1
:10CD500001202070A06881690020884723460022B6
:10CD60004FF40071102000F095F80546A068816925
:10CD7000012088477DB9A06881690020884700228A
:10CD8000234611463B2000F085F80546A0688169DE
:10CD9000012088470DB1002013E7204600F002F97A
:10CDA0000028F9D001200CE770B505460C4608466E
:10CDB00000F0F8F8002806D02146284600F017F9C0
:10CDC000002800D0012070BD2DE9F041064698688A
:10CDD0000F46154681691C460020884723462A468F
:10CDE0003946304600F0A6F80646012D0FD900223C
:10CDF000234611460C2000F04DF8084DA0688168CC
:10CE0000FF208847FF2802D06D1EF7D10026A068BA
:10CE10008169012088473046BDE8F08148E801007B
:10CE200038B101284FF0000002D10870486001209D
:10CE300070478868406800472DE9F04106469868C9
:10CE40000F46154681691C460020884723462A461E
:10CE50003946304600F046F90646012D11D9A06842
:10CE60008168FD208847A0688168FF208847084DB9
:10CE7000A0688168FF208847FF2802D06D1EF7D187
:10CE80000026A0688169012088473046BDE8F0810E
:10CE900048E801002DE9FC4140F040008DF8000019
:10CEA000080E8DF80100080C8DF80200080A8DF8B4
:10CEB0000300002014461D468DF804106A46014602
:10CEC00005234E0707D1B3EBD10F04D902EBD106EE
:10CED000367846EA0000060401D580F40940400097
:10CEE000491C3029EDD3000A40F001008DF80500FF
:10CEF000A8688168FF208847A8680621C26868463C
:10CF000090470027A8688168FF2088470646FF28C9
:10CF100002D17F1C082FF5D34CB1277805E0A86813
:10CF20008168FF20884704F8010B7F1EF7D2F0B21A
:10CF3000BDE8FC812DE9F04111250F4616461C463F
:10CF4000012A00D912252178042900D24002014685
:10CF500000222846FFF79EFF10BB1CE046F2A815F2
:10CF6000A0688168FF208847FE2802D06D1EF7D197
:10CF700016E0ADB1A0684FF40071026938469047E1
:10CF8000A0688168FF208847A0688168FF208847E3
:10CF900007F50077761E002EE0D10120BDE8F08174
:10CFA0000020FBE77FB50446806881690020884740
:10CFB0002346102269460A2000F06CF80546A06856
:10CFC00081690120884775B12078012868460CD016
:10CFD00009300168C07809BA21F0FF01014301203E
:10CFE000616004B070BD0020FBE70A30F1E77FB557
:10CFF000044688680D468169002088472B46102228
:10D000006946092000F046F80646A86881690120B3
:10D010008847B6B19DF80500012100F00F0001FA24
:10D0200000F0A080BDF80C0040BAC0F3831081402E
:10D03000E1809DF80000800906D0012819D002285F
:10D0400002D0002004B070BD9DF806009DF80710C6
:10D05000000440EA01209DF808100843BDF80910BB
:10D06000C0F38B1049BAC1F3C211401C891C88401F
:10D070000DE09DF807009DF80810000440EA01202B
:10D080009DF8091008430004800900F580602060C5
:10D090000120D7E72DE9F04117460E4600221C4635
:10D0A0001146FFF7F7FED8B946F2A815A0688168C7
:10D0B000FF208847FE2802D06D1EF7D110E07DB119
:10D0C000A0683946026930469047A0688168FF2011
:10D0D0008847A0688168FF2088470120BDE8F0816B
:10D0E0000020FBE72DE9F0411826884615461C462E
:10D0F000012A00D919262178042900D240020146CC
:10D1000000223046FFF7C6FE38BBFE27012D29D985
:10D11000FC2727E0A068816838468847A0684FF45C
:10D120000071C26840469047A0688168FF20884728
:10D13000A0688168FF208847A0688168FF20884731
:10D1400000F00F00052812D10A4EA0688168FF2068
:10D150008847FF2802D0761EF7D108E03EB108F5D7
:10D1600000786D1E002DD5D10120BDE8F081002092
:10D17000FBE7000020A1070070B5002480201049C3
:10D180000880032088700420C8700E48F8F748FB18
:10D19000002510E06006040EFCF7CEF8FEF744F917
:10D1A00080210848F8F7B1FB08B144F00104FCF70E
:10D1B000CDF8681CC5B2082DECDB204670BD000020
:10D1C00024010020000C014010B5FCF7DFF8FCF74B
:10D1D000B3F8FCF7BBF8FCF7C3F810BD70B5044614
:10D1E000C0680D46164610B194F8641029B129465E
:10D1F0002046BDE8704000F049B894F8652082B13F
:10D20000A16DA9420DD80A44AA420AD9206E691A12
:10D2100000EB41214FF40072E06DF3F7FCF9656516
:10D2200017E0B04200D206466068E16D324683687E
:10D2300028469847012806D04FF0FF30606500204F
:10D2400084F8650070BD65656D1C761EA56584F863
:10D250006560012070BD70B50E460446C58A016A3E
:10D260000069FEF7FAFF00EB1511206900F00EF8D7
:10D2700000280AD0206905F00F012022C06D00EBC4
:10D2800041113046F3F70CFA012070BD70B5044629
:10D29000406D0D46A84201D1012070BDA06DA8428D
:10D2A0000ED894F864100144A94209D9216E281AB5
:10D2B00001EB40214FF40072E06DF3F7ACF90CE0A4
:10D2C0006068E16D0122836828469847012804D0F0
:10D2D0004FF0FF306065002070BD6565DCE72DE92B
:10D2E000F0410746086988B00C4690F87A6090468D
:10D2F00000253846FDF739FD60B1012E09D03846CA
:10D30000F3F75EF90C300D21B0FBF1F0401CB04298
:10D3100000D9012569462046FFF79DFF002817D058
:10D320002046FEF791F8002812D045B12069214629
:10D33000406FE0613846FDF721FC002808D06B46BD
:10D34000424621463846FDF757FE002800D001200E
:10D3500008B0BDE8F08100002DE9FF4F97B00C4602
:10D36000012A19D00020129001204FF0000ACDE9C7
:10D370000E0A0390E06900901798F3F721F90490E2
:10D380000020109021698346E06908671798FDF72F
:10D39000ECFC012802D009E00120E4E704980D210B
:10D3A0000C30B0FBF1F0401CC0B20E9009A91798E8
:10D3B000FDF7EBFF129808B1092000E00D2007905F
:10D3C00020690099FEF749FF81460026206990F800
:10D3D0007B1019B1B6F5007F13D01BE0818FB142ED
:10D3E00018D1016C009A0026914200D9009169463B
:10D3F00000F0C2F8002805D020690099FFF742FA32
:10D4000018B100201BB0BDE8F08F20690099FDF72E
:10D4100061FD814609EB16112069FFF737FF0028EF
:10D42000F0D0206906F00F01C06D00EB411528789F
:10D430000028E7D0E5286FD095F80B80B8F10F0FE2
:10D4400003D05FEA087067D431E0410609D500993E
:10D450001091697B0F9120F04001491CC9B2B3467D
:10D4600003916A7B0F998A4256D100F01F00401E3B
:10D4700000EB800101EBC0001799DFF8F8C00A1833
:10D48000002000BF1CF80010135C695C81EA0307F0
:10D4900037F0200708D103B911B1401C0D28F1D392
:10D4A0000AF1010000F0FF0AB8F10F0F34D0039821
:10D4B00001280ED029D9A0F1010050451BD12846E2
:10D4C000FFF7FCF90F99884215D10AF10100C0B2AB
:10D4D0001AE00E98012803D007990498884214D2C4
:10D4E00000981090B34609A9284600F097F878B143
:10D4F0004FF0010A12E00E98012806D109A928462A
:10D5000000F08CF808B1039882460398504505D086
:10D5100001204FF0000A0390761C57E7E87AC0F329
:10D52000001112988142F3D11A9808BBE87A20754D
:10D5300005F11A00FFF72EF9074605F11400FFF771
:10D5400029F907EB0040E061E6820098206221693A
:10D550001098486721690020A1F878B0216981F806
:10D560007AA0E06005F11C00FFF719F96060A06087
:10D57000012047E74A4103082DE9F0410D680E46B6
:10D5800004462946FEF77FFE804601462046FDF709
:10D59000A3FB002807D0207F012806D0022825D031
:10D5A000032828D00020BDE8F08105EB4500C0F33A
:10D5B0004800B0F5FF7F04D8E16C0844FFF7EAF8B3
:10D5C0000DE0E06C08F1010190F8FF712046FDF7D5
:10D5D00083FB0028E7D0E06C007847EA0020E907E9
:10D5E00001D000090BE0C0F30B0008E0E16C280655
:10D5F000C00D085A03E06806E16CC00D08583060A1
:10D600000120D0E70A0A4270017070470A0EC2700A
:10D610000A0C82700A0A42700170704730B500220D
:10D62000835C8C5C83EA040535F0200501D0002082
:10D6300030BD04B913B1521C0B2AF1D3012030BD07
:10D6400010B5FBF78DFEFBF777FEFDF7EDFEFBF760
:10D650009DFEFDF7E9FEFBF779FEFDF7E5FE10BD47
:10D6600010B5FBF793FEFDF7DFFEFBF765FEFDF758
:10D67000DBFEFBF775FEFDF7D7FE10BD2DE9F04789
:10D680000026012704460D4602297DD379E0E06E8D
:10D69000A84200D9E56629462046FEF7F4FD8146FA
:10D6A00001462046FDF718FB00287AD0207F01288C
:10D6B00004D0022846D0032872D14DE005EB450086
:10D6C000C0F34808B8F5FF7F16D8E16C01EB0800FD
:10D6D000FFF760F8E90703D000F00F01000903E04D
:10D6E00000F47041C0F30B00E26C814602EB0800CD
:10D6F00089B2FFF787FF3BE0E06CEA0790F8FF1183
:10D70000884604D001F00F0180F8FF1101E080F895
:10D71000FF6184F8507009F101012046FDF7DCFA41
:10D7200000283ED0E06CEB07017848EA012202D0E5
:10D730000670100904E001F0F0010170C2F30B0063
:10D74000814615E02806C50DE06C2844FFF722F855
:10D750008146E06C46530BE06806C50DE06C28443A
:10D76000FFF71DF88146E06C4651A06E401CA06694
:10D7700084F8507049462046FFF784F8012812D0FB
:10D780004D46206B801C02E013E00AE008E0A8424E
:10D790003FF67DAF00212046FDF79EFA002800D01D
:10D7A0000020BDE8F08700212046FDF795FA00280B
:10D7B000F7D00120F5E710B5044600F005F808B1F0
:10D7C000204610BD582010BDA0F12001012917D915
:10D7D000C91E062914D92D2812D02E2810D00D3993
:10D7E00009290DD940280BD01139192908D91D391B
:10D7F0001D2905D97D2803D07E2801D0002070473F
:10D800000120704710B501210248F8F78EF8FDF7A6
:10D810000BFE10BD0018014010B501210248F8F7B9
:10D8200082F8FDF701FE10BD0018014070B50446F6
:10D83000254600260FE005F0800010B1FBF790FDB3
:10D8400001E0FBF7A3FD6806050EFBF775FDFBF78E
:10D850007DFD701CC6B2082EEDDB70BD70B50125D4
:10D86000FBF77EFDFBF768FD80210A48F8F74DF8CD
:10D8700000B10025FBF76AFD07480068012806D1C2
:10D88000002402E0FDF7D0FD641C0A2CFADB2846D8
:10D8900070BD0000000C0140200100202DE9F04186
:10D8A00007460C460A201649086000BFFFF7C8FE6D
:10D8B000A02101EB4701C8B200F072F805460DB98E
:10D8C000FFF7CEFE1DB90E4800680028EED145B125
:10D8D0002646E11704EB1161C1F3072000F060F860
:10D8E000054655B12646E11704EB11610912A4EB78
:10D8F0000121C8B200F054F805462846BDE8F08181
:10D90000180100202DE9F0410D46C1680446E1B13F
:10D9100000261DB3656594F864204FF400779AB330
:10D92000A06D8318AB4227D18A4225D204F15C0452
:10D930006068216800EB42203A46F2F76CFE207ADC
:10D94000401C20720120BDE8F081002DFAD0002299
:10D95000294600F05BF90028F5D0F3E794F864203D
:10D96000002AEFD06368216EA06DDB68984700281D
:10D97000E9D084F86460E5E76368216EDB68984766
:10D980000028E0D084F8646004F158043A46D4E9F1
:10D990000110F2F740FE0120256020736673D1E785
:10D9A00010B504462046FFF741FFFFF757FF08B1C7
:10D9B000012010BD0020FCE72DE9F0410446C769B5
:10D9C000FEF7D0FE0646FEF732FC804620694FF493
:10D9D0000071C06DF2F796FE20690B2234A1C56D6F
:10D9E0002846F2F75DFE1020E872314605F10E0080
:10D9F000FFF708FE414605F11000FFF703FE414620
:10DA000005F11200FFF7FEFD314605F11600FFF7A4
:10DA1000F9FD414605F11800FFF7F4FD05F120007E
:10DA2000202229460646F2F73BFEE069010C05F18B
:10DA30001400FFF7E7FDE06981B205F11A00FFF776
:10DA4000E1FD2E2070702069006F010C06F11400BA
:10DA5000FFF7D8FD2069006F81B206F11A00FFF7C9
:10DA6000D1FD2169E069086739462069FDF732FA7E
:10DA7000064601223146206900F0C8F8002814D07B
:10DA800020694021C06DF2F73DFE012506E07119C5
:10DA9000002200F0BBF8002807D06D1C2069817FB0
:10DAA000A942F4D80220E0820120BDE8F081000004
:10DAB0002E20202020202020202020002DE9F047AB
:10DAC000154604460E46FEF7DEFB8146014620461B
:10DAD000FDF702F9002809D0207F4FF00108012846
:10DAE00006D0022844D0032848D00020BDE8F087A3
:10DAF00006EB4600C0F34807C5F30B05B7F5FF7FFB
:10DB000013D8E06C3844FEF745FEF10702D065F308
:10DB10001F1002E000F470402843E16CCA1981B282
:10DB20004FEA0200FFF76EFD38E0F007E06C06D028
:10DB300090F8FF1165F31F1180F8FF1101E080F8E4
:10DB4000FF5184F8508009F101012046FDF7C4F827
:10DB50000028CBD0F00703D0E16C280908701DE045
:10DB6000E06C017801F0F00141EA1521017015E047
:10DB7000E16C300601EBD050A9B2D3E77006C60DB8
:10DB8000E06C3044FEF70BFE18B9A06E08B1401EE1
:10DB9000A066E06C29463044FFF738FD84F85080D9
:10DBA0000120A3E710B50446C06D4FF40071F2F7F1
:10DBB000A9FD1449E06DFFF729FDE06D124900F55C
:10DBC000F270FFF723FDE06DA16E00F5F470FFF732
:10DBD0001DFDE06DE16E00F5F670FFF717FDE06DDD
:10DBE0004AF6552100F5FF70FFF70CFDB4F844101C
:10DBF000A06901442046FFF785FE002800D00120DF
:10DC000010BD0000525261417272416170B504460C
:10DC10000D464069E16D08B1012A09D06068012212
:10DC2000C36828469847002801D00120656570BD6B
:10DC30000B4600222946FEF78EFAF4E700000000AA
:10DC40003000002000000000000000009F050000E0
:10DC50000000000040480000010000001C000020FF
:10DC6000670000000000000002000000000000004B
:10DC700002E00000020000001C000020680000001C
:10DC800065000000280C00006500000002A00000F4
:10DC9000030000001C00002069000000D007000005
:10DCA000B80B0000DE0700000220000004000000A6
:10DCB0001C0000206A00000001000000E8030000D2
:10DCC0000100000002200000050000001C000020F0
:10DCD000650000000100000040420F00010000004C
:10DCE00002200000640000001C0000206B00000007
:10DCF0000A000000640000002800000012880000F4
:10DD0000650000003400002000000000000000005A
:10DD1000D0070000BC0200001150000066000000A7
:10DD20001C0000207A010000010000000A00000031
:10DD30000A000000022000006700000038000020F8
:10DD400000000000000000000A00000000000000C9
:10DD500001200000680000001C0000207B01000082
:10DD60000000000001000000000000000260000050
:10DD7000690000001C0000207C0100000000000081
:10DD80000100000000000000026000006A000000C6
:10DD90001C0000207D010000000000007800000051
:10DDA00005000000C24800006B0000001C000020BD
:10DDB0007E01000000000000D0070000D007000036
:10DDC000135000006C0000001C0000207F010000C8
:10DDD000000000009F050000000000004348000014
:10DDE0006D0000001C000020800100000000000009
:10DDF000D007000000000000135000006E0000007B
:10DE00001C00002081010000000000009F050000B0
:10DE100000000000434800006F0000001C000020CC
:10DE2000820100000000000001000000000000006E
:10DE300002600000700000001C0000208301000050
:10DE400001000000060000000100000002200000A8
:10DE5000710000001C000020840100000000000090
:10DE60009F05000000000000424800007200000012
:10DE70001C000020850100000000000001000000DF
:10DE80000100000002600000730000001C00002080
:10DE900086010000000000000100000000000000FA
:10DEA00002600000C80000005800002000000000D0
:10DEB00000000000D007000000000000115000002A
:10DEC000C90000005C00002000000000000000000D
:10DED000D00700000000000011500000CA00000040
:10DEE00060000020000000000000000001000000B1
:10DEF0000000000001600000CB0000006400002072
:10DF00000000000000000000010000000000000010
:10DF100001600000CC00000068000020000000004C
:10DF2000000000000100000000000000016000008F
:10DF3000CD0000006C000020000000000000000088
:10DF4000010000000000000001600000CE000000A1
:10DF50007000002000000000000000000A00000027
:10DF60000000000000200000CF000000740000202E
:10DF700000000000000000000100000000000000A0
:10DF800000600000D00000007800002000000000C9
:10DF900000000000D0070000000000002129000060
:10DFA000D10000007C000020000000000000000004
:10DFB000010000000000000000600000D20000002E
:10DFC00080000020000000000000000001000000B0
:10DFD0000000000000600000E80300001C000020BA
:10DFE0006C000000000000000400000000000000C1
:10DFF00002000000E90300001C0000206D0000008A
:10E00000BC020000B00400008403000012500000B5
:10E01000EA0300001C000020860000000100000050
:10E020002C0100000A000000C2480000EB030000C1
:10E030001C0000206E000000000000009F05000092
:10E040000000000042480000EC0300001C0000201B
:10E050006F000000000000009F05000000000000AD
:10E0600042480000ED0300001C000020700000008A
:10E0700001000000D00200003C0000004248000007
:10E08000EE0300001C0000207100000001000000F1
:10E09000D00200001E00000042480000EF03000014
:10E0A0001C00002072000000000000009F0500001E
:10E0B0000000000042480000F00300001C000020A7
:10E0C00073000000000000009F0500000000000039
:10E0D00042480000F10300001C0000207400000012
:10E0E00001000000D00200003C0000004248000097
:10E0F000F20300001C000020750000000100000079
:10E10000D00200001E00000042480000F30300009F
:10E110001C00002076000000000000009F050000A9
:10E120000000000042480000F40300001C00002032
:10E1300077000000000000009F05000000000000C4
:10E1400042480000F50300001C0000207800000099
:10E1500001000000D00200003C0000004248000026
:10E16000F60300001C000020790000000100000000
:10E17000D00200001E00000042480000F70300002B
:10E180001C0000207A000000000000009F05000035
:10E190000000000042480000F80300001C000020BE
:10E1A0007B000000000000009F0500000000000050
:10E1B00042480000F90300001C0000207C00000021
:10E1C00001000000D00200003C00000042480000B6
:10E1D000FA0300001C0000207D0000000100000088
:10E1E000D00200001E00000042480000FB030000B7
:10E1F0001C0000207E000000000000009F050000C1
:10E200000000000042480000FC0300001C00002049
:10E210007F000000000000009F05000000000000DB
:10E2200042480000FD0300001C00002080000000A8
:10E2300001000000D00200003C0000004248000045
:10E24000FE0300001C00002081000000010000000F
:10E25000D00200001E00000042480000FF03000042
:10E260001C00002082000000000000009F0500004C
:10E270000000000042480000000400001C000020D4
:10E2800083000000000000009F0500000000000067
:10E2900042480000010400001C000020840000002F
:10E2A00001000000D00200003C00000042480000D5
:10E2B000020400001C000020850000000100000096
:10E2C000D00200001E0000004248000003040000CD
:10E2D0001C0000208701000020202020FFFFFF7F7E
:10E2E00031302D5602480100D00700001C000020EC
:10E2F0008700000000000000040000000000000093
:10E3000002000000D10700001C000020880000006F
:10E31000BC020000B00400008403000012500000A2
:10E32000D20700001C000020A10000000100000036
:10E330002C0100000A000000C2480000D3070000C2
:10E340001C00002089000000000000009F05000064
:10E350000000000042480000D40700001C0000201C
:10E360008A000000000000009F050000000000007F
:10E3700042480000D50700001C0000208B00000070
:10E3800001000000D00200003C00000042480000F4
:10E39000D60700001C0000208C00000001000000D7
:10E3A000D00200001E00000042480000D707000015
:10E3B0001C0000208D000000000000009F050000F0
:10E3C0000000000042480000D80700001C000020A8
:10E3D0008E000000000000009F050000000000000B
:10E3E00042480000D90700001C0000208F000000F8
:10E3F00001000000D00200003C0000004248000084
:10E40000DA0700001C00002090000000010000005E
:10E41000D00200001E00000042480000DB070000A0
:10E420001C00002091000000000000009F0500007B
:10E430000000000042480000DC0700001C00002033
:10E4400092000000000000009F0500000000000096
:10E4500042480000DD0700001C000020930000007F
:10E4600001000000D00200003C0000004248000013
:10E47000DE0700001C0000209400000001000000E6
:10E48000D00200001E00000042480000DF0700002C
:10E490001C00002095000000000000009F05000007
:10E4A0000000000042480000E00700001C000020BF
:10E4B00096000000000000009F0500000000000022
:10E4C00042480000E10700001C0000209700000007
:10E4D00001000000D00200003C00000042480000A3
:10E4E000E20700001C00002098000000010000006E
:10E4F000D00200001E00000042480000E3070000B8
:10E500001C00002099000000000000009F05000092
:10E510000000000042480000E40700001C0000204A
:10E520009A000000000000009F05000000000000AD
:10E5300042480000E50700001C0000209B0000008E
:10E5400001000000D00200003C0000004248000032
:10E55000E60700001C0000209C00000001000000F5
:10E56000D00200001E00000042480000E707000043
:10E570001C0000209D000000000000009F0500001E
:10E580000000000042480000E80700001C000020D6
:10E590009E000000000000009F0500000000000039
:10E5A00042480000E90700001C0000209F00000016
:10E5B00001000000D00200003C00000042480000C2
:10E5C000EA0700001C000020A0000000010000007D
:10E5D000D00200001E00000042480000EB070000CF
:10E5E0001C0000208801000020202020FFFFFF7F6A
:10E5F00032302D5602480100B80B00001C000020EC
:10E60000A200000000000000040000000000000064
:10E6100002000000B90B00001C000020A300000055
:10E62000BC020000B004000084030000125000008F
:10E63000BA0B00001C000020BC000000010000001C
:10E640002C0100000A000000C2480000BB0B0000C3
:10E650001C000020A4000000000000009F05000036
:10E660000000000042480000BC0B00001C0000201D
:10E67000A5000000000000009F0500000000000051
:10E6800042480000BD0B00001C000020A600000056
:10E6900001000000D00200003C00000042480000E1
:10E6A000BE0B00001C000020A700000001000000BD
:10E6B000D00200001E00000042480000BF0B000016
:10E6C0001C000020A8000000000000009F050000C2
:10E6D0000000000042480000C00B00001C000020A9
:10E6E000A9000000000000009F05000000000000DD
:10E6F00042480000C10B00001C000020AA000000DE
:10E7000001000000D00200003C0000004248000070
:10E71000C20B00001C000020AB0000000100000044
:10E72000D00200001E00000042480000C30B0000A1
:10E730001C000020AC000000000000009F0500004D
:10E740000000000042480000C40B00001C00002034
:10E75000AD000000000000009F0500000000000068
:10E7600042480000C50B00001C000020AE00000065
:10E7700001000000D00200003C0000004248000000
:10E78000C60B00001C000020AF00000001000000CC
:10E79000D00200001E00000042480000C70B00002D
:10E7A0001C000020B0000000000000009F050000D9
:10E7B0000000000042480000C80B00001C000020C0
:10E7C000B1000000000000009F05000000000000F4
:10E7D00042480000C90B00001C000020B2000000ED
:10E7E00001000000D00200003C0000004248000090
:10E7F000CA0B00001C000020B30000000100000054
:10E80000D00200001E00000042480000CB0B0000B8
:10E810001C000020B4000000000000009F05000064
:10E820000000000042480000CC0B00001C0000204B
:10E83000B5000000000000009F050000000000007F
:10E8400042480000CD0B00001C000020B600000074
:10E8500001000000D00200003C000000424800001F
:10E86000CE0B00001C000020B700000001000000DB
:10E87000D00200001E00000042480000CF0B000044
:10E880001C000020B8000000000000009F050000F0
:10E890000000000042480000D00B00001C000020D7
:10E8A000B9000000000000009F050000000000000B
:10E8B00042480000D10B00001C000020BA000000FC
:10E8C00001000000D00200003C00000042480000AF
:10E8D000D20B00001C000020BB0000000100000063
:10E8E000D00200001E00000042480000D30B0000D0
:10E8F0001C0000208901000020202020FFFFFF7F56
:10E9000033302D5602480100A00F00001C000020EB
:10E91000BD00000000000000040000000000000036
:10E9200002000000A10F00001C000020BE0000003B
:10E93000BC020000B004000084030000125000007C
:10E94000A20F00001C000020D70000000100000002
:10E950002C0100000A000000C2480000A30F0000C4
:10E960001C000020BF000000000000009F05000008
:10E970000000000042480000A40F00001C0000201E
:10E98000C0000000000000009F0500000000000023
:10E9900042480000A50F00001C000020C10000003C
:10E9A00001000000D00200003C00000042480000CE
:10E9B000A60F00001C000020C200000001000000A3
:10E9C000D00200001E00000042480000A70F000017
:10E9D0001C000020C3000000000000009F05000094
:10E9E0000000000042480000A80F00001C000020AA
:10E9F000C4000000000000009F05000000000000AF
:10EA000042480000A90F00001C000020C5000000C3
:10EA100001000000D00200003C000000424800005D
:10EA2000AA0F00001C000020C6000000010000002A
:10EA3000D00200001E00000042480000AB0F0000A2
:10EA40001C000020C7000000000000009F0500001F
:10EA50000000000042480000AC0F00001C00002035
:10EA6000C8000000000000009F050000000000003A
:10EA700042480000AD0F00001C000020C90000004B
:10EA800001000000D00200003C00000042480000ED
:10EA9000AE0F00001C000020CA00000001000000B2
:10EAA000D00200001E00000042480000AF0F00002E
:10EAB0001C000020CB000000000000009F050000AB
:10EAC0000000000042480000B00F00001C000020C1
:10EAD000CC000000000000009F05000000000000C6
:10EAE00042480000B10F00001C000020CD000000D3
:10EAF00001000000D00200003C000000424800007D
:10EB0000B20F00001C000020CE0000000100000039
:10EB1000D00200001E00000042480000B30F0000B9
:10EB20001C000020CF000000000000009F05000036
:10EB30000000000042480000B40F00001C0000204C
:10EB4000D0000000000000009F0500000000000051
:10EB500042480000B50F00001C000020D10000005A
:10EB600001000000D00200003C000000424800000C
:10EB7000B60F00001C000020D200000001000000C1
:10EB8000D00200001E00000042480000B70F000045
:10EB90001C000020D3000000000000009F050000C2
:10EBA0000000000042480000B80F00001C000020D8
:10EBB000D4000000000000009F05000000000000DD
:10EBC00042480000B90F00001C000020D5000000E2
:10EBD00001000000D00200003C000000424800009C
:10EBE000BA0F00001C000020D60000000100000049
:10EBF000D00200001E00000042480000BB0F0000D1
:10EC00001C0000208A01000020202020FFFFFF7F41
:10EC100034302D5602480100881300001C000020EB
:10EC2000D800000000000000040000000000000008
:10EC300002000000891300001C000020D900000021
:10EC4000BC020000B0040000840300001250000069
:10EC50008A1300001C000020F200000001000000E8
:10EC60002C0100000A000000C24800008B130000C5
:10EC70001C000020DA000000000000009F050000DA
:10EC800000000000424800008C1300001C0000201F
:10EC9000DB000000000000009F05000000000000F5
:10ECA000424800008D1300001C000020DC00000022
:10ECB00001000000D00200003C00000042480000BB
:10ECC0008E1300001C000020DD0000000100000089
:10ECD000D00200001E000000424800008F13000018
:10ECE0001C000020DE000000000000009F05000066
:10ECF0000000000042480000901300001C000020AB
:10ED0000DF000000000000009F0500000000000080
:10ED100042480000911300001C000020E0000000A9
:10ED200001000000D00200003C000000424800004A
:10ED3000921300001C000020E10000000100000010
:10ED4000D00200001E0000004248000093130000A3
:10ED50001C000020E2000000000000009F050000F1
:10ED60000000000042480000941300001C00002036
:10ED7000E3000000000000009F050000000000000C
:10ED800042480000951300001C000020E400000031
:10ED900001000000D00200003C00000042480000DA
:10EDA000961300001C000020E50000000100000098
:10EDB000D00200001E00000042480000971300002F
:10EDC0001C000020E6000000000000009F0500007D
:10EDD0000000000042480000981300001C000020C2
:10EDE000E7000000000000009F0500000000000098
:10EDF00042480000991300001C000020E8000000B9
:10EE000001000000D00200003C0000004248000069
:10EE10009A1300001C000020E9000000010000001F
:10EE2000D00200001E000000424800009B130000BA
:10EE30001C000020EA000000000000009F05000008
:10EE400000000000424800009C1300001C0000204D
:10EE5000EB000000000000009F0500000000000023
:10EE6000424800009D1300001C000020EC00000040
:10EE700001000000D00200003C00000042480000F9
:10EE80009E1300001C000020ED00000001000000A7
:10EE9000D00200001E000000424800009F13000046
:10EEA0001C000020EE000000000000009F05000094
:10EEB0000000000042480000A01300001C000020D9
:10EEC000EF000000000000009F05000000000000AF
:10EED00042480000A11300001C000020F0000000C8
:10EEE00001000000D00200003C0000004248000089
:10EEF000A21300001C000020F1000000010000002F
:10EF0000D00200001E00000042480000A3130000D1
:10EF10001C0000208B01000020202020FFFFFF7F2D
:10EF200035302D5602480100701700001C000020EB
:10EF3000F3000000000000000400000000000000DA
:10EF400002000000711700001C000020F400000007
:10EF5000BC020000B0040000840300001250000056
:10EF6000721700001C0000200D01000001000000CD
:10EF70002C0100000A000000C248000073170000C6
:10EF80001C000020F5000000000000009F050000AC
:10EF90000000000042480000741700001C00002020
:10EFA000F6000000000000009F05000000000000C7
:10EFB00042480000751700001C000020F700000008
:10EFC00001000000D00200003C00000042480000A8
:10EFD000761700001C000020F8000000010000006F
:10EFE000D00200001E000000424800007717000019
:10EFF0001C000020F9000000000000009F05000038
:10F000000000000042480000781700001C000020AB
:10F01000FA000000000000009F0500000000000052
:10F0200042480000791700001C000020FB0000008F
:10F0300001000000D00200003C0000004248000037
:10F040007A1700001C000020FC00000001000000F6
:10F05000D00200001E000000424800007B170000A4
:10F060001C000020FD000000000000009F050000C3
:10F0700000000000424800007C1700001C00002037
:10F08000FE000000000000009F05000000000000DE
:10F09000424800007D1700001C000020FF00000017
:10F0A00001000000D00200003C00000042480000C7
:10F0B0007E1700001C00002000010000010000007D
:10F0C000D00200001E000000424800007F17000030
:10F0D0001C00002001010000000000009F0500004E
:10F0E0000000000042480000801700001C000020C3
:10F0F00002010000000000009F0500000000000069
:10F1000042480000811700001C000020030100009D
:10F1100001000000D00200003C0000004248000056
:10F12000821700001C000020040100000100000004
:10F13000D00200001E0000004248000083170000BB
:10F140001C00002005010000000000009F050000D9
:10F150000000000042480000841700001C0000204E
:10F1600006010000000000009F05000000000000F4
:10F1700042480000851700001C0000200701000025
:10F1800001000000D00200003C00000042480000E6
:10F19000861700001C00002008010000010000008C
:10F1A000D00200001E000000424800008717000047
:10F1B0001C00002009010000000000009F05000065
:10F1C0000000000042480000881700001C000020DA
:10F1D0000A010000000000009F0500000000000080
:10F1E00042480000891700001C0000200B010000AD
:10F1F00001000000D00200003C0000004248000076
:10F200008A1700001C0000200C0100000100000013
:10F21000D00200001E000000424800008B170000D2
:10F220001C0000208C01000020202020FFFFFF7F19
:10F2300036302D5602480100581B00001C000020EB
:10F240000E010000000000000400000000000000AB
:10F2500002000000591B00001C0000200F010000EC
:10F26000BC020000B0040000840300001250000043
:10F270005A1B00001C0000202801000001000000B3
:10F280002C0100000A000000C24800005B1B0000C7
:10F290001C00002010010000000000009F0500007D
:10F2A00000000000424800005C1B00001C00002021
:10F2B00011010000000000009F0500000000000098
:10F2C000424800005D1B00001C00002012010000ED
:10F2D00001000000D00200003C0000004248000095
:10F2E0005E1B00001C000020130100000100000054
:10F2F000D00200001E000000424800005F1B00001A
:10F300001C00002014010000000000009F05000008
:10F310000000000042480000601B00001C000020AC
:10F3200015010000000000009F0500000000000023
:10F3300042480000611B00001C0000201601000074
:10F3400001000000D00200003C0000004248000024
:10F35000621B00001C0000201701000001000000DB
:10F36000D00200001E00000042480000631B0000A5
:10F370001C00002018010000000000009F05000094
:10F380000000000042480000641B00001C00002038
:10F3900019010000000000009F05000000000000AF
:10F3A00042480000651B00001C0000201A010000FC
:10F3B00001000000D00200003C00000042480000B4
:10F3C000661B00001C0000201B0100000100000063
:10F3D000D00200001E00000042480000671B000031
:10F3E0001C0000201C010000000000009F05000020
:10F3F0000000000042480000681B00001C000020C4
:10F400001D010000000000009F050000000000003A
:10F4100042480000691B00001C0000201E01000083
:10F4200001000000D00200003C0000004248000043
:10F430006A1B00001C0000201F01000001000000EA
:10F44000D00200001E000000424800006B1B0000BC
:10F450001C00002020010000000000009F050000AB
:10F4600000000000424800006C1B00001C0000204F
:10F4700021010000000000009F05000000000000C6
:10F48000424800006D1B00001C000020220100000B
:10F4900001000000D00200003C00000042480000D3
:10F4A0006E1B00001C000020230100000100000072
:10F4B000D00200001E000000424800006F1B000048
:10F4C0001C00002024010000000000009F05000037
:10F4D0000000000042480000701B00001C000020DB
:10F4E00025010000000000009F0500000000000052
:10F4F00042480000711B00001C0000202601000093
:10F5000001000000D00200003C0000004248000062
:10F51000721B00001C0000202701000001000000F9
:10F52000D00200001E00000042480000731B0000D3
:10F530001C0000208D01000020202020FFFFFF7F05
:10F5400037302D5602480100401F00001C000020EB
:10F55000290100000000000004000000000000007D
:10F5600002000000411F00001C0000202A010000D2
:10F57000BC020000B0040000840300001250000030
:10F58000421F00001C000020430100000100000099
:10F590002C0100000A000000C2480000431F0000C8
:10F5A0001C0000202B010000000000009F0500004F
:10F5B0000000000042480000441F00001C00002022
:10F5C0002C010000000000009F050000000000006A
:10F5D00042480000451F00001C0000202D010000D3
:10F5E00001000000D00200003C0000004248000082
:10F5F000461F00001C0000202E010000010000003A
:10F60000D00200001E00000042480000471F00001A
:10F610001C0000202F010000000000009F050000DA
:10F620000000000042480000481F00001C000020AD
:10F6300030010000000000009F05000000000000F5
:10F6400042480000491F00001C000020310100005A
:10F6500001000000D00200003C0000004248000011
:10F660004A1F00001C0000203201000001000000C1
:10F67000D00200001E000000424800004B1F0000A6
:10F680001C00002033010000000000009F05000066
:10F6900000000000424800004C1F00001C00002039
:10F6A00034010000000000009F0500000000000081
:10F6B000424800004D1F00001C00002035010000E2
:10F6C00001000000D00200003C00000042480000A1
:10F6D0004E1F00001C000020360100000100000049
:10F6E000D00200001E000000424800004F1F000032
:10F6F0001C00002037010000000000009F050000F2
:10F700000000000042480000501F00001C000020C4
:10F7100038010000000000009F050000000000000C
:10F7200042480000511F00001C0000203901000069
:10F7300001000000D00200003C0000004248000030
:10F74000521F00001C0000203A01000001000000D0
:10F75000D00200001E00000042480000531F0000BD
:10F760001C0000203B010000000000009F0500007D
:10F770000000000042480000541F00001C00002050
:10F780003C010000000000009F0500000000000098
:10F7900042480000551F00001C0000203D010000F1
:10F7A00001000000D00200003C00000042480000C0
:10F7B000561F00001C0000203E0100000100000058
:10F7C000D00200001E00000042480000571F000049
:10F7D0001C0000203F010000000000009F05000009
:10F7E0000000000042480000581F00001C000020DC
:10F7F00040010000000000009F0500000000000024
:10F8000042480000591F00001C0000204101000078
:10F8100001000000D00200003C000000424800004F
:10F820005A1F00001C0000204201000001000000DF
:10F83000D00200001E000000424800005B1F0000D4
:10F840001C0000208E01000020202020FFFFFF7FF1
:10F8500038302D5602480100282300001C000020EB
:10F86000440100000000000004000000000000004F
:10F8700002000000292300001C00002045010000B8
:10F88000BC020000B004000084030000125000001D
:10F890002A2300001C0000205E010000010000007F
:10F8A0002C0100000A000000C24800002B230000C9
:10F8B0001C00002046010000000000009F05000021
:10F8C00000000000424800002C2300001C00002023
:10F8D00047010000000000009F050000000000003C
:10F8E000424800002D2300001C00002048010000B9
:10F8F00001000000D00200003C000000424800006F
:10F900002E2300001C00002049010000010000001F
:10F91000D00200001E000000424800002F2300001B
:10F920001C0000204A010000000000009F050000AC
:10F930000000000042480000302300001C000020AE
:10F940004B010000000000009F05000000000000C7
:10F9500042480000312300001C0000204C01000040
:10F9600001000000D00200003C00000042480000FE
:10F97000322300001C0000204D01000001000000A7
:10F98000D00200001E0000004248000033230000A7
:10F990001C0000204E010000000000009F05000038
:10F9A0000000000042480000342300001C0000203A
:10F9B0004F010000000000009F0500000000000053
:10F9C00042480000352300001C00002050010000C8
:10F9D00001000000D00200003C000000424800008E
:10F9E000362300001C00002051010000010000002F
:10F9F000D00200001E000000424800003723000033
:10FA00001C00002052010000000000009F050000C3
:10FA10000000000042480000382300001C000020C5
:10FA200053010000000000009F05000000000000DE
:10FA300042480000392300001C000020540100004F
:10FA400001000000D00200003C000000424800001D
:10FA50003A2300001C0000205501000001000000B6
:10FA6000D00200001E000000424800003B230000BE
:10FA70001C00002056010000000000009F0500004F
:10FA800000000000424800003C2300001C00002051
:10FA900057010000000000009F050000000000006A
:10FAA000424800003D2300001C00002058010000D7
:10FAB00001000000D00200003C00000042480000AD
:10FAC0003E2300001C00002059010000010000003E
:10FAD000D00200001E000000424800003F2300004A
:10FAE0001C0000205A010000000000009F050000DB
:10FAF0000000000042480000402300001C000020DD
:10FB00005B010000000000009F05000000000000F5
:10FB100042480000412300001C0000205C0100005E
:10FB200001000000D00200003C000000424800003C
:10FB3000422300001C0000205D01000001000000C5
:10FB4000D00200001E0000004248000043230000D5
:10FB50001C0000208F01000020202020FFFFFF7FDD
:10FB600039302D5602480100102700001C000020EB
:10FB70005F01000000000000040000000000000021
:10FB800002000000112700001C000020600100009E
:10FB9000BC020000B004000084030000125000000A
:10FBA000122700001C000020790100000100000065
:10FBB0002C0100000A000000C248000013270000CA
:10FBC0001C00002061010000000000009F050000F3
:10FBD0000000000042480000142700001C00002024
:10FBE00062010000000000009F050000000000000E
:10FBF00042480000152700001C000020630100009F
:10FC000001000000D00200003C000000424800005B
:10FC1000162700001C000020640100000100000005
:10FC2000D00200001E00000042480000172700001C
:10FC30001C00002065010000000000009F0500007E
:10FC40000000000042480000182700001C000020AF
:10FC500066010000000000009F0500000000000099
:10FC600042480000192700001C0000206701000026
:10FC700001000000D00200003C00000042480000EB
:10FC80001A2700001C00002068010000010000008D
:10FC9000D00200001E000000424800001B270000A8
:10FCA0001C00002069010000000000009F0500000A
:10FCB00000000000424800001C2700001C0000203B
:10FCC0006A010000000000009F0500000000000025
:10FCD000424800001D2700001C0000206B010000AE
:10FCE00001000000D00200003C000000424800007B
:10FCF0001E2700001C0000206C0100000100000015
:10FD0000D00200001E000000424800001F27000033
:10FD10001C0000206D010000000000009F05000095
:10FD20000000000042480000202700001C000020C6
:10FD30006E010000000000009F05000000000000B0
:10FD400042480000212700001C0000206F01000035
:10FD500001000000D00200003C000000424800000A
:10FD6000222700001C00002070010000010000009C
:10FD7000D00200001E0000004248000023270000BF
:10FD80001C00002071010000000000009F05000021
:10FD90000000000042480000242700001C00002052
:10FDA00072010000000000009F050000000000003C
:10FDB00042480000252700001C00002073010000BD
:10FDC00001000000D00200003C000000424800009A
:10FDD000262700001C000020740100000100000024
:10FDE000D00200001E00000042480000272700004B
:10FDF0001C00002075010000000000009F050000AD
:10FE00000000000042480000282700001C000020DD
:10FE100076010000000000009F05000000000000C7
:10FE200042480000292700001C0000207701000044
:10FE300001000000D00200003C0000004248000029
:10FE40002A2700001C0000207801000001000000AB
:10FE5000D00200001E000000424800002B270000D6
:10FE60001C0000209001000020202020FFFFFF7FC9
:10FE700030312D5602480100FFFF00000000000055
:10FE80000000000000000000000000000000000072
:10FE9000000000000000000054220E0001000000DD
:10FEA0000A0000002A070D000200000014000000F4
:10FEB000E7030C00030000001E00000064160B00A6
:10FEC0000400000028000000AF3C0A00050000000C
:10FED0003200000004750900070000003C0000002B
:10FEE000CBBD080008000000460000009115080086
:10FEF0000A00000050000000077B07000B00000014
:10FF00005A000000FCEC06000D0000006400000038
:10FF10005A6A06000F0000006E00000028F205007B
:10FF200011000000780000007F830500130000002E
:10FF300082000000921D0500160000008C000000E9
:10FF4000A2BF04001800000096000000046904002D
:10FF50001B000000A00000001B1904001D00000091
:10FF6000AA00000058CF030021000000B4000000E8
:10FF70003A8B030024000000BE000000494C03003F
:10FF800027000000C80000001A1203002B00000028
:10FF9000D20000004ADC02002F000000DC0000005C
:10FFA0007DAA020033000000E6000000637C02002E
:10FFB00037000000F0000000AE5102003C000000DD
:10FFC000FA0000001A2A02004100000004010000AB
:10FFD00069050200460000000E0100005FE3010019
:10FFE0004C00000018010000C8C3010052000000CE
:10FFF0002201000073A60100580000002C0100003F
:020000040802F0
:10000000348B01005F00000036010000E171010047
:100010006600000040010000565A01006E0000001A
:100020004A0100006F440100760000005401000006
:100030000D3001007E0000005E010000131D010074
:100040008700000068010000660B010090000000BE
:1000500072010000EDFA00009A0000007C0100002F
:1000600091EB0000A4000000860100003EDD0000CE
:10007000AF00000090010000E0CF0000BA000000D7
:100080009A01000066C30000C6000000A401000041
:10009000BFB70000D3000000AE010000DCAC0000E0
:1000A000E0000000B8010000AFA20000EE00000078
:1000B000C20100002B990000FC000000CC010000F0
:1000C000449000000C010000D6010000EF87000002
:1000D0001B010000E0010000228000002C01000054
:1000E000EA010000D47800003D010000F4010000A6
:1000F000FC7100004F010000FE010000916B000048
:1001000062010000080200008D6500007601000019
:1001100012020000E85F00008B0100001C020000DA
:100120009C5A0000A001000026020000A355000018
:10013000B601000030020000F8500000CD010000C0
:100140003A020000944C0000E50100004402000067
:1001500075480000FE0100004E02000094440000BB
:100160001702000058020000EE40000032020000BA
:1001700062020000803D00004D0200006C020000A1
:10018000453A000069020000760200003A3700009C
:1001900087020000800200005D340000A50200001C
:1001A0008A020000AA310000C4020000940200008C
:1001B0001E2F0000E40200009E020000B82C000088
:1001C00005030000A8020000752A000026030000B5
:1001D000B20200005228000049030000BC020000E7
:1001E0004E2600006C030000C602000067240000D9
:1001F00090030000D00200009B220000B503000025
:10020000DA020000E8200000DB030000E402000046
:100210004D1F000002040000EE020000C91D000096
:1002200029040000F8020000591C000051040000DD
:1002300002030000FD1A00007A0400000C03000015
:10024000B4190000A4040000160300007D1800008B
:10025000CD0400002003000056170000F804000041
:100260002A0300003F1600002305000034030000AD
:10027000361500004F0500003E0300003B1400004F
:100280007B050000480300004D130000A805000096
:10029000520300006B120000D50500005C03000053
:1002A000951100000206000066030000CA1000005D
:1002B0002F06000070030000091000005D0600001A
:1002C0007A030000520F00008B0600008403000038
:1002D000A40E0000B90600008E030000FF0D000010
:1002E000E806000098030000620D000016070000F9
:1002F000A2030000CD0C000044070000AC03000086
:100300003F0C000072070000B6030000B80B0000AD
:10031000A0070000C0030000380B0000CE0700005B
:10032000CA030000BD0A0000FC070000D40300005F
:10033000490A00002A080000DE030000DA09000074
:1003400057080000E803000071090000840800005D
:10035000F20300000C090000B1080000FC030000DB
:10036000AC080000DD080000060400005108000091
:100370000909000010040000FA0700003509000018
:100380001A040000A7070000600900002404000010
:10039000580700008A0900002E0400000C07000026
:1003A000B409000038040000C4060000DE090000A3
:1003B000420400007F060000070A00004C04000011
:1003C0003D0600002F0A000056040000FF05000053
:1003D000560A000060040000C30500007D0A00000A
:1003E0006A04000089050000A40A000074040000EB
:1003F00053050000CA0A00007E0400001E0500002C
:10040000EF0A000088040000EC040000130B000059
:1004100092040000BC040000370B00009C040000A4
:100420008E0400005A0B0000A604000063040000C4
:100430007C0B0000B0040000390400009E0B00009B
:10044000BA04000010040000BE0B0000C404000049
:10045000EA030000DF0B0000CE040000C50300002B
:10046000FE0B0000D8040000A20300001D0C0000D9
:10047000E2040000800300003B0C0000EC040000DC
:100480005F030000580C0000F60400004003000069
:10049000750C00000005000023030000910C000013
:1004A0000A05000006030000AC0C00001405000063
:1004B000EB020000C70C00001E050000D002000087
:1004C000E00C000028050000B7020000FA0C000054
:1004D000320500009F020000120D00003C050000E4
:1004E000880200002A0D000046050000710200008D
:1004F000420D0000500500005C020000580D000095
:100500005A050000470200006E0D0000640500005F
:1005100033020000840D00006E0500002002000080
:10052000990D0000780500000E020000AD0D0000DE
:1005300082050000FC010000C10D00008C050000D8
:10054000EC010000D40D000096050000DB01000066
:10055000E70D0000A0050000CC010000F90D00002F
:10056000AA050000BD0100000B0E0000B40500004C
:10057000AE0100001C0E0000BE050000A00100003E
:100580002D0E0000C8050000930100003D0E000084
:10059000D2050000860100004D0E0000DC050000C1
:1005A000790100005C0E0000E60500006E0100000D
:1005B0006B0E0000F005000062010000790E0000E3
:1005C000FA05000057010000870E00000406000035
:1005D0004C010000950E00000E06000042010000D4
:1005E000A20E00001806000038010000AF0E000047
:1005F000220600002E010000BB0E00002C060000A9
:1006000025010000C70E0000360600001C01000096
:10061000D30E00004006000013010000DE0E0000B3
:100620004A0600000B010000E90E0000540600001D
:1006300003010000F40E00005E060000FB00000055
:10064000FE0E000068060000F4000000080F000025
:1006500072060000ED000000120F00007C06000092
:10066000E60000001C0F000086060000DF0000000E
:10067000250F000090060000D90000002E0F00009A
:100680009A060000D2000000360F0000A406000009
:10069000CC0000003F0F0000AE060000C6000000C6
:1006A000470F0000B8060000C10000004F0F000017
:1006B000C2060000BB000000570F0000CC0600007F
:1006C000B60000005E0F0000D6060000B10000007A
:1006D000650F0000E0060000AC0000006D0F000098
:1006E000EA060000A7000000730F0000F4060000F7
:1006F000A20000007A0F0000FE0600009E0000002D
:10070000800F0000080700009A000000860F00001C
:1007100012070000950000008D0F00001C0700006C
:1007200091000000930F0000260700008D000000DC
:10073000980F0000300700008A0000009E0F0000A4
:100740003A07000086000000A30F000044070000E5
:1007500082000000A80F00004E0700007F0000008C
:10076000AE0F0000580700007C000000B20F000030
:100770006207000078000000B70F00006C0700005F
:1007800075000000BC0F000076070000720000003A
:10079000C10F0000800700006F000000C50F0000BF
:1007A0008A0700006C000000C90F000094070000D9
:1007B00069000000CD0F00009E07000067000000E8
:1007C000D10F0000A807000064000000D50F000052
:1007D000B207000062000000D90F0000BC07000053
:1007E0005F000000DD0F0000C60700005D00000094
:1007F000E00F0000D00700005A000000E40F0000E6
:10080000DA07000058000000E70F0000E4070000CE
:1008100056000000EB0F0000EE070000540000003F
:10082000EE0F0000F807000052000000F10F00007A
:100830000208000050000000F40F00000C08000047
:100840004E000000F70F0000160800004C000000EA
:10085000FA0F0000200800004A000000FD0F000011
:100860002A08000048000000FF0F000034080000C4
:1008700047000000021000000000000021100000EE
:10088000422000006330000084400000A5500000BA
:10089000C6600000E7700000088100002991000098
:1008A0004AA100006BB100008CC10000ADD1000076
:1008B000CEE10000EFF10000311200001002000054
:1008C0007332000052220000B55200009442000032
:1008D000F7720000D6620000399300001883000010
:1008E0007BB300005AA30000BDD300009CC30000EE
:1008F000FFF30000DEE30000622400004334000048
:100900002004000001140000E6640000C774000029
:10091000A4440000855400006AA500004BB5000007
:100920002885000009950000EEE50000CFF50000E5
:10093000ACC500008DD500005336000072260000C3
:100940001116000030060000D7760000F6660000A1
:1009500095560000B44600005BB700007AA700007F
:100960001997000038870000DFF70000FEE700005D
:100970009DD70000BCC70000C4480000E558000037
:1009800086680000A7780000400800006118000099
:100990000228000023380000CCC90000EDD9000077
:1009A0008EE90000AFF90000488900006999000055
:1009B0000AA900002BB90000F55A0000D44A000033
:1009C000B77A0000966A0000711A0000500A000011
:1009D000333A0000122A0000FDDB0000DCCB0000EF
:1009E000BFFB00009EEB0000799B0000588B0000CD
:1009F0003BBB00001AAB0000A66C0000877C000027
:100A0000E44C0000C55C0000222C0000033C000008
:100A1000600C0000411C0000AEED00008FFD0000E6
:100A2000ECCD0000CDDD00002AAD00000BBD0000C4
:100A3000688D0000499D0000977E0000B66E0000A2
:100A4000D55E0000F44E0000133E0000322E000080
:100A5000511E0000700E00009FFF0000BEEF00005E
:100A6000DDDF0000FCCF00001BBF00003AAF00003C
:100A7000599F0000788F000088910000A981000034
:100A8000CAB10000EBA100000CD100002DC1000094
:100A90004EF100006FE1000080100000A100000096
:100AA000C2300000E3200000045000002540000098
:100AB0004670000067600000B98300009893000052
:100AC000FBA30000DAB300003DC300001CD300000C
:100AD0007FE300005EF30000B1020000901200000E
:100AE000F3220000D2320000354200001452000010
:100AF0007762000056720000EAB50000CBA5000046
:100B0000A8950000898500006EF500004FE5000003
:100B10002CD500000DC50000E2340000C324000005
:100B2000A014000081040000667400004764000007
:100B30002454000005440000DBA70000FAB70000C1
:100B400099870000B89700005FE700007EF700007B
:100B50001DC700003CD70000D3260000F23600007D
:100B600091060000B016000057660000767600007F
:100B700015460000345600004CD900006DC9000035
:100B80000EF900002FE90000C8990000E989000073
:100B90008AB90000ABA90000445800006548000075
:100BA0000678000027680000C0180000E108000077
:100BB00082380000A32800007DCB00005CDB000031
:100BC0003FEB00001EFB0000F98B0000D89B0000EB
:100BD000BBAB00009ABB0000754A0000545A0000ED
:100BE000376A0000167A0000F10A0000D01A0000EF
:100BF000B32A0000923A00002EFD00000FED000025
:100C00006CDD00004DCD0000AABD00008BAD0000E2
:100C1000E89D0000C98D0000267C0000076C0000E4
:100C2000645C0000454C0000A23C0000832C0000E6
:100C3000E01C0000C10C00001FEF00003EFF0000A0
:100C40005DCF00007CDF00009BAF0000BABF00005A
:100C5000D98F0000F89F0000176E0000367E00005C
:100C6000554E0000745E0000932E0000B23E00005E
:100C7000D10E0000F01E0000000000000000000087
:100C800000005F00000000000007000700000000F7
:100C9000147F147F14000000242A7F2A1200000011
:100CA000231308646200000036495522400000000A
:100CB0000005030000000000001C224100000000AD
:100CC0000041221C0000000014083E08140000002F
:100CD00008083E0808000000005030000000000036
:100CE000080808080800000000606000000000001C
:100CF00020100804020000003E4141413E00000077
:100D000000427F400000000042615149460000005F
:100D10002141454B310000001814127F10000000E3
:100D200027454545390000003C4A4949300000004C
:100D300001710905030000003649494936000000E9
:100D4000064949291E000000000036360000000058
:100D50000056360000000000081C3E7F0000000026
:100D60001414141414000000007F3E1C080000003E
:100D70000201510906000000324979413E0000009D
:100D80007E1111117E0000007F49494936000000A4
:100D90003E414141220000007F4141221C000000F1
:100DA0007F494949410000007F090909010000000D
:100DB0003E4149493A0000007F0808087F000000D2
:100DC00000417F41000000002040413F0100000041
:100DD0007F081422410000007F4040404000000096
:100DE0007F020C027F0000007F0408107F000000DB
:100DF0003E4141413E0000007F0909090600000014
:100E00003E4151215E0000007F0919294600000083
:100E1000464949493100000001017F0101000000FD
:100E20003F4040403F0000001F2040201F000000C6
:100E30003F4070403F00000063140814630000004E
:100E40000708700807000000615149454300000091
:100E5000007F414100000000020408102000000053
:100E60000041417F00000000040201020400000074
:100E7000404040404000000000010200000000002F
:100E800020545454780000007F444444380000004B
:100E90003844444420000000384444487F000000A7
:100EA0003854545418000000087E09010200000064
:100EB00018A4A4A47C0000007F08040478000000AB
:100EC00000447D40000000002040443D0000000040
:100ED0007F1028440000000000417F400000000017
:100EE0007C041804780000007C08040478000000EA
:100EF0003844444438000000FC2424241800000036
:100F0000081414147C0000007C080404080000008D
:100F10004854545420000000043F44402000000086
:100F20003C4040207C0000001C2040201C000000B1
:100F30003C4020403C0000004428102844000000B1
:100F40000C5050503C0000004464544C44000000DD
:100F5000000609090600000000007F0000000000F4
:100F6000414136080000000015150A00000000008D
:100F7000000609090600000015150A00000000001F
:100F8000087C424141427C0804150E04307F7F30CA
:100F90006373160834676300FFFFFFFFFFFFFFFF67
:100FA00082868E9EBEFE8080FEBE9E8E8682808061
:100FB000406070787C7E00007E7C7870604000002D
:100FC00080808080808080801C22617169221C006A
:100FD000000808082A1C080000000000307F7F304D
:100FE00004150E2450022550000000205002255008
:100FF00000000000000000000000000000000000F1
:1010000000000000000000000000000000000000E0
:1010100000000000000000000000000000000000D0
:1010200000000000000000000000000000000000C0
:1010300000000000000000000000000000000000B0
:1010400000000000000000000000000000000000A0
:101050000000000000000000000000000000000090
:101060000000000000000000000000000000000080
:101070000000000000000000000000000000000070
:101080000000000000000000000000000000000060
:101090000000000000000000000000000000000050
:1010A0000000000000000000000000000000000040
:1010B0000000000000000000000000000000000030
:1010C0000000000000000000000000000000000020
:1010D0000000000000000000000000000000000010
:1010E0000000000000000000000000000000000000
:1010F00000000000000000000000000000000000F0
:1011000000000000000000000000000000000000DF
:1011100000000000000000000000000000000000CF
:1011200000000000000000000000000000000000BF
:1011300000000000000000000000000000000000AF
:1011400000000000000000007F05157A500000003C
:10115000000000000000000000000000000000008F
:10116000000000000000000000000000000000007F
:10117000000000000000000000000000000000006F
:10118000000000000000000000000000000000005F
:1011900000000000000000007029242970000000F9
:1011A000702A252A700000007E097F49490000004E
:1011B0000E515171110000000000000000000000FD
:1011C0007C54565544000000000000000000000060
:1011D000000000000000000000000000000000000F
:1011E00000000000000000000000000000000000FF
:1011F00000000000000000000000000000000000EF
:10120000487E494942000000000000000000000044
:1012100000000000000000000000000000000000CE
:1012200000000000000000003D4242423D0000007E
:1012300000000000000000000000000000000000AE
:10124000000000000000000000000000000000009E
:1012500000000000000000003C4140413C00000054
:10126000000000000000000000000000000000007E
:10127000809CA2A2A29C8080205556547800000039
:10128000205456557800000020565556780000002E
:10129000809CBEBEBE9C80802055545578000000C6
:1012A000205455547800000024547854580000000D
:1012B0000C525272120000003855565418000000AB
:1012C000385456551800000038565556180000007E
:1012D000385554551800000000497A4000000000BD
:1012E00000487A4100000000004A794200000000F6
:1012F00000457C41000000007C141C007C140000B0
:101300001C227F222200000030494A4830000000A1
:1013100030484A4930000000304A494A3000000055
:101320001C007C08087C0000304A484A300000005D
:101330004122140814224100001C2222221C000019
:1013400038414220780000003840422178000000F7
:1013500038424122780000003842402278000000E4
:101360004100000000000000001C3E3E3E1C00004A
:101370000C5150513C000000000000000000000033
:10138000000000000000000000000000000000005D
:10139000000000000000000000000000000000004D
:1013A00000FFFF000000000000000000000000003F
:1013B000006767000000000000000000000000005F
:1013C000001F1F001F1F00000000000000000000A1
:1013D000000000000000000000000000000000000D
:1013E0001010FF101010FF1010000000000000008F
:1013F00002023F0202023F02020000000000000061
:10140000387C66C6FFC6C68C0000000000000000E5
:101410000C1818187F180F070000000000000000CB
:101420003E414141BE402010080400000000000081
:1014300008040201003E4141413E0000000000005E
:1014400000E010101010000000000000000000007C
:101450003C624146283C4240000000000000000081
:10146000001F1F000000000000000000000000003E
:10147000000000000000000000000000000000006C
:1014800000F0FE0F0100000000000000000000005E
:1014900000073F784000000000000000000000004E
:1014A000000000010FFEF00000000000000000003E
:1014B00000000040783F070000000000000000002E
:1014C000000000800000000000000000000000009C
:1014D00021120C7F0C12210000000000000000000F
:1014E00000000000E0E0000000000000000000003C
:1014F000060606067F7F06060606000000000000BE
:1015000000000000000000000000000000000000DB
:10151000005838000000000000000000000000003B
:1015200000808080808080808080800000000000BB
:1015300000010101010101010101010000000000A1
:10154000000000000000000000000000000000009B
:10155000000000003030000000000000000000002B
:10156000000080601C03000000000000000000007C
:10157000601C0300000000000000000000000000EC
:10158000F8FE0703030307FEF80000000000000058
:101590000F3F70606060703F0F00000000000000AF
:1015A00000000C0C0CFFFF00000000000000000019
:1015B00000006060607F7F606060000000000000ED
:1015C0000603030303C7FE3C000000000000000008
:1015D00070786C666361606060000000000000006D
:1015E000060303C3C3C3E7BE1C00000000000000E5
:1015F000306060606060713F1F000000000000000C
:1016000080C070380C06FFFF0000000000000000E2
:101610000303030303037F7F0303000000000000B4
:1016200000FFFFC3C3C3C38303000000000000002A
:10163000306060606060313F0F000000000000001B
:10164000F0FCCE636363E7CE8C0000000000000076
:101650000F3F30606060703F0F000000000000002E
:101660000303030303C3F33F0F0000000000000067
:101670000040703C0F03000000000000000000006C
:101680003CFEE7C3C3C3C73E1C00000000000000CF
:101690001E3F70606060713F1E000000000000008F
:1016A000F8FE8703030306FEF800000000000000B8
:1016B000006163636333391F030000000000000012
:1016C00000000E0E000000000000000000000000FE
:1016D00000000E0E000000000000000000000000EE
:1016E00000000707000000000000000000000000EC
:1016F00000607E0F010000000000000000000000FC
:1017000000000000808080C0C000000000000000D9
:101710000E0E1B1B31313160600000000000000024
:10172000C0C0C0C0C0C0C0C0C000000000000000F9
:101730000C0C0C0C0C0C0C0C0C000000000000003D
:10174000606060C0C080C080000000000000000039
:1017500030303018180D0D0D070700000000000094
:101760000603038383C77E3C0000000000000000E6
:10177000000067670000000000000000000000009B
:101780000000000101010000000000000000000056
:101790000000000000000000000000000000000049
:1017A000FCFEC7C3C3C3C3C7FEFC000000000000AB
:1017B0000F0F0000000000000F0F000000000000ED
:1017C000FFFF63636363F3F79E0C000000000000FB
:1017D0000F0F0C0C0C0C0C0E070300000000000097
:1017E000FCFE0703030303070604000000000000DB
:1017F00003070E0C0C0C0C0E06020000000000008B
:10180000FFFF03030307060EFCF8000000000000C2
:101810000F0F0C0C0C0E0607030100000000000067
:1018200000FFFF63636363630300000000000000C8
:10183000000F0F0C0C0C0C0C0C0000000000000042
:1018400000FFFF6363636303030000000000000008
:10185000000F0F000000000000000000000000006A
:10186000FCFE07030303C3C7C6C40000000000005A
:1018700003070E0C0C0C0C0E070300000000000008
:10188000FFFF606060606060FFFF0000000000001C
:101890000F0F0000000000000F0F0000000000000C
:1018A00000000303FFFF030300000000000000002E
:1018B00000000C0C0F0F0C0C0000000000000000DA
:1018C0000000000303FFFF0303000000000000000E
:1018D00003070E0C0E0703000000000000000000CC
:1018E000FFFF60F0980C06030100000000000000FC
:1018F0000F0F00000103060C0800000000000000AC
:101900000000FFFF000000000000000000000000D9
:1019100000000F0F0C0C0C0C000000000000000079
:10192000FFFF060C38380C06FFFF00000000000027
:101930000F0F0000000000000F0F0000000000006B
:10194000FFFF183060C08000FFFF000000000000B3
:101950000F0F0000000001030F0F00000000000047
:10196000FCFE070303030307FEFC00000000000069
:1019700003070E0C0C0C0C0E070300000000000007
:10198000FFFFC3C3C3C3C3E77E3C000000000000E9
:101990000F0F000000000000000000000000000029
:1019A000FCFE070303838307FEFC00000000000029
:1019B00003070E0C0C0C0D07070D000000000000C3
:1019C000FFFF6363E3E363773E1C00000000000059
:1019D0000F0F0000000103060C08000000000000CB
:1019E0001C3E7763636363E3C38000000000000074
:1019F0000C0C0C0C0C0C0C0E07030000000000007B
:101A000003030303FFFF03030303000000000000C0
:101A1000000000000F0F00000000000000000000A8
:101A2000FFFF00000000000000FFFF0000000000BA
:101A300003070E0C0C0C0C0C0E070300000000003A
:101A4000FFFF000000000000FFFF0000000000009A
:101A5000000103060C0C060301000000000000005A
:101A6000FFFF000080800000FFFF0000000000007A
:101A70000103060C07070C0603010000000000002C
:101A8000070F98F06060F0980F070000000000005A
:101A90000E0F0100000000010F0E0000000000000A
:101AA0001F3F60C08080C0603F1F0000000000003A
:101AB000000000000F0F0000000000000000000008
:101AC000030383C363331B0F070000000000000003
:101AD0000E0F0D0C0C0C0C0C0C0000000000000094
:101AE00000FFFF01010100000000000000000000F5
:101AF000007F7F4040400000000000000000000028
:101B0000010FFFF0000000000000000000000000D6
:101B10000000000F7F7000000000000000000000C7
:101B2000010101FFFF0000000000000000000000B4
:101B30004040407F7F0000000000000000000000E7
:101B40006070180C0603060C18706000000000009E
:101B50000000000000000000000000000000000085
:101B60000000000000000000000000000000000075
:101B700060606060606060606060000000000000A5
:101B8000000002060E080000000000000000000037
:101B90000000000000000000000000000000000045
:101BA0000080D8D8D8D8D8F8F00000000000000095
:101BB00000070F0C0C0C060F0F00000000000000C7
:101BC000FFFF3018181838F0E00000000000000097
:101BD0000F0F060C0C0C0E070300000000000000A5
:101BE000E0F0301818181830200000000000000045
:101BF0000307060C0C0C0C0602000000000000009D
